:100000000C9458110C9489110C9489110C94891139
:100010000C9489110C9489110C9489110C948911F8
:100020000C9489110C9489110C9489110C948911E8
:100030000C9489110C946DB60C9489110C9489114F
:100040000C9489110C94A1640C9489110C9489115D
:100050000C9489110C9489110C9449750C945BB023
:100060000C9489110C9472150C9489110C948911BB
:100070000C9489110C9489110C9489110C94891198
:100080000C9489110C9489110C9489110C94891188
:100090000C9489110C9489110C9489110C94891178
:1000A0000C9489110C9489110C9489110C94891168
:1000B0000C9489110C9489110C9489110C94891158
:1000C0000C9489110C9489110C9489110C94891148
:1000D0000C9489110C9489110C9489110C94891138
:1000E0000C948911C075CE75EA75F9751376217671
:1000F0003B763F76E0A9FDA9FFA90BAA11AA14AA95
:100100001EAA91B196B19BB1A5B1AFB128B2B9B158
:10011000C1B1C9B1D3B1DDB1E7B1F6B100B228B216
:100120000AB214B21EB24AB24DB23CB240B246B2AA
:1001300084B251B255B25BB25FB263B269B26DB212
:1001400071B284B277B27BB27FB2084AD73B3BCE62
:10015000016E84BCBFFDC12F3D6C74319ABD5683C6
:100160003DDA3D00C77F11BED9E4BB4C3E916BAA7E
:10017000AABE000000803F05A84CCDB2D44EB938CD
:1001800036A9020C50B9918688083CA6AAAA2ABEB4
:10019000000000803F0048617264636F6465642002
:1001A00044656661756C742053657474696E677319
:1001B000204C6F616465640053746F7265642073D2
:1001C000657474696E6773207265747269657665AB
:1001D000640053657474696E67732053746F72653D
:1001E00064006563686F3A004B494C4C45442E20CF
:1001F000005072696E7465722068616C7465642E5B
:10020000206B696C6C28292063616C6C656421002B
:100210006F6B00526573656E643A20002200556E64
:100220006B6E6F776E20636F6D6D616E643A202226
:1002300000486F74656E64206F6666736574733A08
:10024000007A5F6D696E3A2000795F6D696E3A20C1
:1002500000785F6D696E3A20005A3A00593A0020E2
:10026000436F756E7420583A00453A005A3A005967
:100270003A00583A004649524D574152455F4E4167
:100280004D453A4D54312E355F33445072696E748A
:1002900065725F50524F4752414D20564552534967
:1002A0004F4E3A312E313033204558545255444543
:1002B000525F434F554E543A32204D414348494EC8
:1002C000455F545950453A5265705261702020572D
:1002D0006562736974653A687474703A2F2F777722
:1002E000772E6D756C746F6F2E636F6D200A0042F0
:1002F000656420646F6E652E0020423A0020543100
:100300003A0054303A004265642048656174696E71
:10031000672E0048656174696E6720646F6E652E94
:100320000020573A002054313A0054303A004865D2
:100330006174696E672E2E2E002042403A002040E4
:100340003A00202F0020423A00202F002054313A5A
:1003500000202F006F6B2054303A002569206D6912
:100360006E2C2025692073656300456E64206669E4
:100370006C65206C69737400426567696E206669FC
:100380006C65206C697374004E6F206D6F76652EFE
:10039000005072696E74696E67202E2E2E005761B0
:1003A000697420666F7220757365722E2E2E004D53
:1003B000303500536C6565702E2E2E0046696E69CF
:1003C000736865642E00446F6E65207072696E7488
:1003D000696E672066696C6500473332310053549B
:1003E0004F505045442E20005072696E7465722043
:1003F00073746F707065642064756520746F206518
:1004000072726F72732E2046697820746865206559
:1004100072726F7220616E6420757365204D393978
:100420003920746F20726573746172742E202854A1
:10043000656D70657261747572652069732072658F
:100440007365742E20536574206974206166746529
:10045000722072657374617274696E6729006F6BC4
:10046000004E6F204C696E65204E756D626572207E
:100470007769746820636865636B73756D2C204CB5
:10048000617374204C696E653A20004E6F2043689A
:1004900065636B73756D2077697468206C696E6530
:1004A000206E756D6265722C204C617374204C69EE
:1004B0006E653A2000636865636B73756D206D69C6
:1004C000736D617463682C204C617374204C696E89
:1004D000653A20004C696E65204E756D626572202C
:1004E0006973206E6F74204C617374204C696E6563
:1004F000204E756D6265722B312C204C6173742017
:100500004C696E653A20004D31313000446F6E65A4
:1005100020736176696E672066696C652E006F6B6B
:10052000004D3239002020506C616E6E657242754C
:100530006666657242797465733A2000204672657A
:1005400065204D656D6F72793A20004175672032E4
:1005500031203230313700436F6D70696C65643A19
:1005600020004D554C544F4F00207C20417574683D
:100570006F723A20004175672032312032303137B6
:100580002031393A34393A303200204C61737420CA
:10059000557064617465643A20004D54312E350005
:1005A00020536F66747761726520526573657400BD
:1005B000205761746368646F6720526573657400C7
:1005C0002042726F776E206F757420526573657468
:1005D000002045787465726E616C20526573657495
:1005E00000506F77657255700073746172740022E9
:1005F00000656E717565696E672022002200656E68
:10060000717565696E67202200FFFFFF0000A04042
:100610000000A0400000803F00000000000000003B
:10062000000000006563686F3A004572726F723AAD
:10063000007C3C3E5E2B3D3F2F5B5D3B2C2A225CC9
:10064000004D383420582059205A2045004D32346E
:10065000004D3233202573006175746F25692E6754
:10066000006572726F722077726974696E672074A8
:100670006F2066696C65004E6F7420534420707261
:10068000696E74696E67002F005344207072696E42
:1006900074696E67206279746520002E0044656C71
:1006A0006574696F6E206661696C65642C204669AB
:1006B0006C653A200046696C652064656C657465FC
:1006C000643A002E006F70656E206661696C656427
:1006D0002C2046696C653A200057726974696E6710
:1006E00020746F2066696C653A20002E006F70657B
:1006F0006E206661696C65642C2046696C653A20E1
:10070000002E006F70656E206661696C65642C2038
:1007100046696C653A200046696C652073656C65B6
:1007200063746564002053697A653A200046696CF9
:1007300065206F70656E65643A20002E006F7065ED
:100740006E206661696C65642C2046696C653A2090
:100750000053442063617264206F6B006F70656E9C
:10076000526F6F74206661696C656400766F6C759A
:100770006D652E696E6974206661696C65640053ED
:100780004420696E6974206661696C006563686FF6
:100790003A004572726F723A0020746F6F206C6F6E
:1007A0006E6720657874727573696F6E20707265FC
:1007B00076656E7465640020636F6C642065787480
:1007C000727573696F6E2070726576656E7465649C
:1007D000006563686F3A00656E6473746F707320B0
:1007E0006869743A205A00205A3A00656E6473743E
:1007F0006F7073206869743A20590020593A006577
:100800006E6473746F7073206869743A20580020A6
:10081000583A00656E6473746F7073206869743A37
:10082000200024F4D43050C38E20C2A24017828B03
:100830007011127A910D816CD90AA861E108C7582C
:100840006607615143061E4B5D05C145A7041A4169
:100850001104093D9803713931034036DB026533D9
:100860009102D4305402802E1D02632CEE01752AB1
:10087000C501B028A001102781018F2564012B2418
:100880004B01E0223401AC211F018D200D01801F9E
:10089000FC00841EED00971DDF00B81CD200E61B93
:1008A000C600201BBC00641AB200B219A8000A19C5
:1008B000A0006A189900D117910040178B00B51657
:1008C000840031167E00B31579003A157300C71401
:1008D0006F0058146A00EE13660088136300251336
:1008E0005E00C7125B006C12570015125400C11154
:1008F000510070114F0021114B00D61049008D108E
:1009000047004610440002104200C00F4000800F14
:100910003E00420F3C00060F3B00CB0E3800930E0A
:1009200037005C0E3500270E3400F30D3200C10D88
:100930003100900D3000600D2E00320D2D00050DA0
:100940002C00D90C2B00AE0C2900850C29005C0C66
:100950002700350C27000E0C2600E80B2400C40BE2
:100960002400A00B23007D0B23005A0B2100390B20
:100970002100180B2000F80A1F00D90A1E00BB0A2C
:100980001E009D0A1D00800A1D00630A1C00470A04
:100990001B002C0A1B00110A1A00F7091A00DD09B6
:1009A0001900C4091900AB091900920917007B0945
:1009B0001800630917004C091600360916002009B3
:1009C00016000A091500F5081500E0081400CC0807
:1009D0001400B8081400A4081400900813007D083F
:1009E00012006B0813005808120046081200340861
:1009F0001100230811001208110001081100F0076E
:100A00001000E0071000D0071000C0071000B0076A
:100A10000F00A107100091070E0083070F00740755
:100A20000F0065070E0057070E0049070E003B0731
:100A30000D002E070E0020070D0013070D000607FE
:100A40000D00F9060C00ED060D00E0060C00D406C2
:100A50000C00C8060C00BC060C00B0060C00A40676
:100A60000B0099060C008D060B0082060B00770622
:100A70000B006C060B0061060A0057060B004C06C3
:100A80000A0042060A0038060A002E060A0024065A
:100A90000A001A060A001006090007060A00FD05EA
:100AA0000900F4050900EB050900E2050900D90574
:100AB0000900D0050900C7050900BE050900B505F4
:100AC0000800AD050800A50509009C05080094056F
:100AD00008008C050800840508007C0508007405E2
:100AE00008006C050700650508005D050700560550
:100AF00008004E05070047050700400508003805B7
:100B00000700310507002A050700230507001C051B
:100B10000600160507000F05070008050600020578
:100B20000700FB040600F5040700EE040600E804D5
:100B30000600E2040700DB040600D5040600CF042B
:100B40000600C9040600C3040600BD040600B7047D
:100B50000600B1040500AC040600A6040600A004CB
:100B600005009B04060095040500900406008A0415
:100B7000050085040500800406007A04050075045C
:100B80000500700405006B0405006604050061049F
:100B900005005C04050057040500520405004D04DF
:100BA000050048040500430405003E0404003A041F
:100BB000050035040500300404002C04050027045A
:100BC0000400230405001E0404001A040400160493
:100BD0000500110404000D040400090405000404C8
:100BE000040000040400FC030400F8030400F40300
:100BF0000400F0030400EC030400E8030400E40331
:100C00000400E0030400DC030400D8030400D40360
:100C10000400D0030400CC030400C8030300C50390
:100C2000030024F404D9201BC40C5C0E9804C409EE
:100C30005F0265077101F405F900FB04B300480485
:100C40008700C10369005803550003034500BE0235
:100C50003A008402310053022A00290225000402CE
:100C60002000E4011C00C8011900AF011700980121
:100C70001400840113007101100061011000510182
:100C80000E0043010D0036010B002B010B0020016B
:100C90000B00150109000C01090003010800FB000D
:100CA0000800F3000800EB000700E4000600DE0087
:100CB0000600D8000600D2000600CC000500C700E0
:100CC0000500C2000500BD000400B9000400B50025
:100CD0000400B1000400AD000400A9000400A50058
:100CE0000300A20003009F0004009B000300980083
:100CF00003009500020093000300900003008D00A4
:100D000002008B00030088000200860002008400BD
:100D10000300810002007F0002007D0002007B00D2
:100D200002007900020077000100760002007400E2
:100D3000020072000100710002006F0002006D00ED
:100D400001006C0002006A000100690002006700F7
:100D500001006600010065000100640002006200FD
:100D6000010061000100600001005F0002005D0001
:100D700001005C0001005B0001005A000100590005
:100D80000100580001005700010056000100550005
:100D90000100540001005300000053000100520004
:100DA000010051000100500001004F0001004E0001
:100DB00000004E0001004D0001004C0001004B00FE
:100DC00000004B0001004A000100490001004800FA
:100DD00000004800010047000100460000004600F6
:100DE00001004500000045000100440001004300EF
:100DF00000004300010042000000420001004100E9
:100E0000000041000100400001003F0000003F00E1
:100E100001003E0000003E0001003D0000003D00DA
:100E200001003C0000003C0000003C0001003B00D1
:100E300000003B0001003A0000003A0001003900C8
:100E400000003900010038000000380000003800C0
:100E500001003700000037000100360000003600B6
:100E600000003600010035000000350000003500AC
:100E700001003400000034000000340001003300A1
:100E80000000330000003300010032000000320097
:100E9000000032000100310000003100000031008C
:100EA00001003000000030000000300001002F0081
:100EB00000002F0000002F0000002F0001002E0076
:100EC00000002E0000002E0001002D0000002D006B
:100ED00000002D0000002D0001002C0000002C005F
:100EE00000002C0000002C0001002B0000002B0053
:100EF00000002B0000002B0001002A0000002A0047
:100F000000002A0000002A0001002900000029003A
:100F1000000029000000290000002900010028002D
:100F20000000280000002800000028000000280021
:100F30000100270000002700000027000000270014
:100F40000000270001002600000026000000260007
:100F500000002600000026000100250000002500FA
:100F600000002500000025000000250000002500ED
:100F700001002400000024000000240000002400E0
:100F800000002400010023000000230000002300D3
:100F900000002300000023000000230000002300C5
:100FA00001002200000022000000220000002200B8
:100FB00000002200000022000100210000002100AA
:100FC000000021000000210000002100000021009D
:100FD000000021000100200000002000000020008F
:100FE0000000200000002000000020000000200081
:100FF0000000200001001F0000001F0000001F0073
:1010000000001F0000001F0000001F0000001F0064
:1010100001001E0000001E0000001E0000001E0057
:1010200000006563686F3A00202D20496E76616C80
:101030006964206578747275646572206E756D627E
:101040006572202100504944204175746F74756E9B
:10105000652066696E6973686564202120506C6143
:10106000636520746865204B702C204B6920616E8D
:1010700064204B6420636F6E7374616E74732069B7
:101080006E2074686520636F6E666967757261743F
:10109000696F6E2E6800504944204175746F7475F5
:1010A0006E65206661696C6564212074696D656F89
:1010B00075740020403A006F6B20543A006F6B202B
:1010C000423A00504944204175746F74756E652032
:1010D0006661696C6564212054656D706572617428
:1010E00075726520746F206869676800204B643AE8
:1010F0002000204B693A2000204B703A200020430A
:101100006C617369632050494420002054753A2073
:1011100000204B753A2000206D61783A2000206D48
:10112000696E3A200020643A200020626961733AB7
:1011300020004572726F723A0000000000300E010C
:1011400000C00E0A00500F1400D00F1E00601028BF
:1011500000E010320070113C00F011460070125097
:101160000000135A008013640000146E009014787D
:10117000001015820090158C00101696009016A095
:10118000001017AA009017B4001018BE009018C8DD
:10119000001019D2009019DC00101AE600801AF035
:1011A00000001BFA00801B0401F01B0E01701C18CC
:1011B00001F01C2201601D2C01E01D3601501E4073
:1011C00001D01E4A01401F5401B01F5E013020684B
:1011D00001A020720110217C019021860100229043
:1011E000016026F401902A5802802EBC0250322061
:1011F00003E03584035039E803803C4C04436172BA
:10120000642072656D6F7665640043617264206965
:101210006E736572746564004D3234004D32332054
:101220002573004D30350025730025730051756915
:10123000740051756974004E65787420506167655B
:10124000005072652050616765004D61696E005005
:1012500061757365642E004D6174657269616C20FF
:101260006973206F75742E002D2D3A2D2D004D3889
:10127000340046494E495348004241434B004E45D5
:10128000585400466C6F7700466C6F770046616E6D
:101290002073706565640046616E207370656564D7
:1012A000004E6F7A7A6C6532004E6F7A7A6C6532D6
:1012B000004E6F7A7A6C65004E6F7A7A6C65004DDD
:1012C0006F7665004D6F7665004D61696E005374F1
:1012D0006F7265206D656D6F7279004E6F7A7A6CF2
:1012E00065004E6F7A7A6C650046616E207370659A
:1012F00065640046616E20737065656400507265B8
:10130000706172650053746F7265206D656D6F72E8
:1013100079004E6F7A7A6C65004E6F7A7A6C650050
:1013200046616E2073706565640046616E2073705F
:10133000656564005072657061726500436F6E662A
:1013400069726D2053657474696E6773004E6F7AAD
:101350007A6C65204F6666736574004E6F7A7A6C9E
:1013600065204F6666736574004865696768742810
:101370005A2900486569676874285A2900446570CD
:1013800074682859290044657074682859290057E1
:101390006964746828582900576964746828582952
:1013A00000507265706172650041626F75742075DE
:1013B000730052657365742044656661756C7400D2
:1013C0004D616368696E652053657474696E6773F7
:1013D00000507265686561742041425320436F6E0E
:1013E00066005072656865617420504C4120436FFF
:1013F0006E660046616E2073706565640046616EBE
:10140000207370656564004C6173657220456E677A
:10141000726176696E67204D6F646500436F6F6C13
:10142000646F776E00507265686561742041425345
:10143000005072656865617420504C41004D6F76B4
:1014400065204178697300473238205900486F6D34
:1014500065205900473238205800486F6D65205884
:1014600000473238205A00486F6D65205A004D38C9
:10147000340044697361626C6520537465707065F3
:101480007273004D61696E004732380052657375A2
:101490006D65205072696E740047333232004733F5
:1014A00032320046696E69736865642E004D3834C7
:1014B000004D383420582059205A2045004D6F7671
:1014C0006520302E316D6D004D6F766520316D6D6C
:1014D000004D6F76652031306D6D00507265706122
:1014E0007265005800590045787472756465720021
:1014F00045787472756465720045787472756465B8
:101500007220310045787472756465722030004D28
:101510006F7665205A004D6F76652059004D6F76C5
:10152000652058004D6F76652041786973005A0038
:101530004D3035004D30330041626F757420757346
:1015400000536176652064697374616E636500465B
:101550006F63616C2064697374616E636500466FCC
:1015600063616C2064697374616E636500547572A5
:101570006E206F6666204C61736572005475726EE2
:10158000206F6E204C61736572004D6F7665205A36
:1015900000473238205A3000486F6D65205A004DA0
:1015A00061696E204D656E75004E6F2043617264F7
:1015B00000456E67726176652066726F6D205344D8
:1015C00020636172640053746F7020456E677261AE
:1015D00076696E6700526573756D6520456E67723A
:1015E0006176696E6700506175736520456E67723C
:1015F0006176696E6700473130310053657420624F
:1016000061736520706F696E74004F626A65637400
:1016100020686569676874004F626A656374206852
:10162000656967687400466F63616C205365747404
:10163000696E6773004D6F7665004D6F7665004E7D
:101640006F2043617264005072696E742066726F1D
:101650006D20534420636172640053746F70205096
:1016600072696E7400526573756D65205072696E93
:1016700074005061757365205072696E7400506C0F
:10168000617465204C6576656C696E670047323819
:1016900000486F6D6520616C6C00507265706172FE
:1016A00065004F6666004F6E20004F6666004F6E05
:1016B0002000456E61626C652046570054756E656A
:1016C000005374617475732073637265656E0000F6
:1016D0000B1000000D000000003039000D000D005F
:1016E000090D1A0B0000FF80FF80C180C180C180FE
:1016F000C180C180C180C180C180C180FF80FF8066
:10170000040D0D060000F0F0303030303030303055
:10171000303030090D1A0A0000FF80FF800180017F
:10172000800180FF80FF80C000C000C000C000FFBB
:1017300080FF80090D1A0B0000FF80FF80018001EF
:10174000800180FF80FF800180018001800180FF97
:1017500080FF800B0D1A0D00000180038007800DB3
:1017600080198031806180FFE0FFE001800180010D
:10177000800180090D1A0A0000FF80FF80C000C0B0
:1017800000C000FF80FF800180018001800180FF98
:1017900080FF80090D1A0A0000FF80FF80C000C092
:1017A00000C000FF80FF80C180C180C180C180FF78
:1017B00080FF80090D1A0A0000FF80FF8001800170
:1017C0008001800180018001800180018001800111
:1017D000800180090D1A0B0000FF80FF80C180C1CD
:1017E00080C180FF80FF80C180C180C180C180FF37
:1017F00080FF80090D1A0B0000FF80FF80C180C1AF
:1018000080C180FF80FF800180018001800180FF16
:1018100080FF8000060900000701850308207FFE85
:1018200007FE07FE00000005000001070702000098
:1018300080808080800080030202040005A0A00652
:101840000707060000C0D824202024180507070633
:1018500000002078A07028F0200707070800004249
:10186000A44810244A8406050507000210387C109D
:10187000F0FF030707040000204080808040200321
:101880000707040000804020202040800505050651
:101890000000A870F870A80505050600002020F8D3
:1018A00020200203030300FF4040800301010400E5
:1018B00002E0010202020000808005070706000026
:1018C00008081020408080050707060000F8888877
:1018D000888888F8020707030000C0404040404065
:1018E00040050707060000F80808F88080F805079B
:1018F00007060000F80808F80808F80607070700B8
:101900000008182848FC0808050707060000F880AA
:1019100080F80808F8050707060000F88080F888B6
:1019200088F8050707060000F808080808080805F1
:101930000707060000F88888F88888F80507070672
:101940000000F88888F80808F80105050200008002
:10195000800080800205050300FF400040408005B4
:1019600005050600001860806018040303050001E7
:10197000F000F0050505060000C0300830C005077E
:1019800007070100708808102000200807070900D9
:10199000003C4299A999423C0507070600002050E7
:1019A00088F8888888050707060000F08888F0888E
:1019B00088F0050707060000708880808088700521
:1019C0000707060000F08888888888F00407070564
:1019D0000000F08080F08080F0040707050000F030
:1019E0008080F0808080050707060000708880B83E
:1019F000888870050707060000888888F888888826
:101A00000107070200008080808080808005070732
:101A10000600000808080808887005070706000087
:101A20008890A0C0A09088040707050000808080EF
:101A3000808080F007070708000082C6AA92828291
:101A4000820507070600008888C8A89888880507C7
:101A500007060000708888888888700507070600D8
:101A600000F08888F08080800508080600FF7088F4
:101A7000888888887008050707060000F08888F0C5
:101A800088888805070706000070888070088870BD
:101A9000050707060000F820202020202005070762
:101AA0000600008888888888887005070706000077
:101AB000888888888850200707070800008292924B
:101AC0009292926C05070706000088885020508883
:101AD0008805070706000088885020202020050779
:101AE00007060000F80810204080F80207070300EE
:101AF00000C08080808080C00507070701008080CB
:101B00004020100808020707030000C04040404082
:101B100040C0FF050101060000F8FF0505050600AD
:101B20000070087888780507070600008080F08834
:101B30008888F00505050600007088808870050714
:101B400007060000080878888888780505050600DB
:101B5000007088F88078030707030000608080C069
:101B60008080800507070600FE788888887808301E
:101B70000507070600008080F0888888880107072D
:101B8000020000800080808080800209090300FE3E
:101B90004000404040404040800507070600008864
:101BA00090A0C0A09088010707020000808080807C
:101BB000808080070505080000EC9292929205054E
:101BC00005060000F0888888880505050600007075
:101BD000888888700507070600FEF0888888F080EE
:101BE000800507070600FE788888887808080405BD
:101BF00005050000B0C0808080050505060000785E
:101C0000807008F00307070400004040E0404040B7
:101C100040050505060000888888887805050506C2
:101C200000008888885020070505080000929292DD
:101C3000926C0505050600008850205088050707AE
:101C40000600FE88888888780830050505060000AB
:101C5000F8102040F80307070400002040408040AF
:101C60004020010707020000808080808080800380
:101C7000070704000080404020404080FFFF000034
:101C80000000000000000000000000000000000054
:101C90000000000000000000000000000000000044
:101CA0000000000000000000000000000000000034
:101CB0000000000000000000000000000000000024
:101CC0000000000000000000000000000000000014
:101CD0000000000000000000000000000000000004
:101CE00000000000000000000000000000000000F4
:101CF00000000000000000000000000000000000E4
:101D000000000000000000000000000000000000D3
:101D100000000000000000000000000000000000C3
:101D200000000000000000000000000000000000B3
:101D3000F000000000E000000000000000000001D2
:101D400098000000072000000000000000000003D1
:101D50000C0000001C200000000000000000000239
:101D600005C0000070200000000001F70000000224
:101D700005300001C0200000900000148000000326
:101D80000D0C000700200D92B98C001440000001DA
:101D90009903001C00201252925201F440000000EE
:101DA000F100C07000201252925200144000000056
:101DB000010031C000201252925200148000000035
:101DC00001000E000020124E998C01F70000000364
:101DD000FD000400102000000000000000000002D0
:101DE0000580040030200000000000000000000218
:101DF00004600400D0200000000000000000000289
:101E0000041804031020000000000000000000027D
:101E10000406040C10200000000000000000000276
:101E200004018430102000000000000000000002C7
:101E3000040064C010200000000000000000000248
:101E400004001F00102010023FF883E00000000291
:101E500004000400102018060100820000000002A7
:101E6000040000001020140A01008200000000029B
:101E70000400000010201212010082000000000285
:101E80000400000010201122010083E00000000285
:101E900004000000102010C2010080200000000299
:101EA0000400000010201002010080200000000249
:101EB0000400000010201002010090200000000229
:101EC0000400000010201002010093E00000000256
:101ED00004000000102000000000000000000002CC
:101EE00004000000102000000000000000000002BC
:101EF00004000000102000000000000000000002AC
:101F0000040000001020000000000000000000029B
:101F1000040000001020000000000000000000028B
:101F2000040000001020000000000000000000027B
:101F3000040000001020000000000000000000016C
:101F40000800000010200000000000000000000059
:101F5000900000001FE000000000000000000000F2
:101F60006000000000000000000000000000000011
:101F70000000000000000000000000000000000061
:101F80000000000000000000000000000000000051
:101F90000000000000000000000000000000000041
:101FA0000000000000000000000000000000000031
:101FB0000000000000000000000000000000000021
:101FC0000000000000000000000000000000000011
:101FD0000000000000000000000000000000000001
:101FE00000000000000000000000000000000000F1
:101FF00000000000000000000000000000000000E1
:1020000000000000000000000000000000000000D0
:1020100000000000000000000000000000000000C0
:1020200000000000000000000000000000000000B0
:1020300000000000000000000000000000000000A0
:102040000000000000000000000000000000000090
:102050000000000000000000000000000000000080
:102060000000000000000000000000000000000070
:102070000000000000000000000000000000000060
:102080000000020100000400800008004000100071
:1020900020002000100040000800FFFFFC008048E6
:1020A0000400804804008048040080480400804800
:1020B000040080480400FFCFFC0000000000000086
:1020C00000000000000000000000000000000030E0
:1020D0000C000060060000C00300018001800300C6
:1020E00000C0060000600C0000301800001830002E
:1020F000000C600000067FFFFFFE7FFFFFFE600F09
:10210000F006600C3006600C3006600C3006600C87
:102110003006600C3006600C30067FFC3FFE3FF856
:102120001FFC000000000000000000000000000094
:102130000000000000000000000000000000FFE0C0
:10214000FFD11000FFFEFFD0FFE0FFC1FFD140A094
:10215000C8A6A22FF800238127AC00AFFF64A5FF1B
:1021600064FF64A4FFD0FFFE00000A0B02090C0DFF
:102170000E0807030401000000000000000000003A
:10218000000000000000000000000000000000004F
:10219000000000001211100000000000000000000C
:1021A000000000000000000000000000000001022C
:1021B0001020200808102040102040800201020159
:1021C0000804020101020408102040808040201011
:1021D000080402018004020180402010080402016A
:1021E00008040201010204081020408001020408D2
:1021F00010204080050505050705080808080202AB
:1022000002020A0A08080404040401010101010190
:1022100001010303030303030303040707070C0C73
:102220000C0C0C0C0C0C020202020606060606063A
:1022300006060B0B0B0B0B0B0B0B000022002500F3
:1022400028002B002E00310034000201000005019F
:1022500008010B0100002100240027002A002D00A6
:102260003000330001010000040107010A01024EA1
:10227000414E494E495459494E46CDCCCC3D0AD7E2
:10228000233C17B7D13877CC2B329595E6241FB174
:102290004F0A000020410000C84200401C4620BCFC
:1022A000BE4CCA1B0E5AAEC59D7406382DA80A38FE
:1022B00011241FBECFEFD1E2DEBFCDBF00E00CBFC7
:1022C00015E0A0E0B2E0E4E2F5E801E00BBF02C0F7
:1022D00007900D92A237B107D9F723E1A2E7B5E045
:1022E00001C01D92A13CB207E1F712E2CEEAD2E2B0
:1022F00000E006C022970109FE010BBF0E94DABB75
:10230000CA3AD10780E00807A9F70E94CDB60C941D
:1023100081C20C940000EF92FF920F931F93CF9312
:10232000DF931F92CDB7DEB78C017B01460FF7011B
:1023300061917F01F8018081918149830E94CAC126
:10234000F8018081918101969183808349814E11AA
:10235000EECF0F90DF91CF911F910F91FF90EF90F3
:102360000895EF92FF920F931F93CF93DF931F92E5
:10237000CDB7DEB78C017B01460FF80180819181DA
:1023800049830E94C2C1F70181937F01F8018081D6
:10239000918101969183808349814E11EECF0F90F8
:1023A000DF91CF911F910F91FF90EF9008950F93C0
:1023B0001F93CF93DF93CDB7DEB72A970FB6F8946C
:1023C000DEBF0FBECDBF80E390E3A0E3B0E08D831E
:1023D0009E83AF83B88704E610E01A87098744E03C
:1023E000BE016B5F7F4FCE01099695DF40E16DE640
:1023F00071E1CE0109968FDF40E16DE771E1CE0119
:10240000099689DF40E16DE571E1CE01099683DF30
:1024100044E065E571E1CE0109967DDF44E061E5C8
:1024200071E1CE01099677DF44E069E571E1CE0103
:10243000099671DF44E06DE371E1CE0109966BDF2F
:1024400044E06DE871E1CE01099665DF44E06DE49A
:1024500071E1CE0109965FDF44E069E471E1CE01EC
:10246000099659DF44E065E471E1CE01099653DF36
:1024700044E061E471E1CE0109964DDF4CE06CED82
:1024800078E0CE01099647DF42E06EE179E0CE01C7
:10249000099641DF41E069E079E0CE0109963BDF32
:1024A00042E06AE079E0CE01099635DF42E06CE077
:1024B00079E0CE0109962FDF42E06EE079E0CE01AF
:1024C000099629DF42E064E179E0CE01099623DF35
:1024D00042E065E073E1CE0109961DDF42E063E072
:1024E00073E1CE01099617DF42E061E073E1CE01AE
:1024F000099611DF42E06FEF72E1CE0109960BDF22
:1025000042E06DEF72E1CE01099605DF42E06BEF2C
:1025100072E1CE010996FFDE44E069E672E0CE0189
:102520000996F9DE44E065E672E0CE010996F3DE35
:1025300044E061E672E0CE010996EDDE86E590E3C7
:10254000A7E3B0E089839A83AB83BC831A870987AA
:1025500044E0BE016F5F7F4FCE010996DCDEE2EE04
:10256000F1E08491882341F09091C00095FFFCCF69
:102570008093C6003196F5CFE2EDF1E08491882397
:1025800041F09091C00095FFFCCF8093C60031963A
:10259000F5CF8091C00085FFFCCF8AE08093C60014
:1025A0002A960FB6F894DEBF0FBECDBFDF91CF9154
:1025B0001F910F910895AF92BF92CF92DF92EF9249
:1025C000FF920F931F93CF93DF93CDB7DEB7E097C2
:1025D0000FB6F894DEBF0FBECDBF80E1E9E9F2E0AF
:1025E000DE01919601900D928A95E1F780E1E9EA8A
:1025F000F2E0DE01519601900D928A95E1F780E1BB
:10260000E9EBF2E0DE01119601900D928A95E1F777
:102610006E0181E2C80ED11C8DE6E82E81E1F82E14
:102620008E010F5E1F4F6DE771E1AE014F5F5F4F8F
:102630009DE5A92E91E1B92E20E030E0F6018191CF
:102640009191A191B1916F01F70181939193A19320
:10265000B1937F01F80181919191A191B1918F0185
:10266000FB0181939193A193B193BF01FA018191F1
:102670009191A191B191AF01F50181939193A193B2
:10268000B1935F012F5F3F4F24303105B9F60E94AF
:10269000AE6380E090E0AAEFB4E48093551190938C
:1026A0005611A0935711B093581180E090E8ABE316
:1026B000B5E48093511190935211A0935311B093AC
:1026C00054111092591110925A1110925B111092DC
:1026D0005C1180E29EE4A0E0B0E080938D119093C5
:1026E0008E11A0938F11B093901180E090E0A0EA3A
:1026F000B1E480933D1190933E11A0933F11B093AC
:10270000401180E090E0A0E2B1E480934D119093FD
:102710004E11A0934F11B093501180E090E0A0E0D3
:10272000B1E48093491190934A11A0934B11B09357
:102730004C118DEC9CECACECBEE380934511909376
:102740004611A0934711B093481180E090E0A0EAB1
:10275000B0E48093411190934211A0934311B09340
:1027600044111092E4081092E5081092E6081092C5
:10277000E7081092E0081092E1081092E208109227
:10278000E3081092DC081092DD081092DE08109227
:10279000DF088EE590E090931F0980931E09109248
:1027A000040981E08093090980E991E090930B0985
:1027B00080930A0990930D0980930C0990930F0957
:1027C00080930E09109215091092140988EC90E07C
:1027D00090930613809305138CE390E09093041379
:1027E000809303138EE790E090930213809301137C
:1027F00020EF30E0309300132093FF122AE530E001
:102800003093FE122093FD129093FC128093FB12E2
:102810008AE999E9A1EBB1E48093690290936A0295
:10282000A0936B02B0936C0261E77DE38AE89FE3BB
:102830000E94BE7660936502709366028093670281
:102840009093680260E070E084EE92E40E94CA76A1
:1028500060936102709362028093630290936402BA
:102860000E94DA6D80E090E0A0E8BFE380935D0213
:1028700090935E02A0935F02B093600298DDE2EE57
:10288000F1E08491882341F09091C00095FFFCCF46
:102890008093C6003196F5CFE6E9F1E08491882374
:1028A00041F09091C00095FFFCCF8093C600319617
:1028B000F5CF8091C00085FFFCCF8AE08093C600F1
:1028C000E0960FB6F894DEBF0FBECDBFDF91CF917B
:1028D0001F910F91FF90EF90DF90CF90BF90AF903E
:1028E0000895CF93DF93CDB7DEB72A970FB6F8944C
:1028F000DEBF0FBECDBF84E690E09A87898786E56C
:1029000090E3A7E3B0E089839A83AB83BC8344E080
:10291000BE016B5F7F4FCE01099623DD43E050E09F
:10292000BE016B5F7F4FCE0101960E9411BF892BC4
:1029300009F0CEC040E16DE671E1CE01099611DDEE
:1029400040E16DE771E1CE0109960BDD40E16DE5F7
:1029500071E1CE01099605DD0E94AE6344E065E5B4
:1029600071E1CE010996FDDC44E061E571E1CE0143
:102970000996F7DC44E069E571E1CE010996F1DCE6
:1029800044E06DE371E1CE010996EBDC44E06DE8D3
:1029900071E1CE010996E5DC44E06DE471E1CE0120
:1029A0000996DFDC44E069E471E1CE010996D9DCE7
:1029B00044E065E471E1CE010996D3DC44E061E4D2
:1029C00071E1CE010996CDDC4CE06CED78E0CE01F2
:1029D0000996C7DC42E06EE179E0CE010996C1DCE0
:1029E00041E069E079E0CE010996BBDC42E06AE0B3
:1029F00079E0CE010996B5DC42E06CE079E0CE01E9
:102A00000996AFDC42E06EE079E0CE010996A9DCE0
:102A100042E064E179E0CE010996A3DC42E065E0A2
:102A200073E1CE0109969DDC42E063E073E1CE01E3
:102A3000099697DC42E061E073E1CE01099691DCF2
:102A400042E06FEF72E1CE0109968BDC42E06DEF60
:102A500072E1CE01099685DC42E06BEF72E1CE01B6
:102A600009967FDC44E069E672E0CE01099679DCE4
:102A700044E065E672E0CE01099673DC44E061E66D
:102A800072E0CE0109966DDC0E94DA6DE2EEF1E0B3
:102A90008491882341F09091C00095FFFCCF8093F2
:102AA000C6003196F5CFE8EBF1E08491882341F040
:102AB0009091C00095FFFCCF8093C6003196F5CF72
:102AC0008091C00085FFFCCF8AE08093C60001C0E2
:102AD00072DD2A960FB6F894DEBF0FBECDBFDF9130
:102AE000CF9108951F920F920FB60F9211240BB63B
:102AF0000F922F933F934F935F936F938F939F9377
:102B0000EF93FF936091C6002091F3053091F40597
:102B1000C90101968F7799274091F5055091F605E7
:102B20008417950741F0F901ED58FA4F60839093AF
:102B3000F4058093F305FF91EF919F918F916F9131
:102B40005F914F913F912F910F900BBE0F900FBE51
:102B50000F901F9018959A01AB01211581EE38074F
:102B60004105510549F182E08093C00060E079E0C1
:102B70008DE390E00E94A8BB215031094109510921
:102B8000CA01B90122E030E040E050E00E94A8BB59
:102B90003093C5002093C4008091C1008061809370
:102BA000C1008091C10088608093C1008091C10004
:102BB00080688093C10008951092C00020E130E049
:102BC000E7CF2091F5053091F6058091F3059091BE
:102BD000F4058217930771F0F901ED58FA4F8081DF
:102BE0002F5F3F4F2F7733273093F6052093F5055E
:102BF00090E008958FEF9FEF08958091F5059091F3
:102C0000F6059093F4058093F30508954F925F9233
:102C10006F927F928F929F92AF92BF92CF92DF92EC
:102C2000EF92FF920F931F93CF93DF93CDB7DEB751
:102C3000A0970FB6F894DEBF0FBECDBF5C01411563
:102C4000510561057105E9F420E030E040E350E012
:102C500060E070E0A0960FB6F894DEBF0FBECDBF67
:102C6000DF91CF911F910F91FF90EF90DF90CF9068
:102C7000BF90AF909F908F907F906F905F904F909C
:102C80005BC08E010F5F1F4FC12CD12C7601480114
:102C9000422E512C612C712C8FEFC81AD80AE80AE9
:102CA000F80ACB01BA01A30192010E9486BBCA01B6
:102CB000F80161938F01A901BC014115510561051E
:102CC000710551F7F1E0CF1AD108E108F108F401DC
:102CD000EC0DFD1D80818A3010F440E301C047E314
:102CE000480F552747FD5095652F752F20E030E0A0
:102CF000C50122D081E0C81AD108E108F108EFEF40
:102D0000CE16DE06EE06FE0611F7A0960FB6F89474
:102D1000DEBF0FBECDBFDF91CF911F910F91FF900E
:102D2000EF90DF90CF90BF90AF909F908F907F906B
:102D30006F905F904F9008952115310539F480917F
:102D4000C00085FFFCCF4093C60008952A303105AE
:102D500009F41CC05BCFCF93DF93EC0120E030E09F
:102D60004DE050E060E070E0E7DF20E030E04AE076
:102D700050E060E070E0CE01DF91CF91DDCF9A01AD
:102D8000AB01662757FD6095762FD6CFCF92DF92A5
:102D9000EF92FF92CF93DF93EC016A017B0177FF03
:102DA0000FC020E030E04DE250E060E070E0C4DFB2
:102DB000F094E094D094C094C11CD11CE11CF11C8F
:102DC0002AE0B701A601CE01DF91CF91FF90EF90ED
:102DD000DF90CF901BCF2115310539F48091C000D1
:102DE00085FFFCCF4093C600089510CF9A01462F6F
:102DF00050E060E070E0EFCFCF93DF93EC019A01F9
:102E0000AB0160E070E0E7DFCE01DF91CF91A3CFAF
:102E10008F929F92AF92BF92CF92DF92EF92FF92EA
:102E20001F93CF93DF93EC016A017B01122F20E007
:102E300030E0A901C701B6010E94B5B787FF0CC0F9
:102E400020E030E04DE250E060E070E0CE0174DF61
:102E5000F7FAF094F7F8F094B12C60E070E080E0BD
:102E60009FE3B11641F020E030E040E251E40E94DF
:102E7000BCB7B394F6CF9B01AC01C701B6010E9469
:102E8000DCB66B017C010E9429B84B015C010E94F9
:102E900055B89B01AC01C701B6010E94DBB66B01BE
:102EA0007C012AE0B501A401CE01B0DE112361F05E
:102EB000E9E4F4E08191882339F09091C00095FF16
:102EC000FCCF8093C600F6CF112319F120E030E04B
:102ED00040E251E4C701B6010E948ABA6B017C014D
:102EE0000E9424B84B01AA2497FCA094BA2CB501E7
:102EF000A401CE014BDFC501B4010E9457B89B016C
:102F0000AC01C701B6010E94DBB66B017C01115018
:102F1000DBCFDF91CF911F91FF90EF90DF90CF90AB
:102F2000BF90AF909F908F90089572CF4F925F9215
:102F30006F927F92AF92BF92CF92DF92EF92FF9209
:102F40000F931F93CF93DF935C01FC01EE0FFF1FE4
:102F5000EE0FFF1FE851F74F108211821282138289
:102F600024EF38E040EF58E06CEE78E088EE98E02F
:102F70000E94E362E501C75FD94FFE01549035011D
:102F8000660C771C660C771C83010756174FF301FC
:102F9000EC53F74F20E030E040EC5FE3608171815B
:102FA000828193810E948ABA6B017C01652D77270B
:102FB00067FD7095872F972F0E9457B89B01AC0132
:102FC000C701B6010E948ABAF801608371838283C7
:102FD0009383F301E15DFD4F608171818281938173
:102FE00060930A0270930B0280930C0290930D027F
:102FF00020E030E040E752E40E94BCB72BEAC22E4A
:1030000028E0D22E7B018C0125EA38E041EA58E025
:103010006DE978E089E998E00E94CD580E94C86B7C
:10302000F301E851F74F108211821282138224EFCC
:1030300038E040EF58E06CEE78E088EE98E00E94CF
:10304000E362C301845F994F3C01FC01C590D590B8
:10305000E590F490FE0164918501000F111F000FAF
:10306000111F0756174FF7FAF094F7F8F0947727E7
:1030700067FD7095872F972F0E9457B89B01AC0171
:10308000C701B6010E948ABAF80160837183828306
:10309000938320E030E040E752E460910A027091AF
:1030A0000B0280910C0290910D020E94BCB74BEA7A
:1030B000C42E48E0D42E7B018C0125EA38E041EA99
:1030C00058E06DE978E089E998E00E94CD580E94C7
:1030D000C86BF3016591759185919491FE0174908F
:1030E000E501CC0FDD1FCC0FDD1F8E010756174FFA
:1030F0009B01AC010E94DCB66B017C01672D772738
:1031000067FD7095872F972F0E9457B89B01AC01E0
:10311000C701B6010E948ABAF80160837183828375
:103120009383FE01E15DFD4F20E030E040E05FE38E
:1031300060817181828193810E948ABA60930A02C0
:1031400070930B0280930C0290930D0220E030E00C
:1031500040E752E40E94BCB7EBEACE2EE8E0DE2E58
:103160007B018C0125EA38E041EA58E06DE978E01E
:1031700089E998E00E94CD580E94C86BFE01E45294
:10318000F74FC080D180E280F380FE01E854F74F12
:103190002081318142815381C701B6010E94DCB692
:1031A0002B013C01FE01E851F74F6083718382835C
:1031B0009383C85ED94FFE01659175918591949175
:1031C000E501CC0FDD1FCC0FDD1F8E010053174F23
:1031D000A70196010E94DCB6F801608371838283A7
:1031E00093838E01015E1D4FFE01E455F74FA70149
:1031F000960160817181828193810E94DCB6F80121
:103200006083718382839383C756D74F48825982E4
:103210006A827B8210920A0210920B0210920C02B8
:1032200010920D02DF91CF911F910F91FF90EF90BF
:10323000DF90CF90BF90AF907F906F905F904F9056
:103240000C949164FC012491222341F03091C00040
:1032500035FFFCCF2093C6000196F4CF22E030E08A
:1032600082E795E062CECF93DF931F921F92CDB796
:10327000DEB78091BB139091BC139E012F5F3F4F2F
:10328000009719F4215C334102C0281B390B3A83A3
:10329000298389819A810F900F90DF91CF910895B2
:1032A0002091E2063091E306243031050CF06AC02B
:1032B0004091E4065091E50660E6649F9001659FA9
:1032C000300D1124BC01C9018451994F0E940ABFDD
:1032D000E4E2F6E08491882341F09091C00095FFEC
:1032E000FCCF8093C6003196F5CFEEEFF5E08491E8
:1032F000882341F09091C00095FFFCCF8093C600D9
:103300003196F5CF8091E4069091E50620E6289F5E
:10331000F001299FF00D1124E451F94F8191882388
:1033200039F09091C00095FFFCCF8093C600F6CF96
:10333000ECEFF5E08491882341F09091C00095FF77
:10334000FCCF8093C6003196F5CF8091C00085FFF9
:10335000FCCF8AE08093C6008091E4069091E50658
:10336000019664E070E00E9473BB9093E506809341
:10337000E4068091E2069091E30601969093E306BD
:103380008093E20608952091E2063091E30624300E
:1033900031050CF06AC04091E4065091E50660E604
:1033A000649F9001659F300D1124BC01C9018451B7
:1033B000994F0E9496BEE4E2F6E08491882341F0A2
:1033C0009091C00095FFFCCF8093C6003196F5CF59
:1033D000E1EFF5E08491882341F09091C00095FFE2
:1033E000FCCF8093C6003196F5CF8091E406909192
:1033F000E50620E6289FF001299FF00D1124E451F5
:10340000F94F8191882339F09091C00095FFFCCF4E
:103410008093C600F6CFEFEEF5E08491882341F06B
:103420009091C00095FFFCCF8093C6003196F5CFF8
:103430008091C00085FFFCCF8AE08093C600809118
:10344000E4069091E506019664E070E00E9473BB8B
:103450009093E5068093E4068091E2069091E3065E
:1034600001969093E3068093E20608958F929F92CF
:10347000AF92BF92CF92DF92EF92FF9260910A09D2
:1034800070910B09882777FD8095982F0E9457B877
:103490004B015C0160931F02709320028093210214
:1034A0009093220260910C0970910D09882777FD95
:1034B0008095982F0E9457B86B017C01609323027E
:1034C00070932402809325029093260260910E0946
:1034D00070910F09882777FD8095982F0E9457B823
:1034E00060932702709328028093290290932A0206
:1034F0008092C4089092C508A092C608B092C708EE
:10350000C092C808D092C908E092CA08F092CB08CD
:103510006093CC087093CD088093CE089093CF0829
:103520001092B8081092B9081092BA081092BB080D
:103530001092BC081092BD081092BE081092BF08ED
:103540001092C0081092C1081092C2081092C308CD
:103550008092AC089092AD08A092AE08B092AF08ED
:10356000C092B008D092B108E092B208F092B308CD
:103570006093B4087093B5088093B6089093B70829
:10358000FF90EF90DF90CF90BF90AF909F908F9083
:10359000089560E080E40E9485B29FB7F894E8E067
:1035A000F1E08081846080839FBF0895269A2E98E1
:1035B0000895EFDFFBDF40E950ED63E070E082E764
:1035C00095E0C9DAE9EEF5E08491882341F0909125
:1035D000C00095FFFCCF8093C6003196F5CF809157
:1035E000C00085FFFCCF8AE08093C60084B780FFCF
:1035F00014C0E1EEF5E09491992341F02091C000D0
:1036000025FFFCCF9093C6003196F5CF9091C00076
:1036100095FFFCCF9AE09093C60081FF14C0E1EDC6
:10362000F5E09491992341F02091C00025FFFCCF53
:103630009093C6003196F5CF9091C00095FFFCCFD6
:103640009AE09093C60082FF14C0E0ECF5E09491FC
:10365000992341F02091C00025FFFCCF9093C60034
:103660003196F5CF9091C00095FFFCCF9AE09093F2
:10367000C60083FF14C0E0EBF5E09491992341F07C
:103680002091C00025FFFCCF9093C6003196F5CF66
:103690009091C00095FFFCCF9AE09093C60085FF03
:1036A00014C0E0EAF5E08491882341F09091C000D5
:1036B00095FFFCCF8093C6003196F5CF8091C00076
:1036C00085FFFCCF8AE08093C60014BEEAE9F5E0EE
:1036D0008491882341F09091C00095FFFCCF8093A6
:1036E000C6003196F5CF8091C00085FFFCCF8AE0FF
:1036F0008093C600EAE8F5E08491882341F0909138
:10370000C00095FFFCCF8093C6003196F5CFE5E76A
:10371000F5E08491882341F09091C00095FFFCCFA3
:103720008093C6003196F5CFE9E6F5E084918823D1
:1037300041F09091C00095FFFCCF8093C600319678
:10374000F5CFE2E6F5E08491882341F09091C00046
:1037500095FFFCCF8093C6003196F5CF8091C000D5
:1037600085FFFCCF8AE08093C600E7E5F5E0849111
:10377000882341F09091C00095FFFCCF8093C60054
:103780003196F5CFEBE4F5E08491882341F09091F8
:10379000C00095FFFCCF8093C6003196F5CF809195
:1037A000C00085FFFCCF8AE08093C600ECE3F5E023
:1037B0008491882341F09091C00095FFFCCF8093C5
:1037C000C6003196F5CF4FDD4AE050E0BC0182E7FC
:1037D00095E0D5DAE5E2F5E08491882341F0909117
:1037E000C00095FFFCCF8093C6003196F5CF4AE02C
:1037F00050E060ED74E082E795E0C1DA8091C000AE
:1038000085FFFCCF8AE08093C6001092E8061092F4
:10381000E9061092EA061092EB0610920409109243
:10382000FE08109205091092010981E180930209B6
:103830001092060981E0809307098093090980E9C5
:1038400091E090930B0980930A0990930D0980935E
:103850000C0990930F0980930E091092030910929E
:103860001509109214093DD801DE0E940E700E94C5
:1038700067570E943B6B0E942A8810921C098BE0BC
:103880008093200910921B0910921A0908958091C3
:10389000DC069091DD0660E070E001960C94EDBBD3
:1038A0008091DC069091DD064AE050E060E070E037
:1038B00001960C9455BD682F772767FD7095209170
:1038C000E6063091E70640E6429FC001439F900D17
:1038D00011248451994F0E94FFBE9093DD0680937E
:1038E000DC0621E0892B09F420E0822F08950E9454
:1038F000A5B06093D8067093D9068093DA069093AA
:10390000DB06E091E606F091E706E851F94F808189
:10391000811114C0E0E1F2E08491882341F090919C
:10392000C00095FFFCCF8093C6003196F5CF809103
:10393000C00085FFFCCF8AE08093C600089582E72F
:1039400095E05BD9E3E1F2E08491882341F0909126
:10395000C00095FFFCCF8093C6003196F5CF409113
:1039600071085091720860917308709174084F5FEC
:103970005F4F6F4F7F4F2AE030E082E795E0DCD960
:103980008091C00085FFFCCF8AE08093C600AFCF56
:103990004F925F926F927F929F92AF92BF92CF921F
:1039A000DF92EF92FF920F931F93CF93DF9330E656
:1039B000B32EC4E0D0E008EE13E04AE0A42E5EE5AA
:1039C000E52E54E0F52E992493948091F30590917F
:1039D000F4052091F5053091F605821B930B8F7746
:1039E0009927892B09F424C28091E2069091E3067D
:1039F00004970CF01DC282E795E0E3D88093E106BE
:103A0000109204092091DF063091E0068A3061F0BF
:103A10008D3051F08A3321F49091DE06992321F004
:103A20002F3531050CF427C12115310509F441C1A9
:103A30008091E4069091E506B89E6001B99ED00C95
:103A40001124F601E20FF31FE451F94F1082209187
:103A5000DE0621110BC1FC01E851F94F1082C601AD
:103A60008451994F3C016EE470E00E94FFBE0097C4
:103A7000F1F19093DD068093DC06861997098C0D91
:103A80009D1D4AE050E060E070E08351994F0E9434
:103A900055BD60937508709376088093770890936E
:103AA0007808409071085090720860907308709088
:103AB0007408EFEF4E1A5E0A6E0A7E0AC090E406A2
:103AC000D090E506641575058605970509F4F4C0E0
:103AD000BC9CC001BD9C900D112467E075E0845131
:103AE000994F0E94C4BE892B09F0E6C074C16AE2F6
:103AF00070E0C3010E94FFBE892B09F443C0EAE2D3
:103B0000F6E08491882341F09091C00095FFFCCFAE
:103B10008093C6003196F5CFE1E6F4E084918823E6
:103B200041F09091C00095FFFCCF8093C600319684
:103B3000F5CF4091710850917208609173087091AF
:103B400074082AE030E082E795E0F6D88091C00062
:103B500085FFFCCF8AE08093C6001092E0061092A9
:103B6000DF067CC28091750890917608A091770855
:103B7000B09178088093710890937208A0937308AD
:103B8000B09374088091E4069091E506B89E6001B8
:103B9000B99ED00C1124C6018451994F3C0167E4B1
:103BA00070E00E94FFBE009709F44BC09093DD06C1
:103BB0008093DC06861997098C0D9D1D60E070E0EE
:103BC0008351994F0E94EDBB0E9424B86430710567
:103BD00008F037C08091F70581111AC08091230940
:103BE00081112FC0F7018491EEE5F4E0882349F0BC
:103BF0009091C00095FFFCCF8093C60031968491D0
:103C0000F5CF8091C00085FFFCCFA092C60019C0FF
:103C1000F8018491E8EEF3E0882349F09091C00028
:103C200095FFFCCF8093C60031968491F5CF8091AB
:103C3000C00085FFFCCFA092C6008EED93E00E94ED
:103C40000D878091E4069091E5060196BE010E94E1
:103C500073BB9093E5068093E4068091E206909111
:103C6000E30601969093E3068093E2061092E00645
:103C70001092DF06AACE8B3311F49092DE0690915B
:103C8000DE069111A2CE4091E4065091E506B901FD
:103C90006F5F7F4F7093E0066093DF06B49EF00184
:103CA000B59EF00D1124E20FF31FE451F94F80830C
:103CB0008CCE1092DE06D2C1BC9C3001BD9C700C33
:103CC0001124C3018451994F2C016AE270E00E94D3
:103CD000FFBE009781F5EAE2F6E08491882341F087
:103CE0009091C00095FFFCCF8093C6003196F5CF30
:103CF000EBE8F4E08491882341F09091C00095FFB7
:103D0000FCCF8093C6003196F5CF40917108509159
:103D1000720860917308709174082AE030E082E7BD
:103D200095E00AD88091C00085FFFCCF8AE080939F
:103D3000C60005DE12CF20E0D12CF301E20FF11D09
:103D4000E451F94F30813A3219F02F5FD326F5CF85
:103D50009093DD068093DC0684199509860D971DE6
:103D600060E070E08351994F0E94EDBB0E9424B83F
:103D70002D2D30E02617370709F4F4CEEAE2F6E0FD
:103D80008491882341F09091C00095FFFCCF8093EF
:103D9000C6003196F5CFE5EBF4E08491882341F03D
:103DA0009091C00095FFFCCF8093C6003196F5CF6F
:103DB0004091710850917208609173087091740875
:103DC0002AE030E082E795E00E949C168091C000D6
:103DD00085FFFCCFABCFEAE2F6E08491882341F087
:103DE0009091C00095FFFCCF8093C6003196F5CF2F
:103DF000E4EDF4E08491882341F09091C00095FFB8
:103E0000FCCF8093C6003196F5CF40917108509158
:103E1000720860917308709174082AE030E082E7BC
:103E200095E00E949C168091C00085FFFCCF7ECF5C
:103E300080912509882389F08091DF069091E00622
:103E4000892B59F490E6E92EFF24F394C4E0D0E0E6
:103E500006EC13E02AE0D22EAFC08091040988233B
:103E600009F4FCC08091050987FDF8C08068809343
:103E7000050989ED93E0DF91CF911F910F91FF909C
:103E8000EF90DF90CF90BF90AF909F907F906F901A
:103E90005F904F9078CA8091E2069091E306049774
:103EA0000CF0DCC08091FF099091000AA091010AFA
:103EB000B091020A80931A0A90931B0AA0931C0ADD
:103EC000B0931D0A87EF99E00E94D93C482F809358
:103ED000E1068A3019F04D3009F085C040911A0A88
:103EE00050911B0A60911C0A70911D0A8091120A60
:103EF0009091130AA091140AB091150A4817590716
:103F00006A077B0738F1F8018491E6ECF3E0811150
:103F10007EC08091C00085FFFCCFD092C6008CEBA4
:103F200093E00E940D87F092FE08109201090E9412
:103F3000A5B06093CC067093CD068093CE06909387
:103F4000CF0683E299E00E94675061E083E299E046
:103F50000E94A84E2091DF063091E0062115310520
:103F600009F4A7CE8091E4069091E506E89EF00161
:103F7000E99EF00D1124E20FF31FE451F94F108276
:103F8000FC01E851F94FF0822091E2063091E306FE
:103F90002F5F3F4F3093E3062093E2060196BE0168
:103FA0000E9473BB9093E5068093E4061092DE06B0
:103FB0001092E0061092DF0640911A0A50911B0AF7
:103FC00060911C0A70911D0A8091120A9091130A47
:103FD000A091140AB091150A481759076A077B0780
:103FE00008F03CC058CF4A3329F42091DE06222342
:103FF00009F474CF2091DF063091E0062F353105AA
:104000000CF06CCF8F3FFFEF9F0751F467CF90917B
:10401000C00095FFFCCF8093C6003196849177CF86
:104020004B3311F4F092DE064091DE064111C4CF0D
:104030004091E4065091E506B9016F5F7F4F7093A0
:10404000E0066093DF06E49EF001E59EF00D11248A
:10405000E20FF31FE451F94F8083AECFDF91CF9190
:104060001F910F91FF90EF90DF90CF90BF90AF9096
:104070009F907F906F905F904F9008958F929F9246
:10408000AF92BF92CF92DF92EF92FF920F931F9366
:10409000CF93DF9369ECE62E63E0F62E08EE18E08E
:1040A000C9E9D8E07AEFC72E78E0D72EF7018191E1
:1040B0007F0101DC882311F1EADB4B015C01F60191
:1040C0008081811103C060916C0801C061E070E0E3
:1040D00080E090E00E9457B8F80120813181428150
:1040E00053810E948ABA9B01AC01C501B4010E94B0
:1040F000DCB6688379838A839B8309C0F801808159
:104100009181A281B38188839983AA83BB830C5F49
:104110001F4F2496FFEFCF1ADF0A8DECE81683E0DD
:10412000F80621F686E4C7DB8823D1F0B0DB6B010B
:104130007C0160937D0870937E0880937F08909344
:10414000800820E030E0A9010E94B8B9181644F4B4
:10415000C0920A02D0920B02E0920C02F0920D0281
:10416000DF91CF911F910F91FF90EF90DF90CF9053
:10417000BF90AF909F908F90089580DF89E49BDB84
:10418000882351F084DB60938D0870938E088093B0
:104190008F089093900808C010928D0810928E0896
:1041A00010928F08109290088AE485DB882351F0E2
:1041B0006EDB6093910870939208809393089093BC
:1041C0009408089510929108109292081092930802
:1041D000109294080895CF92DF92EF92FF92CF93BE
:1041E000DF93EC01C090D008D090D108E090D208C5
:1041F000F090D308A7019601688179818A819B811B
:104200000E94B5B787FF04C0C882D982EA82FB82C8
:10421000C090D408D090D508E090D608F090D70888
:10422000A70196016C817D818E819F810E94B5B727
:1042300087FF04C0CC82DD82EE82FF82C090D80866
:10424000D090D908E090DA08F090DB08A701960139
:10425000688579858A859B850E94B5B787FF04C0EC
:10426000C886D986EA86FB86C0901F02D0902002BD
:10427000E0902102F0902202A701960168817981E5
:104280008A819B810E94B8B9181624F4C882D98209
:10429000EA82FB82C0902302D0902402E0902502A3
:1042A000F0902602A70196016C817D818E819F810D
:1042B0000E94B8B9181624F4CC82DD82EE82FF8207
:1042C000C0902702D0902802E0902902F0902A02A4
:1042D000A7019601688579858A859B850E94B8B972
:1042E000181624F4C886D986EA86FB86DF91CF911A
:1042F000FF90EF90DF90CF900895CF92DF92EF92F2
:10430000FF920F931F9389E998E065DF0E94A5B0A3
:104310006093D8067093D9068093DA069093DB06F3
:104320002091990830919A0840919B0850919C08DF
:104330006091E8087091E9088091EA089091EB0893
:104340000E94B5B7811179C020919D0830919E08D7
:1043500040919F085091A0086091EC087091ED0881
:104360008091EE089091EF080E94B5B7811165C069
:1043700020E030E040E752E460910A0270910B02C5
:1043800080910C0290910D020E94BCB7EBEACE2EF8
:10439000E8E0DE2E7B018C0125EA38E041EA58E0B6
:1043A0006DE978E089E998E00E94CD5880919908FC
:1043B00090919A08A0919B08B0919C088093E8087E
:1043C0009093E908A093EA08B093EB0880919D08C8
:1043D00090919E08A0919F08B091A0088093EC084E
:1043E0009093ED08A093EE08B093EF088091A10898
:1043F0009091A208A091A308B091A4088093F0081E
:104400009093F108A093F208B093F3088091A50867
:104410009091A608A091A708B091A8088093F408ED
:104420009093F508A093F608B093F7081F910F91A9
:10443000FF90EF90DF90CF90089560912D027091E2
:104440002E02882777FD8095982F0E9457B82091DB
:104450000A0230910B0240910C0250910D020E9411
:104460008ABA20E030E040E752E40E94BCB720E086
:1044700030E048EC52E488CFAF92BF92CF92DF9207
:10448000EF92FF920F931F93CF93DF93D82F20913A
:10449000910830919208409193085091940860914E
:1044A0008D0870918E0880918F08909190080E94DD
:1044B000C5B9C62F172F082FF92E60912D027091C4
:1044C0002E02882777FD8095982F0E9457B820915B
:1044D0000A0230910B0240910C0250910D020E9491
:1044E0008ABA20E030E040E752E40E94BCB720E006
:1044F00030E048EC52E40E94BCB72091AB082F9307
:10450000DF93FF920F931F93CF935B016C01F2E057
:10451000EF2E01E020E04DE858E069E978E088EE10
:1045200098E00E949E508091990890919A08A091DD
:104530009B08B0919C088093E8089093E908A093A9
:10454000EA08B093EB0880919D0890919E08A09195
:104550009F08B091A0088093EC089093ED08A09379
:10456000EE08B093EF088091A1089091A208A09165
:10457000A308B091A4088093F0089093F108A09349
:10458000F208B093F3088091A5089091A608A09135
:10459000A708B091A8088093F4089093F508A09319
:1045A000F608B093F7080E94A5B06093D806709300
:1045B000D9068093DA069093DB060F900F900F9048
:1045C0000F900F900F90DF91CF911F910F91FF905F
:1045D000EF90DF90CF90BF90AF90089520910209A7
:1045E000223111F4109204098091FE088D30E1F41B
:1045F0008091210990912209843F31E0930709F4C9
:104600002C98813D974020F01092220910922109A8
:104610008091210990912209009709F42C9A019622
:1046200090932209809321098091FE088D7F81302B
:1046300031F4223121F480911D0981112C9880914F
:104640000409882331F12091FE088EEF820F823019
:1046500010F53CB13295317040910301809103090E
:10466000837090910509813039F0833071F43111F4
:1046700005C040FD03C009C0332339F09160909319
:104680000509223041F40C94B7879078909305097E
:104690000895109205090895F8940E94F5705F9AA4
:1046A0008A9A9FB7F89480910801816080930801ED
:1046B0009FBF129A479A60E08CE00E9485B2EAE2BE
:1046C000F6E08491882341F09091C00095FFFCCFE3
:1046D0008093C6003196F5CFE1EFF1E08491882315
:1046E00041F09091C00095FFFCCF8093C6003196B9
:1046F000F5CF8091C00085FFFCCF8AE08093C60093
:1047000088EE91E00E94C887FFCFCF92DF92EF92B0
:10471000FF920F931F930E94A5B00091D4061091B1
:10472000D5062091D6063091D706C090D806D090F5
:10473000D906E090DA06F090DB066C197D098E0947
:104740009F09061717072807390728F4012B022BA2
:10475000032B09F0A1DF8091060290910702A0913E
:104760000802B0910902892B8A2B8B2BC9F1809109
:10477000FE088730D1F40E94A5B00091D8061091B0
:10478000D9062091DA063091DB06601B710B820B93
:10479000930B653C79408105910510F19091370CA0
:1047A0008091360C98131CC027C00E94A5B00091C0
:1047B000D8061091D9062091DA063091DB06601BED
:1047C000710B820B930B009106021091070220914E
:1047D000080230910902061717072807390780F0E9
:1047E0008091060182FFB6CF1F910F91FF90EF904D
:1047F000DF90CF900C94B05881E08093CB06F0CF3F
:104800009091370C8091360C9813EACF5F9A8A9A70
:104810009FB7F894809108018160809308019FBF41
:10482000129A479ADDCFCF93DF93EC018091AB08CA
:104830008093F80584E53FD8811102C080E064C010
:1048400026D80E9429B86093F8056230B8F3E4E2F4
:10485000F6E08491882341F09091C00095FFFCCF51
:104860008093C6003196F5CFC936D10599F034F45E
:10487000C836D105C9F5EEE0F3E015C0CD36D10557
:1048800031F0CA3DD10581F5E9ECF2E02AC0E0EE55
:10489000F2E01DC0E7EFF2E010C09091C00095FF7C
:1048A000FCCF8093C60081918111F7CF1DC09091FC
:1048B000C00095FFFCCF8093C60081918111F7CF96
:1048C00013C09091C00095FFFCCF8093C6008191EA
:1048D0008111F7CF09C09091C00095FFFCCF809364
:1048E000C60081918111F7CF40E050E06091F8055A
:1048F00082E795E00E94F6168091C00085FFFCCF0C
:104900008AE08093C60081E0DF91CF9108953F92C5
:104910004F925F926F927F928F929F92AF92BF92CF
:10492000CF92DF92EF92FF920F931F93CF93DF937B
:10493000CDB7DEB7A2970FB6F894DEBF0FBECDBFDE
:1049400087E40E945B1C882309F46BC40E94471C07
:104950000E9424B86A35710509F477C3ACF462305B
:10496000710509F4C0C024F477FFB5C00C94D635A6
:104970006430710509F4C7C00CF4BCC06C3171051A
:1049800009F408C10C94D6356636710509F412C4D1
:104990000CF051C06C35710509F460C30CF459C3B7
:1049A0006536710511F00C94D6358FEA93E00E94BC
:1049B000C31960911A0970911B0980911E09909189
:1049C0001F09680F791F62537109882777FD809549
:1049D000982F0E9457B86093F0087093F108809365
:1049E000F2089093F308198220E030E040EA50E4A6
:1049F00060913702709138028091390290913A02A9
:104A00000E94BCB7FE0131966F017B018C0124EF3F
:104A100038E040EF58E06CEE78E088EE98E00E94D5
:104A2000CD580E94C86B8DE08093FE088EE0809385
:104A300020090C94D635623421E0720709F4BFC313
:104A4000683E33E0730709F454C36134714011F0D8
:104A50000C94D6356091F0087091F1088091F208BD
:104A60009091F308609316097093170980931809C1
:104A70009093190920E030E040E251E40E94DCB656
:104A80006093F0087093F1088093F2089093F30814
:104A9000198220E030E040EA50E4609137027091E2
:104AA00038028091390290913A020E94BCB79E016F
:104AB0002F5F3F4F69017B018C0124EF38E040EF0D
:104AC00058E06CEE78E088EE98E00E94CD580E94A5
:104AD000C86B0C94D6358091F705811104C0CEDAED
:104AE0000CDC0C945E378091F705811103C045DB27
:104AF00081E006C08091F705811105C03EDB80E0B2
:104B0000BBDC0C945E3783EB93E00E940D8780E55D
:104B10000E945B1C882339F00E94471C0E9429B820
:104B20004B015C0103C0812C912C540183E50E9450
:104B30005B1C882361F00E94471C20E030E04AE7BC
:104B400054E40E948ABA0E9429B84B015C010E9479
:104B5000C86B0E94A5B06B017C01C80CD91CEA1C73
:104B6000FB1C0E94A5B06093D8067093D906809371
:104B7000DA069093DB060E94A5B06C157D058E05C4
:104B80009F0510F00C94D6350E94046EBEDD0E9485
:104B90005088F1CF80910A0290910B02A0910C02F3
:104BA000B0910D028093790890937A08A0937B08C6
:104BB000B0937C0880912D0290912E029093F90879
:104BC0008093F80884E690E090932E0280932D0263
:104BD0000E94A5B06093D8067093D9068093DA0638
:104BE0009093DB0681E00E9498648091E8089091A0
:104BF000E908A091EA08B091EB0880939908909396
:104C00009A08A0939B08B0939C088091EC0890911F
:104C1000ED08A091EE08B091EF0880939D08909365
:104C20009E08A0939F08B093A0088091F0089091EF
:104C3000F108A091F208B091F3088093A108909335
:104C4000A208A093A308B093A4088091F4089091BF
:104C5000F508A091F608B091F7088093A508909305
:104C6000A608A093A708B093A80810920A02109271
:104C70000B0210920C0210920D0288E50E945B1C40
:104C8000882311F010E00AC089E50E945B1C8111A5
:104C9000F9CF8AE50E945B1C11E0182710930E02E1
:104CA00088E50E945B1CB82E80910209813109F0D1
:104CB0005DC0111103C0BB2009F458C020E030E0F2
:104CC00040EC50E46091890870918A0880918B08CB
:104CD00090918C080E94B5B787FF48C020E030E073
:104CE00040EC50E46091F0087091F1088091F20876
:104CF0009091F3080E94B5B787FF38C040E050E0BC
:104D000060EC70E44093F0085093F1086093F2086F
:104D10007093F3083BEAC32E38E0D32EE12CF12C3C
:104D200000E810E424EF38E040EF58E06CEE78E063
:104D300088EE98E00E94CD580E94C86B4091F00820
:104D40005091F1086091F2087091F308409389083E
:104D500050938A0860938B0870938C081092F00827
:104D60001092F1081092F2081092F30880910E024E
:104D700081110C94D93589E50E945B1C81110C943A
:104D8000D93580910E02811103C0BB2009F45BC0AC
:104D900080E090E00E94961780910209813109F02D
:104DA00052C06091140970911509882777FD80958C
:104DB000982F0E9457B86B017C019B01AC01609158
:104DC000E8087091E9088091EA089091EB080E9448
:104DD000B5B787FF38C08091030981FF34C0C09206
:104DE000E808D092E908E092EA08F092EB089BEA22
:104DF000C92E98E0D92EE12CF12C00EF11E424EF1C
:104E000038E040EF58E06CEE78E088EE98E00E94E1
:104E1000CD580E94C86B8091E8089091E908A09154
:104E2000EA08B091EB088093810890938208A093E0
:104E30008308B09384081092E8081092E908109251
:104E4000EA081092EB0880910E02882321F082E09C
:104E500090E00E9496178AE50E945B1C882309F463
:104E60005BC080910209813109F052C06091140940
:104E700070911509882777FD8095982F0E9457B863
:104E80006B017C019B01AC016091810870918208EB
:104E900080918308909184080E94B5B787FF38C03D
:104EA0008091030981FF34C0C092E808D092E908DC
:104EB000E092EA08F092EB080BEAC02E08E0D02E50
:104EC000E12CF12C00EF11E424EF38E040EF58E042
:104ED0006CEE78E088EE98E00E94CD580E94C86B96
:104EE0008091E8089091E908A091EA08B091EB0858
:104EF0008093810890938208A0938308B0938408DC
:104F00001092E8081092E9081092EA081092EB0853
:104F100082E090E00E94961788E50E945B1C88233F
:104F2000D1F00E94501C672B682B692BA1F00E94C6
:104F3000471C2091DC083091DD084091DE0850913B
:104F4000DF080E94DCB66093E8087093E90880935C
:104F5000EA089093EB0889E50E945B1C8823D1F056
:104F60000E94501C672B682B692BA1F00E94471CE4
:104F70002091E0083091E1084091E2085091E30867
:104F80000E94DCB66093EC087093ED088093EE0805
:104F90009093EF088AE50E945B1C8823D1F00E9461
:104FA000501C672B682B692BA1F00E94471C209195
:104FB000E4083091E5084091E6085091E7080E9426
:104FC000DCB66093F0087093F1088093F208909338
:104FD000F30824EF38E040EF58E06CEE78E088EE1C
:104FE00098E00E94E36280E00E94986480917908D2
:104FF00090917A08A0917B08B0917C0880930A0276
:1050000090930B02A0930C02B0930D028091F808CC
:105010009091F90890932E0280932D020E94A5B0E2
:105020006093D8067093D9068093DA069093DB06D6
:105030000E9491648091FE08853011F00C94D63561
:1050400086E08093FE080C94D63510926C080C9480
:10505000D63581E080936C080C94D63585E40E94A7
:105060005B1C811102C00E94C86BB9ECCB2EB3E06F
:10507000DB2E1CEDE12E18E0F12E08EE18E0B12C2D
:10508000D6018D916D010E945B1C882339F1B3E03C
:10509000BB120CC00E94471CF8016083718382839D
:1050A000938384EF98E00E94886318C00E94471C95
:1050B000D7012D913D914D915C910E94DCB6F80194
:1050C000608371838283938324EF38E040EF58E05C
:1050D0006CEE78E088EE98E00E94E362B394F4E02E
:1050E000EF0EF11C0C5F1F4F24E0B212C9CF0C94DD
:1050F000D6358FE0809320091092E8081092E908D5
:105100001092EA081092EB0824EF38E040EF58E0E4
:105110006CEE78E088EE98E00E94E3621092EC0872
:105120001092ED081092EE081092EF0824EF38E08C
:1051300040EF58E06CEE78E088EE98E00E94E36281
:1051400060911A0970911B0980911E0990911F09A5
:10515000680F791F882777FD8095982F0E9457B890
:105160006093F0087093F1088093F2089093F3082D
:10517000198220E030E040EA50E4609137027091FB
:1051800038028091390290913A020E94BCB7DE0148
:1051900011966D017B018C0124EF38E040EF58E05F
:1051A0006CEE78E088EE98E00E94CD580E94C86BC3
:1051B0000C94D63581E080931C090C94D6358091EF
:1051C000160990911709A0911809B09119098093B7
:1051D000F0089093F108A093F208B093F3081982B5
:1051E00020E030E040EA50E46091370270913802EC
:1051F0008091390290913A020E94BCB7DE0111966B
:105200006D017B018C0124EF38E040EF58E06CEE3B
:1052100078E088EE98E00E94CD580E94C86B0C940C
:10522000D6358DE40E945B1C882311F40C948034E5
:105230000E94471C0E9424B86A36710509F4DBC538
:105240000CF0A1C06B31710509F417C20CF051C00C
:105250006431710509F4B1C1FCF46330710509F4DE
:1052600092C134F46230710508F433C10C94D63520
:105270006131710509F48FC16231710509F4FBC513
:105280006530710511F00C94D6350E94C86B2C98CE
:1052900010921D090C94D6356731710509F4C1C10E
:1052A0007CF46531710509F4B6C16631710511F000
:1052B0000C94D63583E299E00E94B24A0C94D6351C
:1052C0006931710509F4C5C10CF0C9C183E299E0E7
:1052D0000E94B64A0E94A5B06093D0067093D10692
:1052E0008093D2069093D30682E08093FE080C94BC
:1052F000D6356235710509F4B7C5DCF46F31710537
:1053000009F468C254F46C31710509F4BCC16E3102
:10531000710509F4EDC10C94D6356035710509F4B9
:105320009DC50CF09EC56A32710509F4DAC20C9471
:10533000D6356535710509F4D3C554F46335710567
:1053400009F495C56435710509F495C50C94D635F5
:105350006836710509F4F0C20CF01DC36C35710597
:1053600011F00C94D63529EC33E038A32F8F0DE6DD
:1053700011E13DE7832E31E1932E4DE2A42E41E170
:10538000B42E312C24C66D3C710511F40C94E4311B
:105390000CF045C06837710509F436C7FCF4623774
:1053A000710509F452C654F46B36710509F451C500
:1053B0006D36710509F4DEC30C94D6356537710579
:1053C00009F422C66737710509F480C06337710597
:1053D00011F00C94D635E5E7F2E012C66E3B71058C
:1053E00009F447C454F46937710509F411C76C38DE
:1053F000710509F4BFC20C94D6356B3C710509F4F4
:10540000A7C70CF0C1C7693C710511F00C94D635E3
:1054100009EC13E02DE5E22E21E1F22E7FC76E327A
:10542000B1E07B0711F40C941A3414F56C3D71054E
:1054300011F40C94083364F46E3C710511F40C946F
:1054400051326A3D710511F40C946D320C94D635CD
:105450006C32F1E07F0711F40C94263314F00C94B5
:1054600054336D3D710511F40C9417330C94D635FB
:10547000653F31E0730711F40C9466349CF4603995
:1054800091E0790711F40C946034643FA1E07A074D
:1054900011F40C9463346F32714011F00C94D635D2
:1054A0000C942834603AE3E07E0709F45FC1673E5C
:1054B000F3E07F0711F40C946934663F714011F0FA
:1054C0000C94D6350E94DB120C94D635E4E3F3E05D
:1054D000A9C68EE993E00E940D8780E50E945B1CBF
:1054E000882339F00E94471C0E9429B86B017C0177
:1054F00003C0C12CD12C760183E50E945B1C88235C
:1055000061F00E94471C20E030E04AE754E40E942A
:105510008ABA0E9429B86B017C010E94C86B0E9464
:10552000A5B06093D8067093D9068093DA0690935D
:10553000DB06C114D104E104F104A9F00E94A5B076
:105540004B015C018C0C9D1CAE1CBF1C0E94A5B0C5
:10555000681579058A059B0580F40E94568981119A
:105560000CC00C94DF350E945689811106C00E9440
:10557000046ECBD80E945088F6CF81E993E00E9458
:105580000D870C94D6350E94C86B2C9A81E08093CD
:105590001D090C94D63588E893E00E940D875F982A
:1055A0008A989FB7F894809108018E7F80930801B4
:1055B0009FBF129847980C94D635E8E7F3E08491A2
:1055C000882341F09091C00095FFFCCF8093C600E6
:1055D0003196F5CF8091C00085FFFCCF8AE08093A3
:1055E000C60083E299E00E949849EAE6F3E08491DC
:1055F000882341F09091C00095FFFCCF8093C600B6
:105600003196F5CF8091C00085FFFCCF8AE0809372
:10561000C6000C94D63583E299E00E94EF490C94C1
:10562000D6350091DC061091DD060C5F1F4F6AE253
:1056300070E0C8010E94FFBE009719F0FC0131978D
:10564000108241E0B80183E299E00E94C24A0C94C2
:10565000D63583E299E00E94BD4A0C94D6358091FC
:105660002609882311F40C94D63583E50E945B1C2F
:1056700081110C94E7350C94D63583E299E00E94B1
:10568000E34D0C94D6358091DC069091DD066AE2FC
:1056900070E004960E94FFBE8C010097E1F020911B
:1056A000E6063091E70640E6429FC001439F900D19
:1056B00011246EE470E08451994F0E94FFBE60E2B5
:1056C00070E00E94FFBE01969093DD068093DC0699
:1056D000F801319710826091DC067091DD066C5FF5
:1056E0007F4F40E083E299E00E94C24A0C94D63595
:1056F00080912609882311F40C94D63583E299E031
:105700000E949C4F8091DC069091DD066AE270E079
:1057100004960E94FFBE8C010097E1F02091E606FE
:105720003091E70640E6429FC001439F900D11244F
:105730006EE470E08451994F0E94FFBE60E270E019
:105740000E94FFBE01969093DD068093DC06F8016F
:10575000319710826091DC067091DD066C5F7F4F9F
:1057600083E299E00E94AA4C0C94D6358091DC0625
:105770009091DD066AE270E005960E94FFBE8C0102
:105780000097E1F02091E6063091E70640E6429F5F
:10579000C001439F900D11246EE470E08451994F35
:1057A0000E94FFBE60E270E00E94FFBE01969093EF
:1057B000DD068093DC06F801319710826091DC06EB
:1057C0007091DD066B5F7F4F83E299E00E94A54CEC
:1057D0000C94D6350E94A5B06093CC067093CD068C
:1057E0008093CE069093CF060091D0061091D106FB
:1057F0002091D2063091D306601B710B820B930B64
:1058000028EE33E040E050E00E9486BBCA01B901B7
:105810002CE330E040E050E00E9486BB7F936F9322
:105820003F932F938BE593E09F938F93CE01019647
:105830009F938F930E94A6BFE4E2F6E084910FB697
:10584000F894DEBF0FBECDBF882349F09091C00011
:1058500095FFFCCF8093C60031968491F5CFFE0171
:1058600031968191882339F09091C00095FFFCCF4B
:105870008093C600F6CF8091C00085FFFCCF8AE000
:105880008093C600CE0101960E94FE868091081189
:10589000882311F40C94D635109208110091AB08AE
:1058A00010E0000F111F0C5A1D4EF801608171812C
:1058B000882777FD8095982F0E9457B8209147023E
:1058C000309148024091490250914A020E94B8B971
:1058D000181614F00C94D635D8011D921C920C9415
:1058E000D63583E50E945B1C882311F40C94D635D1
:1058F0000E94471C6B017C0180E50E945B1C882391
:1059000051F0C701B6010E9424B86F3F710509F03C
:1059100010F40C94F7356DE070E020E0E22FEE0F0C
:10592000FF0BE757FC4F808191818617970711F491
:105930000C94D6352F5FF2CF88E690E00E941324B6
:1059400081110C94D63583E50E945B1C882371F08D
:105950000091F8050E94471C10E0000F111F0C5A1F
:105960001D4E0E9424B8F801718360830E94F47078
:105970000C94D63583E50E945B1C882311F40C94AB
:10598000D6350E94471C0E9424B87093531260932E
:1059900052120C94D63589E690E00E9413248111AE
:1059A0000C94D635E4E5F3E08491882341F090919E
:1059B000C00095FFFCCF8093C6003196F5CF409193
:1059C000461250914712609148127091491221E09D
:1059D00030E082E795E00E949517E1E5F3E08491DD
:1059E000882341F09091C00095FFFCCF8093C600C2
:1059F0003196F5CF6091541270915512882777FD3A
:105A00008095982F0E9457B8AB01BC0121E030E08F
:105A100082E795E00E949517ECE4F3E084918823F7
:105A200041F09091C00095FFFCCF8093C600319665
:105A3000F5CF40914A1250914B1260914C127091E7
:105A40004D1221E030E082E795E00E949517E9E4ED
:105A5000F3E08491882341F09091C00095FFFCCF42
:105A60008093C6003196F5CF60915612709157120F
:105A7000882777FD8095982F0E9457B8AB01BC010D
:105A800021E030E082E795E00E949517E5E4F3E03D
:105A90008491882341F09091C00095FFFCCF8093C2
:105AA000C6003196F5CF409140125091411260915D
:105AB00042127091431221E030E082E795E00E94AB
:105AC0009517E2E4F3E08491882341F09091C000BF
:105AD00095FFFCCF8093C6003196F5CF60915212AE
:105AE00070915312882777FD8095982F0E9457B8A0
:105AF000AB01BC0121E030E082E795E00E94951700
:105B0000EEE3F3E08491882341F09091C00095FF8B
:105B1000FCCF8093C6003196F5CF8091F80590E0D8
:105B20000E94F96D4AE050E0BC0182E795E00E94D6
:105B3000BF16E9E3F3E08491882341F09091C0001F
:105B400095FFFCCF8093C6003196F5CF8FEF9FEF86
:105B50000E94F96D4AE050E0BC0182E795E00E94A6
:105B6000BF168091C00085FFFCCF8AE08093C600FD
:105B70000C94D6358DE690E00E94132481110C948C
:105B8000D6358EE293E00E940D871092081183E5CE
:105B90000E945B1C882371F00091F8050E94471C4D
:105BA00010E0000F111F0C5A1D4E0E9424B8D8019E
:105BB0006D937C9383E50E945B1C882351F00E94C7
:105BC000471C609347027093480280934902909368
:105BD0004A0282E40E945B1C882351F00E94471C09
:105BE00060934B0270934C0280934D0290934E024F
:105BF00086E40E945B1C882369F00E94471C609326
:105C0000430270934402809345029093460281E0E0
:105C1000809308110E94F4700E94A5B04B015C01B2
:105C20000091F80510E0F801EE0FFF1FEC5AFD4E51
:105C300060817181882777FD8095982F0E9457B8E1
:105C40002B013C01F801EE0FFF1FEE0FFF1FEA5B77
:105C5000FD4E80819181A281B3818F8F98A3A9A3EA
:105C6000BAA3CC24CA94DC2C76016AE0362E0C94BC
:105C7000623680910709811199C786E093E00E94FE
:105C80000D8783E50E945B1C882341F00E94471C1E
:105C90000E9424B870935312609352120E94A5B0D0
:105CA0004B015C0102E013E05DEFE52E52E0F52EC2
:105CB00069EFC62E62E0D62E7AE0772E60915212FE
:105CC00070915312882777FD8095982F0E9457B8BE
:105CD0002091401230914112409142125091431252
:105CE0000E94B8B918160CF077C00E94A5B06819C8
:105CF00079098A099B09693E73408105910508F479
:105D000061C0F8018491E2E0F3E0882349F09091CA
:105D1000C00095FFFCCF8093C60031968491F5CFEB
:105D20004091461250914712609148127091491269
:105D300022E030E082E795E00E949517F701849118
:105D4000EDEFF2E0882349F09091C00095FFFCCF81
:105D50008093C60031968491F5CF40914A125091BC
:105D60004B1260914C1270914D1222E030E082E7AC
:105D700095E00E949517F6018491E9EFF2E08823FF
:105D800049F09091C00095FFFCCF8093C6003196FA
:105D90008491F5CF4091401250914112609142128E
:105DA0007091431221E030E082E795E00E94951760
:105DB0008091C00085FFFCCF7092C6000E94A5B004
:105DC0004B015C010E94046E0E9485230E94508852
:105DD00080910909811172CF8FEE92E00E940D87A8
:105DE0000E94A5B06093D8067093D9068093DA0616
:105DF0009093DB06DBC683E50E945B1C882311F1D0
:105E00000E94471C20E030E0A9010E94B5B787FD41
:105E10000FC00E94471C20E030E04FE753E40E948F
:105E2000B8B9181644F00E94471C0E9424B805C057
:105E300060E070E002C06FEF70E07093AA086093BA
:105E4000A908B4C68FEF90E09093AA088093A908A0
:105E5000ADC61092AA081092A908A8C6269A2E9834
:105E6000A5C6269A2E9AA2C61092FD089FC681E06A
:105E70008093FD089BC683E50E945B1C882399F0F4
:105E80000E94471C20E030E04AE754E40E948ABAAE
:105E90000E9429B86093060270930702809308025B
:105EA000909309021AC088E50E945B1C8111E4C727
:105EB00089E50E945B1C8111DFC78AE50E945B1C9B
:105EC0008111DAC785E40E945B1C8111D5C70E944D
:105ED000C86B129A479A0E94306C1092010966C6EC
:105EE00083E50E945B1C0E94471C20E030E04AE7EB
:105EF00054E40E948ABA0E9429B86093D406709331
:105F0000D5068093D6069093D70650C6B3E03B12D1
:105F100068C00E94471C6B017C0120E030E040EA31
:105F200051E40E94B5B787FF3FC0A7019601F80171
:105F300060817181828193810E94BCB72B013C01F9
:105F40009B01AC016091411170914211809143110C
:105F5000909144110E948ABA60934111709342114A
:105F60008093431190934411A3019201D4016D9148
:105F70007D918D919C910E948ABAF4016083718316
:105F800082839383D5016D917D918D919C910E9427
:105F900055B8A30192010E948ABA0E9429B8F5015E
:105FA0006083718382839383D801CD92DD92ED92D9
:105FB000FC92139733940C5F1F4FF4E08F0E911CEB
:105FC00024E0A20EB11C34E0331609F4EFC5AF8D06
:105FD000B8A18D91B8A3AF8F0E945B1C882351F3A9
:105FE00095CF0E94471CF80160837183828393835D
:105FF000E1CF9091C00095FFFCCF8093C600319611
:1060000084918111F6CFD2C50091DC061091DD0696
:106010000B5F1F4F6AE270E0C8010E94FFBE00974D
:1060200019F0FC0131971082C8010E94FE860E947F
:10603000A5B06093D0067093D1068093D20690935A
:10604000D30681E080930109B1C5E2E7F2E08491D3
:10605000882341F09091C00095FFFCCF8093C6004B
:106060003196F5CF4091E8085091E9086091EA082F
:106070007091EB0822E030E082E795E00E949517EE
:10608000EFE6F2E08491882341F09091C00095FF03
:10609000FCCF8093C6003196F5CF4091EC0850912B
:1060A000ED086091EE087091EF0822E030E082E7A1
:1060B00095E00E949517ECE6F2E08491882341F088
:1060C0009091C00095FFFCCF8093C6003196F5CF2C
:1060D0004091F0085091F1086091F2087091F30836
:1060E00022E030E082E795E00E949517E9E6F2E0D1
:1060F0008491882341F09091C00095FFFCCF80935C
:10610000C6003196F5CF4091F4085091F5086091A2
:10611000F6087091F70822E030E082E795E00E94EF
:106120009517EFE5F2E08491882341F09091C0004B
:1061300095FFFCCF8093C6003196F5CF0E94226C6C
:106140000E9457B820916D1130916E1140916F11DE
:10615000509170110E94BCB7AB01BC0122E030E04D
:1061600082E795E00E949517ECE5F2E084918823A0
:1061700041F09091C00095FFFCCF8093C60031960E
:10618000F5CF81E00E94226C0E9457B820917111D6
:106190003091721140917311509174110E94BCB7EB
:1061A000AB01BC0122E030E082E795E00E94951748
:1061B000E9E5F2E08491882341F09091C00095FFD9
:1061C000FCCF8093C6003196F5CF82E00E94226C0E
:1061D0000E9457B820917511309176114091771136
:1061E000509178110E94BCB7AB01BC0122E030E0B5
:1061F00082E795E00E9495178091C00085FFFCCF53
:106200008AE08093C600D2C480E00E949864CEC425
:1062100081E00E949864CAC49091C00095FFFCCFB1
:106220008093C60081918111F7CF8091C00085FFD6
:10623000FCCF8AE08093C600E1E5F2E084918823F8
:1062400041F09091C00095FFFCCF8093C60031963D
:10625000F5CF659903C0E5E2F3E009C0EFE2F3E0B2
:1062600006C09091C00095FFFCCF8093C60081913D
:106270008111F7CF8091C00085FFFCCF8AE0809329
:10628000C600E9E4F2E08491882341F09091C000D7
:1062900095FFFCCF8093C6003196F5CF8091030126
:1062A00081FD03C0E5E2F3E009C0EFE2F3E006C0E0
:1062B0009091C00095FFFCCF8093C6008191811121
:1062C000F7CF8091C00085FFFCCF8AE08093C600A5
:1062D000E1E4F2E08491882341F09091C00095FFC1
:1062E000FCCF8093C6003196F5CF4B9903C0E5E211
:1062F000F3E009C0EFE2F3E006C09091C00095FF23
:10630000FCCF8093C60081918111F7CF8091C000AE
:1063100085FFFCCF8AE08093C60048C4D8018D91E8
:106320008D010E945B1C882349F00E94471C0E943B
:1063300029B8F7016083718382839383F4E0EF0EC1
:10634000F11C23E00D3C120749F70E94AE632EC4F6
:1063500009EC13E09DE7E92E91E1F92ED8018D912A
:106360008D010E945B1C882339F00E94471CF701B5
:106370006083718382839383F4E0EF0EF11C23E04A
:106380000D3C120759F712C483E50E945B1C882359
:1063900051F00E94471C60935511709356118093E1
:1063A00057119093581184E50E945B1C882309F4CF
:1063B000FDC30E94471C609351117093521180934A
:1063C000531190935411F2C383E50E945B1C882300
:1063D00051F00E94471C6093591170935A11809399
:1063E0005B1190935C1184E50E945B1C882351F043
:1063F0000E94471C60933D1170933E1180933F11A2
:106400009093401182E40E945B1C882361F00E94FB
:10641000471C0E9429B860938D1170938E11809350
:106420008F119093901188E50E945B1C882351F096
:106430000E94471C60934D1170934E1180934F1131
:106440009093501189E50E945B1C882351F00E94B3
:10645000471C6093491170934A1180934B1190939C
:106460004C118AE50E945B1C882351F00E94471C56
:106470006093451170934611809347119093481192
:1064800085E40E945B1C882309F490C30E94471C8A
:106490006093411170934211809343119093441182
:1064A00085C309EC13E08CEDE82E88E0F82ED801C6
:1064B0008D918D010E945B1C882339F00E94471C3E
:1064C000F7016083718382839383F4E0EF0EF11C04
:1064D00023E00C3C120759F769C38AED90E00E9453
:1064E0001324811163C388E50E945B1C882381F01B
:1064F0000091F80510E00E94471CF801EE0FFF1F05
:10650000EE0FFF1FE15FFD4F6083718382839383F2
:1065100089E50E945B1C882381F00091F80510E05A
:106520000E94471CF801EE0FFF1FEE0FFF1FE95EF0
:10653000FD4F6083718382839383E4E2F6E084916C
:10654000882341F09091C00095FFFCCF8093C60056
:106550003196F5CFE1E3F2E08491882341F0909108
:10656000C00095FFFCCF8093C6003196F5CF109206
:10657000F8058091F805823008F042C0ECEBF4E0B9
:106580008191882339F09091C00095FFFCCF8093D2
:10659000C600F6CFE091F80534E0E39FF001112446
:1065A000E15FFD4F408151816281738122E030E0E3
:1065B00082E795E00E949517EFE4F3E0819188234C
:1065C00039F09091C00095FFFCCF8093C600F6CFC4
:1065D000E091F80584E0E89FF0011124E95EFD4FA9
:1065E000408151816281738122E030E082E795E051
:1065F0000E9495178091F8058F5F8093F805B9CFB9
:106600008091C00085FFFCCF8AE08093C600CEC297
:1066100083E50E945B1C882309F4C8C20E94471CC2
:106620000E9424B870932E0260932D02BFC283E5AE
:106630000E945B1C882309F4B9C20E94471C0E9477
:1066400024B870932C0260932B02B0C283E50E94A1
:106650005B1C882331F00E94471C0E9424B88B01E8
:1066600002C000E911E080E50E945B1C882331F044
:106670000E94471C0E9424B87B0104C058EEE52EFE
:1066800053E0F52E20E030E0A901B80185E20E9438
:1066900039B3B701882777FD8095982F0E94D4B031
:1066A00085E20E945AB682C280E50E945B1C882364
:1066B00051F00E94471C6093690270936A028093B4
:1066C0006B0290936C0289E40E945B1C882361F04A
:1066D0000E94471C0E94BE7660936502709366021A
:1066E000809367029093680284E40E945B1C882375
:1066F00061F00E94471C0E94CA7660936102709309
:106700006202809363029093640283E40E945B1CA4
:10671000882351F00E94471C60935D0270935E02D3
:1067200080935F02909360020E94DA6DE1E5F3E0EE
:106730008191882339F09091C00095FFFCCF809320
:10674000C600F6CFE4E5F3E08191882339F090911B
:10675000C00095FFFCCF8093C600F6CF4091690240
:1067600050916A0260916B0270916C0222E030E0FD
:1067700082E795E00E949517E8E5F3E08191882390
:1067800039F09091C00095FFFCCF8093C600F6CF02
:106790006091650270916602809167029091680233
:1067A0000E94C476AB01BC0122E030E082E795E0B4
:1067B0000E949517ECE5F3E08191882339F09091E0
:1067C000C00095FFFCCF8093C600F6CF60916102B8
:1067D0007091620280916302909164020E94D0766F
:1067E000AB01BC0122E030E082E795E00E94951702
:1067F000E0E6F3E08191882339F09091C00095FFA5
:10680000FCCF8093C600F6CF40915D0250915E02AE
:1068100060915F027091600222E030E082E795E0D3
:106820000E9495178091C00085FFFCCF8AE080937D
:10683000C600BCC183E50E945B1C882319F00E943E
:10684000471C03C060E070E0CB010E94A563AEC1AD
:1068500085E40E945B1C882341F00E94471C0E9433
:1068600024B88B0177FD0AC002C000E010E0C12C03
:10687000D12C46E1E42E43E4F42E06C0C12CD12CE9
:106880003CE8E32E32E4F32E83E50E945B1C882370
:1068900021F00E94471C6B017C0183E40E945B1C79
:1068A000882331F00E94471C0E9424B89B0102C03B
:1068B00025E030E0A801C701B6010E941B7176C136
:1068C0000E94C86B73C10E94D71170C10E947114DD
:1068D0006DC11092F7050E94CE8780916D0890914E
:1068E0006E08A0916F08B091700880937108909322
:1068F0007208A0937308B09374080E949F1C56C13D
:1069000084E50E945B1C882309F40CC10E94471C8B
:106910000E9429B86093F8056230A8F1E4E2F6E03D
:106920008491882341F09091C00095FFFCCF809323
:10693000C6003196F5CFE4E6F3E08191882339F083
:106940009091C00095FFFCCF8093C600F6CF40E049
:1069500050E06091F80582E795E00E94F616E6E6C1
:10696000F3E08191882339F09091C00095FFFCCF2E
:106970008093C600F6CF8091C00085FFFCCF8AE0EF
:106980008093C60013C186E40E945B1C8823E1F05B
:106990000E94471C6B017C0160937D0870937E0808
:1069A00080937F089093800820E030E0A9010E9446
:1069B000B8B918165CF4C0920A02D0920B02E092A9
:1069C0000C02F0920D0202C0D12C02C0DD24D3943F
:1069D000C090F805E090AB08CE1409F479C080E1CE
:1069E000E8EEF8E0A9E9B8E001900D928A95E1F7A8
:1069F00080910109882309F457C0F12C0C2D10E077
:106A0000F701EE0FFF1FEE0FFF1FE15FFD4F20812B
:106A10003181428153816091E8087091E908809149
:106A2000EA089091EB080E94DBB6F801EE0FFF1F19
:106A3000EE0FFF1FE15FFD4F2081318142815381C5
:106A40000E94DCB66093E8087093E9088093EA0836
:106A50009093EB08F701EE0FFF1FEE0FFF1FE95EAB
:106A6000FD4F20813181428153816091EC0870910A
:106A7000ED088091EE089091EF080E94DBB6F801D6
:106A8000EE0FFF1FEE0FFF1FE95EFD4F20813181EA
:106A9000428153810E94DCB66093EC087093ED084C
:106AA0008093EE089093EF08C092AB0824EF38E093
:106AB00040EF58E06CEE78E088EE98E00E94E362E8
:106AC000DD2031F08091F705811102C00E947D2107
:106AD000E4E2F6E08491882341F09091C00095FFB4
:106AE000FCCF8093C6003196F5CFE7E7F3E08191C4
:106AF000882339F09091C00095FFFCCF8093C600A9
:106B0000F6CF6091AB0870E04AE050E082E795E094
:106B10000E94BF168091C00085FFFCCF8AE0809361
:106B2000C60044C0E4E2F6E08491882341F09091ED
:106B3000C00095FFFCCF8093C6003196F5CFEEE103
:106B4000F2E08491882341F09091C00095FFFCCF42
:106B50008093C6003196F5CF8091E6069091E706C6
:106B600020E6289FF001299FF00D1124E451F94FF0
:106B70008191882339F09091C00095FFFCCF8093DC
:106B8000C600F6CFECE1F2E08491882341F09091C9
:106B9000C00095FFFCCF8093C6003196F5CF809161
:106BA000C00085FFFCCF8AE08093C6000E94771C5E
:106BB00085C181E090E00E9496170C94C1260E9446
:106BC000046E0E9485230E9450880C94A62A0E947D
:106BD000501CAB01BC0140931A0A50931B0A6093EE
:106BE0001C0A70931D0A87EF99E0ACD7DFCF0E9493
:106BF000471C0E9424B80C948D2C0E94A5B08B01D8
:106C00009C01C701B6016053784F8F4F9F4F601BA7
:106C1000710B820B930B28EE33E040E050E00E94B2
:106C200086BBBA01A9012AE030E082E795E00E9424
:106C3000EB168091C00085FFFCCF3092C6000E9409
:106C4000A5B04B015C010E94046E0E9485230E9446
:106C50005088FFEFCF16DF06EF06FF0609F0ACC045
:106C60002F8D38A149A15AA1C301B2010E94B8B920
:106C7000E091F805F0E08F01000F111F000F111FC8
:106C80000A5B1D4EEE0FFF1FEC5AFD4E60817181B5
:106C900018160CF079C0882777FD8095982F0E94F0
:106CA00057B820E030E040EA50E40E94DBB69B0198
:106CB000AC01D8016D917D918D919C910E94B8B9E4
:106CC00087FFB6C00E94A5B0681979098A099B0997
:106CD000693E73408105910508F4B5CFEAE2F3E01F
:106CE0008491882341F09091C00095FFFCCF809360
:106CF000C6003196F5CF40914612509147126091EF
:106D000048127091491222E030E082E795E00E943B
:106D10009517E5E2F3E08491882341F09091C0005B
:106D200095FFFCCF8093C6003196F5CF40914A1273
:106D300050914B1260914C1270914D1222E030E054
:106D400082E795E00E949517E1E2F3E084918823C1
:106D500041F09091C00095FFFCCF8093C600319622
:106D6000F5CFF7FE4ACFEDE4F3E006C09091C00006
:106D700095FFFCCF8093C60081918111F7CF809160
:106D8000C00085FFFCCF59CF882777FD8095982FCD
:106D90000E9457B820E030E040EA50E40E94DCB6A0
:106DA0009B01AC01F80160817181828193810E9415
:106DB000B5B71816ECF586CFF7FC2FC0E091F805B3
:106DC000F0E08F01000F111F000F111F0A5B1D4E15
:106DD000EE0FFF1FEC5AFD4E60817181882777FD11
:106DE0008095982F0E9457B89B01AC01D8016D91F6
:106DF0007D918D919C910E94DBB60E9424B897FFF3
:106E000007C090958095709561957F4F8F4F9F4FEC
:106E100067307105810591055CF4F7FC14C00E9490
:106E2000A5B06C197D09603D774008F44BCF0BC0CD
:106E30000E94A5B06B017C019FEFC916D906E90637
:106E4000F90659F73FCF83E193E00E940D870E9436
:106E5000A5B06093D0067093D1068093D20690932C
:106E6000D3060E94A5B06093D8067093D90680938C
:106E7000DA069093DB069ACE0E94C86B88E50E94E2
:106E80005B1C81115F9A89E50E945B1C81118A9AC3
:106E90008AE50E945B1C882341F09FB7F89480919B
:106EA00008018160809308019FBF85E40E945B1CFC
:106EB000882309F412C8129A479A0FC8A2960FB6EF
:106EC000F894DEBF0FBECDBFDF91CF911F910F9120
:106ED000FF90EF90DF90CF90BF90AF909F908F90FA
:106EE0007F906F905F904F903F900895CF93DF9386
:106EF0008091E2069091E306039714F40E94C81C67
:106F000060E083E299E00E94A84E8091E2069091B1
:106F1000E306892B09F463C0809123098823E1F0FB
:106F20008091E6069091E70620E6289FE001299FE0
:106F3000D00D1124C451D94F61E275E0CE010E94F9
:106F4000C4BE892BF1F4BE0183E299E00E94384E61
:106F500080912409882319F00E9487242AC0EEE139
:106F6000F5E08491882341F09091C00095FFFCCF1B
:106F70008093C6003196F5CF8091C00085FFFCCF8D
:106F800015C083E299E00E949C4FECE0F5E084910B
:106F9000882341F09091C00095FFFCCF8093C600FC
:106FA0003196F5CF8091C00085FFFCCF8AE08093B9
:106FB000C6008091E2069091E30601979093E30664
:106FC0008093E2068091E6069091E706019664E0E0
:106FD00070E00E9473BB9093E7068093E6060E94E0
:106FE000046E0E9485230E94F6630E94EE22DF91C8
:106FF000CF910C94508821ED33E0FC013183208344
:107000002781222311F0049680C6089583E299E037
:107010000C94B34783EF99E0EEDF81EB99E0EBDF6F
:1070200082E999E0E8DF83E799E0E5DF82E599E02E
:10703000E2CF8FEF8EBD0DB407FEFDCF8EB5089564
:107040008EBD0DB407FEFDCF089561E0FC01808187
:107050000C94BEB2FC012281322F306A36953CBDC1
:1070600020FD06C031E0263009F430E0232F01C0B6
:1070700020E02DBD60E0FC0180810C94BEB2CF9277
:10708000DF92EF92FF920F931F93CF93DF93EC0168
:107090008B017A010E94A5B06B01CBDF8B838F3F00
:1070A00049F40E94A5B06C197D096D327140A8F3B6
:1070B00081E103C08E3F31F08FE08983CE01C5DFCF
:1070C00080E024C0E114F104E1F081E0E81AF10865
:1070D0008FEF8EBDF8012FEFCF01801B910B8E1526
:1070E0009F0538F40DB407FEFDCF8EB581932EBDFC
:1070F000F3CF0DB407FEFDCF8EB5F801EE0DFF1DE9
:10710000808397DF96DFCE01A0DF81E0DF91CF9112
:107110001F910F91FF90EF90DF90CF9008950F9304
:107120001F93CF93DF93EB010E94A5B08B0181DF0A
:107130008F3F49F00E94A5B0601B710B6C177D0753
:10714000B0F380E001C081E0DF91CF911F910F91FA
:107150000895CF92DF92FF920F931F93CF93DF9307
:1071600000D01F92CDB7DEB76C01F62E29833A838B
:107170004B835C836FDF6CE271E0C601D0DF8F2D43
:1071800080645EDF08E110E05C814B813A812981F7
:10719000DA01C901002E04C0B695A7959795879589
:1071A0000A94D2F729833A834B835C8349DF0850E2
:1071B000110929813A814B815C81083F8FEF1807C3
:1071C00039F7FF2029F0E8E0FE1621F08FEF03C029
:1071D00085E901C087E834DFFCE0FF1201C029DF48
:1071E00010E027DFF601838387FF04C01F3F11F003
:1071F0001F5FF7CF0F900F900F900F90DF91CF91FF
:107200001F910F91FF90DF90CF900895BF92CF9282
:10721000DF92EF92FF920F931F93CF93DF93EC01D6
:10722000B62E1C82198248830E94A5B08B0161E0B2
:1072300088810E9485B2CE0108DF60E082E30E946F
:1072400085B261E083E30E9485B261E084E30E943D
:1072500085B261E085E30E9485B261E085E30E942A
:10726000BEB285E08A8382E58CBD1DBC2AE0F22E89
:107270008FEFE6DEFA94E1F720E030E0A90160E06C
:10728000CE0167DFF82E8B8381E0F81649F00E946B
:10729000A5B0601B710B613D774070F381E046C083
:1072A0002AEA31E040E050E068E0CE0152DF82FFA0
:1072B00002C0FC820CC094E0F92EBBDE8B83FA94F2
:1072C000E1F78A3A11F082E031C082E08C838C8150
:1072D000823031F4C12CD12CE12C80E4F82E03C093
:1072E000C12CD12C760120E030E0A90167E3CE016A
:1072F00030DFA701960169E2CE012BDF8B83882363
:1073000049F00E94A5B0601B710B613D774058F3B6
:107310008AE00CC08C818230B1F420E030E0A90119
:107320006AE3CE0116DF882329F088E08983CE0145
:107330008CDE14C07EDE807C803C11F483E08C8384
:1073400078DE77DE76DECE0180DE86E08B1518F4FF
:1073500088E1898303C0BA8281E001C080E0DF91C7
:10736000CF911F910F91FF90EF90DF90CF90BF9042
:1073700008950F931F93CF93DF93EC0189018C81C4
:10738000833039F039E0440F551F661F771F3A9557
:10739000D1F79A01AB0161E1CE01DBDE811109C0B9
:1073A00040E052E0B801CE01DF91CF911F910F91E3
:1073B00066CE84E08983CE0148DE80E0DF91CF9104
:1073C0001F910F910895CF93DF93EC016EBD20E0E4
:1073D00030E00DB407FEFDCFFA01E20FF31F80810C
:1073E0008EBD0DB407FEFDCF81818EBD2E5F3F4F58
:1073F000211582E0380769F70DB407FEFDCF8FEF46
:107400001FDE8FEF1DDE15DE8B838F71853031F02F
:1074100083E18983CE0119DE80E001C081E0DF9144
:10742000CF9108950F931F93CF93DF93EC018901C0
:107430008C81833039F089E0440F551F661F771F18
:107440008A95D1F79A01AB0168E1CE0182DE8823EB
:1074500011F086E01EC0A8016EEFCE01B4DF8823D4
:10746000C9F068E572E0CE015ADE182F811102C022
:1074700087E10FC020E030E0A9016DE0CE0169DEB8
:10748000811106C0D6DD811103C0CE01DEDD05C04D
:1074900086E18983CE01D9DD10E0812FDF91CF9184
:1074A0001F910F910895CF93DF93EC019C012C5F06
:1074B0003F4F41E050E060E070E0898D9A8D0E947E
:1074C0000F45882399F04D895E896F89788D452B0A
:1074D000462B472B59F44C815D816E817F814D8B0A
:1074E0005E8B6F8B788F998190689983DF91CF91B4
:1074F0000895CF92DF92EF92FF920F931F93CF9355
:10750000DF93EC0189899A89AB89BC89803E9F4FC2
:10751000AF41B10510F080E06AC0CE01C4DF88231E
:10752000D1F30E942343182F8823A9F3E98DFA8D04
:10753000CC80DD80EE80FF8032E0C31AD108E10804
:10754000F108058404C0CC0CDD1CEE1CFF1C0A9461
:10755000D2F786859785A089B189C80ED91EEA1E03
:10756000FB1E81E080932B0AC0922E0CD0922F0C30
:10757000E092300CF092310C80E092E0EEE2FAE022
:10758000DF019C011D9221503040E1F701E0E98DBF
:10759000FA8D8481081788F42EE23AE0B701A6013B
:1075A000400F511D611D711D80912C0A90912D0A73
:1075B00039DF8823E1F00F5FEACFC12C82E0D82EBB
:1075C000E12CF12C058404C0CC0CDD1CEE1CFF1C4E
:1075D0000A94D2F749895A896B897C894C0D5D1DC3
:1075E0006E1D7F1D498B5A8B6B8B7C8B812FDF919E
:1075F000CF911F910F91FF90EF90DF90CF90089562
:10760000CF93DF93EC0141E0611101C040E06C8554
:107610007D858E859F850E946343882341F08889FC
:1076200020E2829FC0011124825D954F02C080E05C
:1076300090E0DF91CF91089530E020E04EE2DC0150
:107640005C91503271F0383029F4FB01E20FF11DEA
:1076500040832F5FFB01E20FF11DDC015C91508341
:107660002F5F3F5F01963B3051F7FB01E20FF11DA9
:1076700010820895CF93DF93EB01FC012381211148
:1076800002C080E00EC02250223020F48FE28883B6
:10769000198206C060E0B4DF009799F3BE01CCDF29
:1076A00081E0DF91CF910895FB012BE030E231932F
:1076B0002150E9F7DC0190E027E03A2FEB2F8D9184
:1076C00081110AC0DA013C931196EC9381E0FB0131
:1076D0009081903239F525C08F32A1F38E3219F0A6
:1076E000E1E3F6E008C02A30E1F098E02AE0E5CFD7
:1076F00031963817B1F034913111FACF291788F04B
:107700003FED380F3E3568F431E0390FFB01E90FEA
:10771000F11D9FE9980F9A3108F480528083932FCE
:10772000CCCF80E008950F931F93CF93DF93EC01AC
:107730008B018B81882311F080E042C0FB01878997
:10774000803139F18032C1F783E08B83F801428DBB
:10775000538D648D758D4D8B5E8B6F8B788F9E01F5
:107760002F5E3F4FC8010E941A44882329F31A8FC5
:10777000098F81E089831C821D821E821F821886E8
:1077800019861A861B861C861D861E861F86188AE9
:1077900017C082E08B831D8A1E8A1F8A188EFB0108
:1077A000408D518D60E070E095E0440F551F661FDD
:1077B000771F9A95D1F7498B5A8B6B8B7C8BD7CFE0
:1077C000DF91CF911F910F9108952F923F924F9289
:1077D0005F926F927F928F929F92AF92BF92CF9261
:1077E000DF92EF92FF920F931F93CF93DF93EC0101
:1077F0005B016A018B81811103C08FEF9FEFC6C0CF
:10780000898180FFFACF49895A896B897C8988856B
:107810009985AA85BB852601612C712C8A019B0163
:10782000081B190B2A0B3B0B401651066206730608
:1078300018F06A01C81AD90A76013E0124E0620EE6
:10784000711CE114F10409F476C0488559856A85F4
:107850007B854A0181E098222B811A012B01E9E006
:107860005694479437942794EA95D1F7898D9A8D49
:10787000FC01223049F4628D738D848D958D620DEB
:10788000731D841D951D3CC014811150122181145B
:107890009104C1F4111116C0452B462B472B49F416
:1078A0008D899E89AF89B88D8C839D83AE83BF837C
:1078B00009C04C815D816E817F8193013CD7882313
:1078C00009F49BCFE98DFA8D6C817D818E819F813A
:1078D0006250710981099109058404C0660F771F00
:1078E000881F991F0A94D2F72685378540895189C8
:1078F000620F731F841F951F610F711D811D911DE4
:1079000020E032E02819390987012E153F0508F4D7
:1079100089010115F2E01F0761F520912E0C3091CD
:107920002F0C4091300C5091310C62177307840773
:10793000950719F41EC0C60129C09501AB01BC0111
:1079400080912C0A90912D0A14DD882309F455CFDB
:10795000A00EB11E88859985AA85BB85800F911FD1
:10796000A11DB11D88879987AA87BB87E01AF10AF4
:1079700068CF40E0A8D6882309F43FCFB401625D08
:10798000754FA801C5010E94EBBEE2CFDF91CF91F8
:107990001F910F91FF90EF90DF90CF90BF90AF902D
:1079A0009F908F907F906F905F904F903F902F901F
:1079B0000895CF93DF931F92CDB7DEB741E050E03B
:1079C000BE016F5F7F4F01DF019719F4898190E05D
:1079D00002C08FEF9FEF0F90DF91CF910895CF926C
:1079E000DF92EF92FF920F931F93CF93DF936C017F
:1079F000EB017A01FC018381823060F00085118502
:107A0000228533850F71112722273327012B022B63
:107A1000032B11F08FEF5CC04115510511F0F701F8
:107A200010821DE040E250E0BE01C601CEDE803291
:107A3000910539F021E0892B09F420E0822F81950E
:107A400047C028812223C1F0253E61F32E3251F335
:107A50003B853F733F3061F4E114F10449F04A8DF6
:107A60005B8D452B29F42F713FEF320F323030F010
:107A70002B8523FDD7CF2CC080E02AC030E02150D9
:107A80003109129FC001139F900D1124F701E80FD7
:107A9000F91F298120832B8121832D8122832F812E
:107AA0002383298524832E852583288926832A8973
:107AB00027832C8920872E892187288D22872C8D4A
:107AC00023872E8D2487288126FFD2CF1586D0CFFD
:107AD000DF91CF911F910F91FF90EF90DF90CF90AA
:107AE00008951F93CF93DF93EC018B81823018F4BC
:107AF00080E090E023C0488559856A857B85A5E0B4
:107B00007695679557954795AA95D1F7142F1F70CD
:107B1000CE014FDF97FDECCF488559856A857B857F
:107B2000415E5F4F6F4F7F4F488759876A877B87DA
:107B300020E2129FC0011124825D954FDF91CF9109
:107B40001F9108954F925F926F927F92AF92BF9272
:107B5000CF92DF92EF92FF920F931F93CF93DF9319
:107B6000EC016A017B012B81222349F089899A89E2
:107B7000AB89BC8984179507A607B70710F480E086
:107B80006BC0223009F463C0C114D104E104F104D4
:107B900049F41C821D821E821F82188619861A864D
:107BA0001B8659C088859985AA85BB85E98DFA8D84
:107BB000E585F0E03996AC01BD01415051096109FC
:107BC00071090E2E04C076956795579547950A94CE
:107BD000D2F797018601015011092109310904C02A
:107BE0003695279517950795EA95D2F70417150747
:107BF0002607370720F0892B8A2B8B2B49F48D8998
:107C00009E89AF89B88D8C839D83AE83BF8304C06A
:107C1000041B150B260B370B280139015E0184E08C
:107C2000A80EB11C411451046104710481F04C810F
:107C30005D816E817F819501898D9A8D7CD591E0E2
:107C4000491A5108610871088111ECCF05C0C88636
:107C5000D986EA86FB8681E0DF91CF911F910F9153
:107C6000FF90EF90DF90CF90BF90AF907F906F909C
:107C70005F904F9008950F931F93CF93DF93EC0184
:107C80008B818823D1F1898187FF32C061E0CE01E9
:107C9000B7DC8C01009789F1FC018081853E69F198
:107CA0008B81823040F449895A896B897C89448F61
:107CB000558F668F778F4D895E896F89788DF80132
:107CC000538F428F758B648BE091250AF091260AC1
:107CD000309759F0B8016A5E7F4FC80148961995F0
:107CE000F801808D918D938B828B89818F77898329
:107CF000DF91CF911F910F91A6C481E0888380E02E
:107D0000DF91CF911F910F910895CF93DF93EC01F5
:107D1000B2DF1B82DF91CF910895FC0123812111F5
:107D2000F4CF08954F925F926F927F92AF92BF927D
:107D3000CF92DF92EF92FF920F931F93CF93DF9337
:107D400000D01F92CDB7DEB75C016A017B01FC0158
:107D500083818130E9F4818181FF1AC0F501818935
:107D60009289A389B48984179507A607B70780F07D
:107D7000892B8A2B8B2B09F472C0F5014084518426
:107D800062847384B701A601C501DCDE811102C0E3
:107D900080E066C0F501818D928DC114D104E104AB
:107DA000F10469F4458956896789708D41D7882324
:107DB00079F3F501158A168A178A108E37C0F501F6
:107DC00044815581668177819E012F5F3F4FB3D4F7
:107DD0008823F1F249815A816B817C81F501818D83
:107DE000928DFC012789203139F4483FFFEF5F076E
:107DF00061057105D8F407C0483F2FEF52076207AD
:107E00002FE0720798F414D7882309F4C1CFF50145
:107E100044815581668177810FEF1FEF2FEF3FE09F
:107E2000818D928D6DD5882309F4B2CFF501C18A79
:107E3000D28AE38AF48A818180688183C5011BDF4D
:107E4000882309F4A5CFB701A6014C145D046E0484
:107E50007F0410F4B301A201C50174DE01C081E00A
:107E60000F900F900F900F90DF91CF911F910F9176
:107E7000FF90EF90DF90CF90BF90AF907F906F908A
:107E80005F904F900895FF920F931F93CF93DF93CE
:107E9000EC01F42E80E2689FF0011124E25DF54FC1
:107EA0008385817121F0842F827109F04EC0809109
:107EB0002E0C90912F0CA091300CB091310C8C872E
:107EC0009D87AE87BF87688B4489558960E070E0E5
:107ED000BA0155274427028D138D20E030E0402B56
:107EE000512B622B732B4D8B5E8B6F8B788F838521
:107EF000887151F4048D158D268D378D098B1A8B61
:107F00002B8B3C8B81E00BC08031F9F49E012F5EFE
:107F10003F4F898D9A8D8ED48823B9F084E08B836E
:107F20008F2D8F7089831C821D821E821F8218866E
:107F300019861A861B86F4FE0BC040E050E0BA0199
:107F4000CE01F0DE811104C011C01B8280E00EC0A2
:107F5000F5FE0BC049895A896B897C89CE01DF9176
:107F6000CF911F910F91FF90EDCD81E0DF91CF91E7
:107F70001F910F91FF900895AF92BF92CF92DF9221
:107F8000EF92FF920F931F93CF93DF937C01EB014E
:107F90006A01B22E898D9A8DF701928F818F40E010
:107FA00050E0BA01CE01CEDDA12C088519852A85C5
:107FB0003B8589899A89AB89BC89081719072A07E3
:107FC0003B07A0F585E036952795179507958A9587
:107FD000D1F70F70CE0185DD009709F481C0FC0157
:107FE0002081222311F0253EB9F4A1100EC040914A
:107FF0002E0C50912F0C6091300C7091310CF701C8
:108000004487558766877787008BFC018081AA2487
:10801000A3948111CACF0AC04BE050E0BC01C60155
:108020000E94DEBE892B09F0C0CF58C08B2D827410
:10803000823409F055C0AA2049F0F701008961E0B7
:10804000C701DEDAEC01009769F44AC08B81823007
:1080500009F446C0CE014DDA882309F441C0CEE2CE
:10806000DAE000E080E2FE0111928A95E9F78BE008
:10807000F601DE0101900D928A95E1F7E091250A63
:10808000F091260A309739F0BE01625F7F4FCE0132
:108090004096199508C081E298E2998B888B80E020
:1080A00098E09F878E87888999899B8B8A8B998F87
:1080B000888F8E859F859F8B8E8BC5D2882381F07C
:1080C0004B2D602FC701DF91CF911F910F91FF9032
:1080D000EF90DF90CF90BF90AF90D5CEB7FEF0CFAE
:1080E00080E0DF91CF911F910F91FF90EF90DF9093
:1080F000CF90BF90AF9008953F924F925F926F9252
:108100007F928F929F92AF92BF92CF92DF92EF9227
:10811000FF920F931F93CF93DF93CDB7DEB7C35476
:10812000D1090FB6F894DEBF0FBECDBF5C016B0165
:1081300024965FAF4EAF2497522E1C8E1F8E19824D
:108140001C826115710511F410E073C0FC0183817C
:108150008111FACF2496EEADFFAD249780818F3246
:1081600011F076011DC02496EEADFFAD24978081FD
:108170008F3231F431962496FFAFEEAF2497F3CFD0
:10818000F60183818250823060F3F601618D728D39
:10819000CE010196C8DA8823B9F2CE0101967C019E
:1081A0008E01045E1F4F3801FE0131964F01402EB3
:1081B000312E19C08823A9F121E0AE01495C5F4F3F
:1081C000B701C801D9DE882309F4BECFEC14FD0441
:1081D00011F0C7019ADD0615170501F1942D832DC5
:1081E0007801092F182FAE014E5B5F4FBE01695C0D
:1081F0007F4F24968EAD9FAD249756DA882309F4DD
:10820000A3CF2496EEADFFAD249780818F3291F6F7
:1082100031962496FFAFEEAF2497F3CF982D892D9A
:10822000DFCF252DAE01495C5F4FB701C501A4DE4C
:10823000182FCE01019671DDCE014C966EDD812F97
:10824000CD5BDF4F0FB6F894DEBF0FBECDBFDF9121
:10825000CF911F910F91FF90EF90DF90CF90BF9043
:10826000AF909F908F907F906F905F904F903F90D6
:108270000895CF93DF93EC0140E050E0BA0152DD66
:10828000882361F061E0CE01BBD9009739F025EE7B
:10829000FC0120831B82DF91CF91D5C180E0DF916B
:1082A000CF9108951F93CF93DF93CDB7DEB76B9730
:1082B0000FB6F894DEBF0FBECDBFAB0119821C8292
:1082C00022E0BC01CE01019617DF182F882321F090
:1082D000CE010196CEDF182FCE0101961EDD812F33
:1082E0006B960FB6F894DEBF0FBECDBFDF91CF9176
:1082F0001F9108952F923F924F925F926F927F92BB
:108300008F929F92AF92BF92CF92DF92EF92FF92A5
:108310000F931F93CF93DF9300D01F921F92CDB77F
:10832000DEB78C015B013A01DC0113968C91139747
:108330008130C1F411968C9181FF14C082FF18C066
:10834000F801418952896389748980859185A28564
:10835000B38584179507A607B70751F0C801F2DB6C
:10836000811106C081E0F80180838FEF9FEF37C154
:10837000630183C0D80159968D919C915A97FC0155
:10838000F481F1501A012B0169E056944794379417
:1083900027946A95D1F7F221FD834A0121E09222C8
:1083A000FF2309F476C080E092E0881999097601EC
:1083B0008C159D0508F47C01D8015996ED91FC912E
:1083C0005A9714962D903D904D905C901797B2E07F
:1083D0002B1A310841085108058404C0220C331CB3
:1083E000441C551C0A94D2F786859785A089B189CB
:1083F000280E391E4A1E5B1EED812E0E311C411CBB
:10840000511CE114F2E0FF0609F089C080912E0CA6
:1084100090912F0CA091300CB091310C82159305E6
:10842000A405B50569F410922B0A8FEF9FEFDC01CC
:1084300080932E0C90932F0CA093300CB093310CA2
:108440009501B201A10180912C0A90912D0A0E9400
:10845000123A882309F486CFF80180859185A28598
:10846000B3858E0D9F1DA11DB11D80879187A287A9
:10847000B387AE0CBF1CCE18DF08D80118964D91FB
:108480005D916D917C911B97C114D10409F072CF5D
:108490007AC08114910409F086CF14964D915D91B4
:1084A0006D917C911797411551056105710559F43E
:1084B00055968D919D910D90BC91A02D0097A10591
:1084C000B10539F520C09E012F5F3F4F34D188237D
:1084D00009F448CF89819A81AB81BC81F801218D53
:1084E000328DF9012789203139F4883FFFEF9F074A
:1084F000A105B10540F40DC0883F2FEF9207A207F8
:108500002FE0B20730F0C8010E94533A81114BCFDF
:1085100029CFF80184839583A683B78344CF811440
:10852000910411F5D80118964D915D916D917C9152
:108530001B9751968D919D910D90BC91A02D481740
:1085400059076A077B0780F07ED0882309F40ACF99
:1085500081E080932B0A20922E0C30922F0C4092B7
:10856000300C5092310C07C041E0C201B101ABD0D8
:10857000882309F4F7CEA701B501C401825D954FA8
:108580000E94EBBE69CF51968D919D910D90BC914B
:10859000A02DF801218184179507A607B70738F4A5
:1085A000418B528B638B748B206821830CC080912C
:1085B000250A9091260A892B31F06114710419F073
:1085C0002068F8012183D80111968C9183FD02C0A7
:1085D000C30105C0C8014FDB8111FACFC3CE0F9094
:1085E0000F900F900F900F90DF91CF911F910F91EF
:1085F000FF90EF90DF90CF90BF90AF909F908F90C3
:108600007F906F905F904F903F902F900895CF9301
:10861000DF931F92CDB7DEB7698341E050E0BE0122
:108620006F5F7F4F049666DE0F90DF91CF910895C4
:10863000FB0101900020E9F7AF0141505109461BB1
:10864000570B049657CECF9380912B0A8823B9F10C
:1086500040912E0C50912F0C6091300C7091310C88
:108660002EE23AE080912C0A90912D0A0E94123A53
:10867000C82F811102C0C0E023C04091270A509149
:10868000280A6091290A70912A0A4115510561054D
:10869000710591F02EE23AE080912C0A90912D0A1A
:1086A0000E94123A882339F31092270A1092280A5E
:1086B0001092290A10922A0A10922B0A01C0C1E0D6
:1086C0008C2FCF910895CF92DF92EF92FF92CF93AC
:1086D0006B017C01C42F80912E0C90912F0CA091E6
:1086E000300CB091310C8C159D05AE05BF05C9F05D
:1086F000AADF811102C080E018C02EE23AE0B70183
:10870000A60180912C0A90912D0A0E94B9398823E4
:1087100091F3C0922E0CD0922F0CE092300CF0927C
:10872000310C81E0C11180932B0ACF91FF90EF9023
:10873000DF90CF9008958F929F92AF92BF92CF9289
:10874000DF92EF92FF920F931F93CF93DF93EC0191
:108750006A017B01890189859A85AB85BC85019673
:10876000A11DB11D84179507A607B70710F480E077
:1087700054C08F89803129F49927872F762F652F50
:108780000BC08032A1F7CB01BA0127E096958795FF
:10879000779567952A95D1F78B889C88AD88BE8898
:1087A000680D791D8A1D9B1D80902E0C90902F0CBA
:1087B000A090300CB090310C681579058A059B05A6
:1087C00081F48F89803191F4DD24EE24FF24F601B9
:1087D000EE0FFF1FE25DF54F80819181A0E0B0E0D8
:1087E00016C040E070DF8111ECCFC1CFE894C7F82C
:1087F000DD24EE24FF24F601EE0FFF1FEE0FFF1F16
:10880000E25DF54F80819181A281B381BF70F80153
:1088100080839183A283B38381E0DF91CF911F9105
:108820000F91FF90EF90DF90CF90BF90AF909F900F
:108830008F9008954F925F926F927F92AF92BF9206
:10884000CF92DF92EF92FF920F931F93CF93DF931C
:1088500000D01F92CDB7DEB78C0149835A836B835A
:108860007C835901C12CD12C7601412C42E0542E3D
:10887000612C712C49815A816B817C819E012F5F13
:108880003F4FC80158DF882341F1D301C201F801ED
:10889000058404C0880F991FAA1FBB1F0A94D2F732
:1088A000C80ED91EEA1EFB1E49815A816B817C814C
:1088B0008789803139F481E0483F5F4F6105710558
:1088C00038F4D8CF81E0483F5F4F6F4F7F4090F240
:1088D000F501C082D182E282F3820F900F900F9057
:1088E0000F90DF91CF911F910F91FF90EF90DF904C
:1088F000CF90BF90AF907F906F905F904F90089512
:108900004F925F926F927F928F929F92AF92BF929F
:10891000CF92DF92EF92FF920F931F93CF93DF934B
:10892000EC014A015B012801390142305105610522
:10893000710508F462C049855A856B857C854F5F57
:108940005F4F6F4F7F4F481559056A057B0508F447
:1089500054C08F89803129F4FF24EB2CDA2CC92CE8
:108960000CC0803209F049C07501640177E0F694CB
:10897000E794D794C7947A95D1F74B895C896D8930
:108980007E89C40ED51EE61EF71E41E0C701B60162
:108990009ADE882391F19F89903159F49924AA2471
:1089A000BB24F401EE0FFF1FE25DF54F51824082C0
:1089B00010C0E89487F89924AA24BB24F401EE0F90
:1089C000FF1FEE0FFF1FE25DF54F40825182628272
:1089D00073829A89923090F04D815E816F817885A3
:1089E0004C0D5D1D6E1D7F1D4093270A5093280A74
:1089F0006093290A70932A0A01C080E0DF91CF9129
:108A00001F910F91FF90EF90DF90CF90BF90AF90AC
:108A10009F908F907F906F905F904F9008952F92CE
:108A20003F924F925F926F927F928F929F92AF92FE
:108A3000BF92CF92DF92EF92FF920F931F93CF934B
:108A4000DF93CDB7DEB72F970FB6F894DEBF0FBE1A
:108A5000CDBF1C014C875D876E877F873B872A8748
:108A6000DC0119960D911D912D913C911C970F5F82
:108A70001F4F2F4F3F4F0D831E832F833887EA856B
:108A8000FB8580809180A280B38081149104A10431
:108A9000B10431F0FFEF8F1A9F0AAF0ABF0A10C06E
:108AA000DC018D909D90AD90BC90B1E0B9870C85B4
:108AB0001D852E853F85013011052105310509F001
:108AC000198675016401412C512C3201F101818517
:108AD0009285A385B485481659066A067B0608F078
:108AE0004EC00D811E812F8138850C151D052E0568
:108AF0003F0550F4F2E0CF2ED12CE12CF12CA2E076
:108B00008A2E912CA12CB12C9E012F5F3F4FB701D3
:108B1000A601C10110DE882391F149815A816B8140
:108B20007C81D701C6010196A11DB11D452B462BA5
:108B3000472B19F04C015D010FC0AC01BD01481974
:108B400059096A097B090C851D852E853F854017CB
:108B500051076207730741F01FEF411A510A610A7A
:108B6000710A6C017D01B2CF0FEF1FEF2FEF3FE0D5
:108B7000B701A601C101C4DE8D83811113C01D821E
:108B80003DC02601370121E0421A510861087108F1
:108B900097018601B301A201C101B2DE882379F3F6
:108BA000730162018C149D04AE04BF0450F3AA85C6
:108BB000BB854D915D916D917C914115510561058C
:108BC0007105A9F4EA85FB8580829182A282B38235
:108BD000F985FF2399F00FEF801A900AA00AB00AD6
:108BE000D1018D929D92AD92BC92139707C09501D1
:108BF0008401C10185DE8111E5CFC1CF8D812F9622
:108C00000FB6F894DEBF0FBECDBFDF91CF911F919D
:108C10000F91FF90EF90DF90CF90BF90AF909F901B
:108C20008F907F906F905F904F903F902F9008951E
:108C3000AF92BF92CF92DF92EF92FF920F931F936A
:108C4000CF93DF9300D01F92CDB7DEB75C016A01EE
:108C50007B0182E090E0A0E0B0E0F50180839183A9
:108C6000A283B3839E012F5F3F4FB701A601C501C9
:108C700062DD811102C080E023C000E010E09801B5
:108C8000B701A601C5013CDE8823A9F3C980DA80BB
:108C9000EB80FC80F5018789803149F481E0F8EFB1
:108CA000CF16FFEFDF06E104F10450F4DBCF81E0E3
:108CB00098EFC9169FEFD906E9069FE0F90690F2F2
:108CC0000F900F900F900F90DF91CF911F910F9108
:108CD000FF90EF90DF90CF90BF90AF9008957F927C
:108CE0008F929F92AF92BF92CF92DF92EF92FF92BC
:108CF0000F931F93CF93DF93EC01142F70932D0AE2
:108D000060932C0A1F8A82E090E0A0E0B0E08883A4
:108D10009983AA83BB8310922B0A1092270A109280
:108D2000280A1092290A10922A0A8FEF9FEFDC017D
:108D300080932E0C90932F0CA093300CB093310C99
:108D4000442349F1453008F0DEC040E060E070E0C7
:108D5000CB01B9DC882309F4D6C020E1129FF001D1
:108D60001124E452F44F80818F7709F0CCC08485C0
:108D70009585A685B78584369105A105B10508F4CA
:108D8000C2C0C084D184E284F384C114D104E1045C
:108D9000F10421F4B8C0C12CD12C760140E0C70108
:108DA000B60191DC782E882309F4ADC08091390A90
:108DB00090913A0A8115924009F0A5C030913E0A7F
:108DC000332309F4A0C080913C0A90913D0A892B7D
:108DD00009F499C020913B0A222309F494C03A8BEC
:108DE0002C831D8630E041E050E06D85062FCA01DE
:108DF000062E02C0880F991F0A94E2F72817390738
:108E000031F081E0860F8D87683078F37CC0209147
:108E1000440A3091450A2115310519F040E050E02F
:108E200008C02091520A3091530A4091540A50913F
:108E3000550A2D833E834F83588780913C0A909139
:108E40003D0A46015701880E991EA11CB11C8B8A50
:108E50009C8AAD8ABE8AE0913F0AF091400AF98F60
:108E6000E88FA0913E0AB0E00E94CABB680D791D50
:108E70008A1D9B1D6A8F7B8F8C8F9D8FB5E0EE0FB7
:108E8000FF1FBA95E1F7E150FE4FEF2FFF27E69560
:108E9000DC01CB018E0F9F1FA11DB11D8E879F8707
:108EA000A88BB98B8090410A9090420A811491045A
:108EB00019F0A12CB12C08C080904E0A90904F0A56
:108EC000A090500AB090510AA7019601281B390BB7
:108ED0004A0B5B0BDA01C901880D991DAA1DBB1D48
:108EE00004C0B695A795979587950A95D2F7898777
:108EF0009A87AB87BC87853F3FE09307A105B10503
:108F000020F48CE08F8B712C15C0853F9F4FA105FD
:108F1000B10510F480E10DC080915A0A90915B0A6E
:108F2000A0915C0AB0915D0A8A8F9B8FAC8FBD8F38
:108F300080E28F8B872DDF91CF911F910F91FF9052
:108F4000EF90DF90CF90BF90AF909F908F907F90E9
:108F50000895FC01148217821382128281ED93E03E
:108F60009183808308950F931F93CF93DF93EC0138
:108F70008F96EFDFCE01805B9F4FEBDFCE018159F3
:108F80009F4FE7DFCE0182579F4FE3DFFE01E3559E
:108F9000FF4F89E1818314823596178ACE01805371
:108FA0009F4FD7DFFE01E151FF4F108211821282E5
:108FB0001382389610821182128213821A821B82C7
:108FC000188219828E010D501F4FF80110821182F4
:108FD00012821382389681E080831EA61DA60E940D
:108FE000A5B068577C4E8F4F9F4FF8016083718307
:108FF00082839383DF91CF911F910F910895FC019C
:1090000020E03EE2DB014C91403241F0283011F487
:1090100030833196DB014C91408331962F5F6F5F37
:109020007F4F2B3079F7108208953F924F925F92D5
:109030006F927F928F929F92AF92BF92CF92DF9268
:10904000EF92FF920F931F93CF93DF93CDB7DEB7CD
:10905000C758D1090FB6F894DEBF0FBECDBF8C0143
:109060006B017A01312C84E0E80EF11C2801E1E16A
:109070004E0E511C5801FCEFAF0EB11C48018EEF93
:10908000880E911C80E4682E712C6C0E7D1EE4E02D
:109090006E0E711CA201BE016F5F7F4FC7010E945F
:1090A000EF3C18160CF02BC12C85322F3871303163
:1090B00009F09EC0F501808191810197029708F423
:1090C00097C0BE016F5F7F4FCE0187589F4F97DFDC
:1090D000A0961FAEA097F6018081811107C065EDB3
:1090E00073E0CE01815A9F4F0E94F4BEB601CE01BB
:1090F000815A9F4F0E94F4BEBE0167587F4FCE0138
:10910000815A9F4F0E94F4BE65ED73E0CE01815AF3
:109110009F4F0E94F4BECE01805C9F4F1ADF21E07A
:10912000AE0147585F4FB701C3010E947C408111D7
:1091300039C0F50180819181892BA1F5ECE8F7E038
:109140008491882341F09091C00095FFFCCF8093DB
:10915000C6003196F5CFE7EDF3E08191882339F031
:109160009091C00095FFFCCF8093C600F6CF809110
:10917000C00085FFFCCF8AE08093C600FE01E7585F
:10918000FF4F8191882339F09091C00095FFFCCF6B
:109190008093C600F6CF8091C00085FFFCCF8AE0A7
:1091A0008093C6008BE1FE01EC5BFF4FDE019596DC
:1091B00001900D928A95E1F724968EAD9FAD24978C
:1091C0009CA38BA381ED93E09AA389A3AE014F5D8D
:1091D0005F4FBE01615A7F4FC80127DFCE018196E4
:1091E0000E94FB37CE01805C9F4F0E94FB3752CF1D
:1091F0008981882309F483C0853E09F44BCF8E32E0
:1092000009F448CF8F3509F445CFF80181898823C7
:1092100031F08E3209F43ECF8F3509F43BCF23FD78
:1092200039CF81E0303109F080E0F80184A7811165
:1092300010C0909102098985923121F48E3409F091
:1092400029CF03C0873409F025CF8A858E3709F4EA
:1092500021CF98012C5F3F4FBE016F5F7F4FC90147
:10926000CA57DF4F2883C658D040C957DF4F3883CD
:10927000C758D040C4DEF50180819181CA57DF4FC5
:109280002881C658D040C957DF4F3881C758D040D1
:109290000097F1F4F6018191882339F09091C00094
:1092A00095FFFCCF8093C600F6CFF901819188230A
:1092B00039F09091C00095FFFCCF8093C600F6CFA7
:1092C0008091C00085FFFCCF8AE08093C600E2CE8B
:1092D0008130910539F4F401808191810196918367
:1092E0008083D8CE029709F0D5CE232D30E0F4014B
:1092F000808191812817390711F03394CBCEC9575B
:10930000DF4F0FB6F894DEBF0FBECDBFDF91CF9118
:109310001F910F91FF90EF90DF90CF90BF90AF9093
:109320009F908F907F906F905F904F903F900895A7
:10933000EF92FF920F931F93CF93DF93CDB7DEB7DA
:109340006F970FB6F894DEBF0FBECDBF8C01FC0146
:10935000E450FF4F118210827C0183E3E80EF11C80
:1093600040E050E0BA01C7010E94A23D8BE1F70145
:10937000DE01159601900D928A95E1F7F80181A919
:1093800092A99C838B8381ED93E09A838983AE01BC
:109390004F5F5F4F6DEB74E0C80147DECE01019671
:1093A0000E94FB376F960FB6F894DEBF0FBECDBF9D
:1093B000DF91CF911F910F91FF90EF9008952BE1D6
:1093C000FB013496DC01149601900D922A95E1F789
:1093D000FB0122813381FC01338322830895EF92C4
:1093E000FF920F931F93CF93DF93EC011B828EA903
:1093F000882321F0CE01C3960E94853E7E018DEA2E
:10940000E80EF11C45E360E0C7010E9406398111B6
:109410001FC0ECE8F7E08491882341F09091C000F0
:1094200095FFFCCF8093C6003196F5CFEFE7F7E0CC
:109430008491882341F09091C00095FFFCCF8093E8
:10944000C6003196F5CF8091C00085FFFCCF74C077
:109450008E010E541F4F41E0B701C80140DC81115D
:1094600025C040E0B701C8013ADC81111FC0E2E924
:10947000F7E08491882341F09091C00095FFFCCFE4
:109480008093C6003196F5CFECE6F7E0849188230F
:1094900041F09091C00095FFFCCF8093C6003196BB
:1094A000F5CF8091C00085FFFCCF46C0B801CE014A
:1094B000C3960E94933B81111FC0E2E9F7E08491BB
:1094C000882341F09091C00095FFFCCF8093C600A7
:1094D0003196F5CFECE5F7E08491882341F0909147
:1094E000C00095FFFCCF8093C6003196F5CF8091E8
:1094F000C00085FFFCCF20C081E08B83ECE8F7E063
:109500008491882341F09091C00095FFFCCF809317
:10951000C6003196F5CFE1E5F7E08491882341F06C
:109520009091C00095FFFCCF8093C6003196F5CF97
:109530008091C00085FFFCCF8AE08093C6008E0139
:10954000015D1F4FB801CE01805B9F4F38DFC25BCA
:10955000DF4F19830883DF91CF911F910F91FF9007
:10956000EF900895FC01128213820895FC0123817B
:10957000222311F021E022830895FC012281211190
:10958000128208952F923F924F925F926F927F9234
:109590008F929F92AF92BF92CF92DF92EF92FF9203
:1095A0000F931F93CF93DF93CDB7DEB7AD970FB671
:1095B000F894DEBF0FBECDBF7C016B014DA7FC014F
:1095C0008381882309F4A8C14701F4ED8F0E911C13
:1095D000C4010E94853EF7011282CE0101965C0112
:1095E000B8DC17019EE4290E311CC7018F96F101EA
:1095F00091838083F60180818F3209F07FC06FE212
:1096000070E0C6010E94FFBE8C010F5F1F4F09F47E
:109610007BC06FE270E0C8010E94FFBE2C01009782
:1096200009F473C00817190708F06FC03C01601AED
:10963000710AA301B801CE0180960E941FBFE0E22B
:10964000F0E0EC0FFD1FE60DF71D1082FE01B09655
:109650008191882339F09091C00095FFFCCF8093D1
:10966000C600F6CF8091C00085FFFCCFFAE0F093F2
:10967000C600F101608171816115710519F06C5F9F
:109680007F4F02C060E070E021E0AE01405E5F4FBE
:10969000CE0105960E947C4081112BC0EDE3F7E0DE
:1096A0008491882341F09091C00095FFFCCF809376
:1096B000C6003196F5CFFE01B0968191882339F02E
:1096C0009091C00095FFFCCF8093C600F6CFEBE3EE
:1096D000F7E08491882341F09091C00095FFFCCF82
:1096E0008093C6003196F5CF8091C00085FFFCCFF6
:1096F000E7C0F101B182A082820187CFC701805B00
:109700009F4FF101918380838601FDA5FF2309F41A
:109710009CC0F101608171816115710519F06C5F68
:109720007F4F02C060E070E021E0A801C4010E9408
:109730007C40882309F45FC0F40181899289A38960
:10974000B489F701E151FF4F80839183A283B383F2
:10975000EDE2F7E08491D701A151BF4F882349F092
:109760009091C00095FFFCCF8093C6003196849104
:10977000F5CFF8018191882339F09091C00095FFD1
:10978000FCCF8093C600F6CFE5E2F7E08491882312
:1097900041F09091C00095FFFCCF8093C6003196B8
:1097A000F5CF4D915D916D917C912AE030E082E79B
:1097B00095E00E94EB168091C00085FFFCCF8AE007
:1097C0008093C600F701E950FF4F10821182128288
:1097D0001382E7E1F7E08491882341F09091C00083
:1097E00095FFFCCF8093C6003196F5CF8091C000E5
:1097F00085FFFCCF88C0E3E0F7E08491882341F047
:109800009091C00095FFFCCF8093C6003196F5CFB4
:10981000F8018191882339F09091C00095FFFCCF29
:109820008093C600F6CFE1E0F7E08491882341F011
:109830009091C00095FFFCCF8093C6003196F5CF84
:109840008091C00085FFFCCF3BC0F1016081718138
:109850006115710519F06C5F7F4F02C060E070E028
:1098600026E5A801C4010E947C4081112DC0EDEEC7
:10987000F6E08491882341F09091C00095FFFCCFE1
:109880008093C6003196F5CFF8018191882339F095
:109890009091C00095FFFCCF8093C600F6CFEBEE11
:1098A000F6E08491882341F09091C00095FFFCCFB1
:1098B0008093C6003196F5CF8091C00085FFFCCF24
:1098C0008AE08093C60025C081E0F7018083E9ED3E
:1098D000F6E08491882341F09091C00095FFFCCF81
:1098E0008093C6003196F5CFF6018191882339F037
:1098F0009091C00095FFFCCF8093C600F6CF809179
:10990000C00085FFFCCF8AE08093C600C8010E949A
:10991000FE86C5010E94FB37AD960FB6F894DEBFF8
:109920000FBECDBFDF91CF911F910F91FF90EF90B0
:10993000DF90CF90BF90AF909F908F907F906F906F
:109940005F904F903F902F90089521E0FC0121837C
:1099500040E018CE3F924F925F926F927F928F922B
:109960009F92AF92BF92CF92DF92EF92FF920F93AE
:109970001F93CF93DF93CDB7DEB7AC970FB6F894B4
:10998000DEBF0FBECDBF7C015B01FC01838188235C
:1099900009F401C1C7018C529F4F0E94853EF70117
:1099A0001282CE0101966C01D4DA27019EE4490EA1
:1099B000511CC7018F96F20191838083F50180814C
:1099C0008F3209F084C06FE270E0C5010E94FFBED3
:1099D0008C010F5F1F4F9AE0392E0115110509F414
:1099E0007CC06FE270E0C8010E94FFBE4C0100978E
:1099F00009F474C00817190708F070C03C01601A18
:109A0000710AA301B801CE0180960E941FBFE0E257
:109A1000F0E0EC0FFD1FE60DF71D1082FE01B09681
:109A20008191882339F09091C00095FFFCCF8093FD
:109A3000C600F6CF8091C00085FFFCCF3092C600F3
:109A4000F201608171816115710519F06C5F7F4FC2
:109A500002C060E070E021E0AE01405E5F4FCE01E9
:109A600005960E947C4081112BC0E5ECF6E08491C4
:109A7000882341F09091C00095FFFCCF8093C600F1
:109A80003196F5CFFE01B0968191882339F09091FF
:109A9000C00095FFFCCF8093C600F6CFE3ECF6E064
:109AA0008491882341F09091C00095FFFCCF809372
:109AB000C6003196F5CF8091C00085FFFCCF65C010
:109AC000F201D182C08284010F5F1F4F86CFC70190
:109AD000805B9F4FF201918380838501F201808139
:109AE0009181009711F0049602C080E090E0B801E7
:109AF0000E945241882301F1E5EBF6E0849188232E
:109B000041F09091C00095FFFCCF8093C600319644
:109B1000F5CFF8018191882339F09091C00095FF2D
:109B2000FCCF8093C600F6CFF701E950FF4F1082BB
:109B30001182128213822CC0EDE9F6E08491882311
:109B400041F09091C00095FFFCCF8093C600319604
:109B5000F5CFF8018191882339F09091C00095FFED
:109B6000FCCF8093C600F6CFEBE9F6E08491882322
:109B700041F09091C00095FFFCCF8093C6003196D4
:109B8000F5CF8091C00085FFFCCF8AE08093C600AE
:109B9000C6010E94FB37AC960FB6F894DEBF0FBE2D
:109BA000CDBFDF91CF911F910F91FF90EF90DF908C
:109BB000CF90BF90AF909F908F907F906F905F906D
:109BC0004F903F900895CF93DF93EC018B818823D2
:109BD000C1F1E9E8F6E08491882341F09091C0005A
:109BE00095FFFCCF8093C6003196F5CFFE01E9507A
:109BF000FF4F40815181628173812AE030E082E72A
:109C000095E00E94EB16E7E8F6E08491882341F0A6
:109C10009091C00095FFFCCF8093C6003196F5CFA0
:109C2000C151DF4F488159816A817B812AE030E050
:109C300082E795E00E94EB168091C00085FFFCCF83
:109C400011C0E7E7F6E08491882341F09091C000CD
:109C500095FFFCCF8093C6003196F5CF8091C00070
:109C600085FFFCCF8AE08093C600DF91CF910895F5
:109C7000AF92BF92CF92DF92EF92FF920F931F931A
:109C8000CF93DF935C01EB01FB0101900020E9F72A
:109C90008F0101501109061B170B6C01F4EDCF0E5B
:109CA000D11CF60110826EE470E0CE010E94FFBE6E
:109CB0007C01009729F4F8013197EC0FFD1F0DC0CE
:109CC00060E270E00E94FFBEEC0121966AE270E063
:109CD000C7010E94FFBEFC0131978DE081838AE0BD
:109CE00082831382BE01C50180539F4F0E94184397
:109CF000F6018081882309F1E2E9F7E08491882365
:109D000041F09091C00095FFFCCF8093C600319642
:109D1000F5CFE1E6F6E08491882341F09091C00010
:109D200095FFFCCF8093C6003196F5CF8091C0009F
:109D300085FFFCCF8AE08093C600DF91CF911F9111
:109D40000F91FF90EF90DF90CF90BF90AF9008956C
:109D50002F923F924F925F926F927F928F929F923B
:109D6000AF92BF92CF92DF92EF92FF920F931F9329
:109D7000CF93DF93CDB7DEB7CC55D1090FB6F894AA
:109D8000DEBF0FBECDBF8C0185509F4F5C016623A7
:109D900039F0F5011082F801838181111DC015C0D1
:109DA000FC018081882309F4ADC0F801ED50FF4F1C
:109DB000C080D180E280F3800E94A5B0C616D7068D
:109DC000E806F90608F49EC0E4CFC80108DBF801F4
:109DD0008381882309F496C0F80186A58F9385A511
:109DE0008F9388E596E09F938F937E01FFE3EF0EBC
:109DF000F11CFF92EF920E94A6BF0F900F900F9060
:109E00000F900F900F90B12CF70101900020E9F70F
:109E10003197EE19FF09BE1684F46701CB0CD11CF3
:109E2000B7FCDA94F6018081992787FD90950E940E
:109E30008EBEF6018083B394E7CF4801F3E38F0E23
:109E4000911C40E050E0BA01C4010E94A23D512C97
:109E5000CE0101966C0121E5622E26E0722E5E0194
:109E600091E2A90EB11C40E050E0B601C4010E948D
:109E7000EF3C1816DCF5412CF60101900020E9F7C3
:109E80003197EC19FD094E1674F41601240C311C9F
:109E900047FC3A94F101808190E00E948EBEF1016E
:109EA00080834394E9CF8A858E37E9F245E050E01C
:109EB000B701C6010E9411BF892BA9F6FF92EF924C
:109EC0007F926F92BF92AF920E94A6BFC5010E947F
:109ED00050198DE496E00E94C3190F900F900F90D7
:109EE0000F900F900F9055245394BDCF511004C084
:109EF0008FEF9FEFF80104C0F80185A596A50196A4
:109F000096A785A7C45ADF4F0FB6F894DEBF0FBEE1
:109F1000CDBFDF91CF911F910F91FF90EF90DF9018
:109F2000CF90BF90AF909F908F907F906F905F90F9
:109F30004F903F902F9008950F931F93CF93DF93EF
:109F4000EC018C010C521F4FC8010E943B3EC8011E
:109F50000E94853E18821982DF91CF911F910F9147
:109F60000895EF92FF920F931F93CF93DF93CDB796
:109F7000DEB76F970FB6F894DEBF0FBECDBF8C0172
:109F80007C018EE4E80EF11CC801805B9F4FF70155
:109F900091838083E255FF4F22E030E031832083BC
:109FA000329670E07183608340E050E0BA0104961D
:109FB0000E94A23DF701808191812BE1FC01349642
:109FC000DE01159601900D922A95E1F7FC01828140
:109FD00093819C838B8381ED93E09A838983AE0187
:109FE0004F5F5F4F6DEB74E0C8011FD8CE01019643
:109FF0000E94FB376F960FB6F894DEBF0FBECDBF41
:10A00000DF91CF911F910F91FF90EF900895CF9224
:10A01000DF92EF92FF920F931F93CF93DF93CDB711
:10A02000DEB76F970FB6F894DEBF0FBECDBF8C01C1
:10A030006C012EE4C20ED11C805B9F4FF601918310
:10A040008083E255FF4F21E030E0318320837801A7
:10A05000FEEFEF0EF11CF7011182108240E050E09C
:10A06000BA0104960E94A23DF601808191812BE104
:10A07000FC013496DE01159601900D922A95E1F7C8
:10A08000FC01828193819C838B8381ED93E09A8391
:10A090008983AE014F5F5F4F6DEB74E0C8010E9492
:10A0A0001548CE0101960E94FB37F701808191810E
:10A0B0006F960FB6F894DEBF0FBECDBFDF91CF9184
:10A0C0001F910F91FF90EF90DF90CF900895CF9365
:10A0D000DF93EC010E94C86B0E943E6CCE018C5253
:10A0E0009F4F0E94853E1A8281E496E00E94C31928
:10A0F000809108118823F9F010920811C091AB08E3
:10A10000D0E0CC0FDD1FCC5ADD4E688179818827E5
:10A1100077FD8095982F0E9457B820914702309183
:10A1200048024091490250914A020E94B8B918165B
:10A1300014F419821882DF91CF9108952F923F92E3
:10A140004F925F926F927F928F929F92AF92BF9247
:10A15000CF92DF92EF92FF920F931F93CF93DF93F3
:10A16000CDB7DEB7C454D1090FB6F894DEBF0FBE29
:10A17000CDBF3C011B014A012FA309A7EBA62196E5
:10A18000ACAEBDAECEAEDFAE219734E0239F200152
:10A190001124440D551D5AAB49ABDA01CD90DD9029
:10A1A000ED90FC90FC01E40DF51D20813181428190
:10A1B0005381C701B6010E94DCB66BAB7CAB8DABA3
:10A1C0009EABB4E00B9F80011124F401E00FF11F5E
:10A1D000F8AFEFAB80809180A280B380F301E00FF5
:10A1E000F11F2081318142815381C501B4010E9458
:10A1F000DCB669AF7AAF8BAF9CAF2BA5F4E02F9F95
:10A20000C0011124F301E80FF91F2081318142813F
:10A210005381298F3A8F4B8F5C8FF101E80FF91F23
:10A2200060817181828193810E94DBB66F8F78A3F8
:10A2300089A39AA3D1011C968D919D910D90BC91FB
:10A24000A02D8DA79EA7AFA7B8ABD3011C962D91CB
:10A250003D914D915C911F972BA33CA34DA35EA311
:10A26000A701960150582D8B3E8B4F8B588FD501EF
:10A27000C401B058898B9A8BAB8BBC8BF101E40D78
:10A28000F51D2BA93CA94DA95EA960817181828130
:10A2900093810E94DBB66B017C01F101E00FF11F9D
:10A2A00029AD3AAD4BAD5CAD608171818281938106
:10A2B0000E94DBB64B015C01A70196016D897E8986
:10A2C0008F89988D0E948ABA2B013C01A5019401C7
:10A2D00069897A898B899C890E948ABA9B01AC0121
:10A2E000C301B2010E94DCB62B013C01A50194011F
:10A2F0006D897E898F89988D0E948ABA4B015C0195
:10A30000A701960169897A898B899C890E948ABAFA
:10A310009B01AC01C501B4010E94DBB6A30192010F
:10A320000E944FB76B017C0120E030E0A9010E9440
:10A33000B5B787FF0AC02BED3FE049EC50E4C701F9
:10A34000B6010E94DCB66B017C016F968FAD6F97F2
:10A35000882351F02BED3FE049EC50E4C701B601F2
:10A360000E94DBB66B017C016E962CAD3DAD4EAD0F
:10A370005FAD6E97C701B6010E948ABA2F8D38A1D2
:10A3800049A15AA15F770E94C5B94B015C012FE634
:10A3900032E143E85AE30E94B5B787FDC4C1C50165
:10A3A000B4010E9492B80E9429B87E8F6D8FDB01A4
:10A3B000AB2B21F4E1E0F0E0FE8FED8F2D8D3E8D93
:10A3C000B90180E090E00E9455B84B015C019B010F
:10A3D000AC01C701B6010E94BCB72B013C01A5012D
:10A3E00094016F8D78A189A19AA10E94BCB725968E
:10A3F0006CAF7DAF8EAF9FAF25972BA13CA14DA138
:10A400005EA16DA57EA58FA598A90E94DBB6A501CA
:10A4100094010E94BCB76DA77EA78FA798AB20E0E0
:10A4200030E040E05FE3C301B2010E948ABAA301B9
:10A4300092010E948ABA9B01AC0160E070E080E862
:10A440009FE30E94DBB66F8F78A389A39AA3CE0106
:10A450000196FC014BA534E0439FE00DF11D112452
:10A46000298D3A8D4B8D5C8D2083318342835383BC
:10A470002BA13CA14DA15EA12D873E874F87588B14
:10A48000B12C41E050E05A8F498F81E090E08C0F71
:10A490009D1FBFA1A4E0BA9F800D911D11249CA710
:10A4A0008BA721E030E02C0F3D1F59A544E0549FBD
:10A4B000200D311D11243AA729A7F8A7EFA3498D34
:10A4C0005A8D8D8D9E8D4817590708F017C188E168
:10A4D0008B150CF444C02F8D38A149A15AA169896C
:10A4E0007A898B899C890E948ABA6B017C01A301BD
:10A4F00092016D897E898F89988D0E948ABAA70101
:10A5000096010E94DCB6A62E172F982E892E2F8D2D
:10A5100038A149A15AA16D897E898F89988D0E94A1
:10A520008ABA6B017C01A301920169897A898B89BE
:10A530009C890E948ABA9B01AC01C701B6010E94A6
:10A54000DBB66D8B7E8B8F8B988FB3948A2D912F7A
:10A55000A92DB82D898B9A8BAB8BBC8B6AC0A98D2A
:10A56000BA8DBD0180E090E00E9455B8A301920130
:10A570000E948ABA6B017C010E94B9B7698B7A8B01
:10A580008B8B9C8BC701B6010E94EDBA4B015C011D
:10A59000E9A9FAA9C080D180E280F380F7FAF094AB
:10A5A000F7F8F094AFA9B8AD2D913D914D915C9124
:10A5B0002BA33CA34DA35EA329893A894B895C89CF
:10A5C000C701B6010E948ABA6D8B7E8B8F8B988FE4
:10A5D000A50194016BA17CA18DA19EA10E948ABAC4
:10A5E0009B01AC016D897E898F89988D0E94DCB6B4
:10A5F0006D8B7E8B8F8B988FA5019401C701B6015F
:10A600000E948ABA6B017C0129893A894B895C894D
:10A610006BA17CA18DA19EA10E948ABA9B01AC0175
:10A62000C701B6010E94DBB6698B7A8B8B8B9C8B42
:10A63000B12C2D893E894F89588D6BA97CA98DA994
:10A640009EA90E94DCB6EBA5FCA560837183828382
:10A65000938329893A894B895C8969AD7AAD8BAD41
:10A660009CAD0E94DCB6A9A5BAA56D937D938D9390
:10A670009C93139725962CAD3DAD4EAD5FAD2597C0
:10A68000EFA1F8A560817181828193810E94DCB67F
:10A69000AFA1B8A56D937D938D939C9313972DA532
:10A6A0003EA54FA558A96D857E858F8598890E9406
:10A6B000DCB66D877E878F87988BCE0101960E94CE
:10A6C000EB20FE01E15AFF4F6F012196ECACFDAC8F
:10A6D0000EAD1FAD21979E01235F3F4FAE01475F37
:10A6E0005F4FBE016B5F7F4FCE01019656D5298D1E
:10A6F0003A8D2F5F3F4F3A8F298FE1CE9101245F32
:10A700003F4FA101485F5F4FB1016C5F7F4FDE019A
:10A71000A15ABF4F6D012196ECACFDAC0EAD1FAD43
:10A720002197C1013AD5CC5BDF4F0FB6F894DEBF5D
:10A730000FBECDBFDF91CF911F910F91FF90EF9092
:10A74000DF90CF90BF90AF909F908F907F906F9051
:10A750005F904F903F902F9008952F923F924F928D
:10A760005F926F927F928F929F92AF92BF92CF92A1
:10A77000DF92EF92FF920F931F93CF93DF93CDB7AA
:10A78000DEB768970FB6F894DEBF0FBECDBF1C01D1
:10A790002A013B0148015901DC01D8966D917D9158
:10A7A0008D919C91DB970E9455B86B017C01A301B0
:10A7B00092010E948ABA0E94A2B70E9429B86D87AE
:10A7C0007E878F87988BA5019401C701B6010E94EF
:10A7D0008ABA0E94A2B70E9429B8698B7A8B8B8BA8
:10A7E0009C8B2D853E854F8558892837310541053D
:10A7F000510540F488E790E0A0E0B0E08D879E87A7
:10A80000AF87B88B29893A894B895C89283731050C
:10A810004105510540F488E790E0A0E0B0E0898B65
:10A820009A8BAB8BBC8B91012C5B3F4FD9018D91E7
:10A830009D910D90BC91A02D8D839E83AF83B88791
:10A84000BC01CD010E9457B869837A838B839C83B6
:10A85000F10164AD75AD86AD97AD0E9455B86987BD
:10A860007A878B879C8720E030E0A90169817A8113
:10A870008B819C810E94B5B7882339F1A70196018D
:10A88000C701B6010E948ABA4B015C0129853A854D
:10A890004B855C85CA01B9010E948ABA9B01AC0153
:10A8A000C501B4010E94DBB64B015C0129813A81EC
:10A8B0004B815C81CA01B9010E94DCB69B01AC01ED
:10A8C000C501B4010E94BCB703C060E070E0CB01D9
:10A8D0000E94A2B70E9424B82B013C016D817E81A9
:10A8E0008F81988590958095709561957F4F8F4F5A
:10A8F0009F4F0E9457B84B015C01F101E05CFF4F94
:10A9000060817181828193810E9455B86D837E83BD
:10A910008F83988720E030E0A901C501B4010E942F
:10A92000B5B7882349F12D813E814F815885CA01F1
:10A93000B9010E948ABA6D8B7E8B8F8B988FA7018D
:10A940009601C701B6010E948ABA9B01AC016D89CC
:10A950007E898F89988D0E94DBB66B017C01A501F1
:10A960009401C501B4010E94DCB69B01AC01C70192
:10A97000B6010E94BCB703C060E070E0CB010E944A
:10A9800092B8D10150968D909D90AD90BC90539708
:10A9900075016401C418D508E608F7080E9424B8B8
:10A9A000C61AD70AE80AF90AF7FE6BC020E030E0C1
:10A9B000A90169817A818B819C810E94B5B7882326
:10A9C00009F447C029813A814B815C81CA01B901F0
:10A9D0000E94DCB66B017C01C501B4010E9455B830
:10A9E0009B01AC01C701B6010E948ABA6B017C01D0
:10A9F00029853A854B855C85CA01B9010E948ABACE
:10AA00009B01AC01C701B6010E94DBB66B017C0162
:10AA10002D813E814F815885CA01B9010E948ABAB1
:10AA20009B01AC01C701B6010E94DCB66B017C0141
:10AA300020E030E040E850E469817A818B819C819C
:10AA40000E948ABA9B01AC01C701B6010E94BCB743
:10AA500003C060E070E0CB010E94A2B70E9424B85E
:10AA60002B013C0197FF03C0412C512C32014814AB
:10AA700059046A047B0410F024013501C12CD12C47
:10AA800076018FB7F894F101E45BFF4F908191114B
:10AA900021C0F101448A558A668A778AC40CD51C84
:10AAA000E61CF71CD101C08ED18EE28EF38E2D856F
:10AAB0003E854F85588924AF35AF46AF57AFA05C70
:10AAC000BF4F29893A894B895C892D933D934D93DA
:10AAD0005C9313978FBF68960FB6F894DEBF0FBED6
:10AAE000CDBFDF91CF911F910F91FF90EF90DF903D
:10AAF000CF90BF90AF909F908F907F906F905F901E
:10AB00004F903F902F9008954F925F926F927F9257
:10AB1000AF92BF92CF92DF92EF92FF920F931F936B
:10AB2000CF93DF93EB017A01209709F458C04115C8
:10AB3000510509F454C0AAA4BBA40CA51DA59501F8
:10AB4000A8016EA17FA188A599A50E94B5B7882309
:10AB500009F445C08FA981113AC0F70146A057A05A
:10AB600060A471A4A3019201B501C8010E94B8B903
:10AB700018166CF5A3019201C301B2010E948ABAB2
:10AB80006B017C018AA99BA9ACA9BDA9BC01CD011F
:10AB900090589B01AC010E94DCB62EA53FA548A9A8
:10ABA00059A90E948ABA9B01AC01C701B6010E9453
:10ABB000DBB60E94F7BA6B017C019B01AC01B501C9
:10ABC000C8010E94B5B787FD02C056018701A501E3
:10ABD000B8014EA35FA368A779A781E08EABDF9190
:10ABE000CF911F910F91FF90EF90DF90CF90BF908A
:10ABF000AF907F906F905F904F900895DF92EF92AB
:10AC0000FF920F931F93CF93DF938091370C8FB7F1
:10AC1000F894E090360C8FBF8091370C90E08E193D
:10AC200091098F7099270497F4F01091370C135005
:10AC30001F7040E050E000E0F12C8DE4D82E1E158E
:10AC400091F0111101C010E11150D19EE0011124C9
:10AC5000C85CD34F602F7F2DCE0156DF402F5F2D74
:10AC60000C2FFD2EECCFDF91CF911F910F91FF9014
:10AC7000EF90DF9008954F925F926F927F92AF9224
:10AC8000BF92CF92DF92EF92FF920F931F93CF93D9
:10AC9000DF938C01EB01009709F453C0FC0187A9F5
:10ACA00081114FC046A057A060A471A4AEA0BFA060
:10ACB000C8A4D9A49501A601C301B2010E94B5B7E9
:10ACC00087FF3FC0A3019201C301B2010E948ABA6B
:10ACD0002B013C01F80182A993A9A4A9B5A9BC0143
:10ACE000CD0190589B01AC010E94DCB6F80126A56D
:10ACF00037A540A951A90E948ABA9B01AC01C301A2
:10AD0000B2010E94DBB60E94F7BA7B018C019B0165
:10AD1000AC01B501C6010E94B5B787FF02C075013D
:10AD200086019701A801B501C6010E94B5B7882325
:10AD300041F0A701B8014EA35FA368A779A781E0FE
:10AD40008EABDF91CF911F910F91FF90EF90DF902D
:10AD5000CF90BF90AF907F906F905F904F9008958D
:10AD6000EF92FF920F931F93CF93DF93F090360CE7
:10AD700000E010E080E090E02DE4E22E2091370C1E
:10AD8000F21689F0EF9CE0011124C85CD34FAE01AC
:10AD9000B80171DF81E08F0D803109F480E0F82E79
:10ADA000C8018E01EBCF40E050E0B801DF91CF91B8
:10ADB0001F910F91FF90EF905ECF4F925F926F9235
:10ADC0007F928F929F92AF92BF92CF92DF92EF923B
:10ADD000FF920F931F93CF93DF939090360CC0E0B8
:10ADE000D0E03DE4832E892D992787FD9095209111
:10ADF000370C30E082179307B9F1889E5001899E85
:10AE0000B00C1124C501885C934F5C01209729F197
:10AE10008EA9811104C0F50186A98823F1F0CAA08A
:10AE2000DBA0ECA0FDA0A7019601F50166A177A12A
:10AE300080A591A50E94BCB72B013C01A7019601FA
:10AE40006EA17FA188A599A50E94BCB7AB01BC01EA
:10AE500093018201CE0181DC1EAA9394F0E19F123E
:10AE600001C0912CE501BFCF2097E9F0CAA0DBA07B
:10AE7000ECA0FDA0A70196016DEC7CEC8CE49DE3B9
:10AE80000E94BCB74B015C01A70196016EA17FA196
:10AE900088A599A50E94BCB7AB01BC0195018401AE
:10AEA000CE015BDC1EAADF91CF911F910F91FF9025
:10AEB000EF90DF90CF90BF90AF909F908F907F905A
:10AEC0006F905F904F90089599DE4ADF76CF109291
:10AED000370C1092360C80E1EDE1F1E1DF011D92BB
:10AEE0008A95E9F710920D1110920E1110920F1120
:10AEF0001092101110921111109212111092131140
:10AF0000109214111092151110921611109217111F
:10AF1000109218111092191110921A1110921B11FF
:10AF200010921C111092091110920A1110920B111B
:10AF300010920C1108954F925F926F927F928F92B0
:10AF40009F92AF92BF92CF92DF92EF92FF920F93B8
:10AF50001F93CF93DF9380910811882309F4EFC0EA
:10AF6000C0904702D0904802E0904902F0904A0217
:10AF70006091541270915512882777FD8095982F13
:10AF80000E9457B820E030E040E050E40E94DCB678
:10AF90009601A7010E94B5B787FDD1C05090360C2D
:10AFA000612C712C00E010E04DE4442E8091370CB0
:10AFB000581609F453C0852D90E0489EF001499E33
:10AFC000F00D1124E85CF34F40815181628173815F
:10AFD000452B462B472B81F444815581668177812F
:10AFE000452B462B472B41F440855185628573855F
:10AFF000452B462B472B69F1489EE001499ED00D19
:10B000001124C85CD34F6C857D858E859F850E94F9
:10B0100057B84B015C01688979898A899B890E94AC
:10B0200055B89B01AC01C501B4010E94BCB72AA16F
:10B030003BA14CA15DA10E948ABA5B01D82FC92F08
:10B040009301A8010E94B8B918161CF435010D2F00
:10B050001C2F5394852D8F70582EA8CF209143021A
:10B06000309144024091450250914602B301C8011B
:10B070000E948ABA9B01AC01B601C7010E94DCB6EE
:10B080008B01D82FC92F9601A7010E94B5B787FD64
:10B0900003C06801ED2EFC2E00914B0210914C0272
:10B0A000D0914D02C0914E0298014D2F5C2FB601F8
:10B0B000C7010E94B8B918161CF08601DE2DCF2DED
:10B0C0008090320C9090330CA090340CB090350CE2
:10B0D00098014D2F5C2FC501B4010E94B8B9181614
:10B0E000D4F420E037ED43EA5CE3B8018D2F9C2FC8
:10B0F0000E948ABA6B017C0128E431EE4AE75FE3E3
:10B10000C501B4010E948ABAA70196010E94DCB66B
:10B110008B01D82FC92FC801AD2FBC2F8093320CC3
:10B120009093330CA093340CB093350CB8018D2F51
:10B130009C2F0E9424B87093551260935412DF9193
:10B14000CF911F910F91FF90EF90DF90CF90BF9024
:10B15000AF909F908F907F906F905F904F900895E9
:10B160006091A9089091360C8091370C981781F066
:10B170008091360C9DE4899FF0011124E058F34F33
:10B1800060819091370C891719F08F5F8F70F9CF1C
:10B1900070E089E00E946DB1CECE2F923F924F9227
:10B1A0005F926F927F928F929F92AF92BF92CF9257
:10B1B000DF92EF92FF920F931F93CF93DF93CDB760
:10B1C000DEB7C357D1090FB6F894DEBF0FBECDBFAF
:10B1D0002C015B014A013901ECAAFBAAD9AEC8AE29
:10B1E0002091370C2F5F29962FAF2997203119F422
:10B1F00029961FAE299729963FAD2997E32EFF2464
:10B20000E7FCF0948091360C90E08E159F0539F4A0
:10B210000E94046E0E9485230E945088F3CF2091E3
:10B220006D1130916E1140916F1150917011D201DA
:10B230006D917D918D919C910E948ABA0E945ABA1B
:10B240006D966CAF7DAF8EAF9FAF6D9720917111F2
:10B25000309172114091731150917411F501608118
:10B260007181828193810E948ABA0E945ABAA19602
:10B270006CAF7DAF8EAF9FAFA197209175113091CC
:10B2800076114091771150917811D4016D917D9193
:10B290008D919C910E948ABA0E945ABAA5966CAF71
:10B2A0007DAF8EAF9FAFA5972091791130917A1124
:10B2B00040917B1150917C11F301608171818281F9
:10B2C00093810E948ABA0E945ABA28966CAF7DAFC9
:10B2D0008EAF9FAF28978091291190912A11A0914C
:10B2E0002B11B0912C1128962CAD3DAD4EAD5FAD1C
:10B2F0002897281739074A075B0709F4B9C0E09176
:10B30000AB0834E0E39FF0011124EA5BFD4E20918D
:10B310003F023091400240914102509142026081CF
:10B320007181828193810E94B5B787FF2FC02896D3
:10B330008CAD9DADAEADBFAD289780932911909394
:10B340002A11A0932B11B0932C11E1EDF7E0849119
:10B35000882341F09091C00095FFFCCF8093C600F8
:10B360003196F5CFE7EBF7E08491882341F0909197
:10B37000C00095FFFCCF8093C6003196F5CF809139
:10B38000C00085FFFCCF8AE08093C6008091291120
:10B3900090912A11A0912B11B0912C1128962CADCF
:10B3A0003DAD4EAD5FAD2897281B390B4A0B5B0BAB
:10B3B000CA01B90157FF07C09095809570956195B6
:10B3C0007F4F8F4F9F4F0E9457B86B017C01609158
:10B3D0000A0970910B0980910C0990910D09680F71
:10B3E000791F882777FD8095982F0E9457B8209164
:10B3F000791130917A1140917B1150917C110E940A
:10B400008ABA9B01AC01C701B6010E94B8B91816EF
:10B410007CF528968CAD9DADAEADBFAD28978093E1
:10B42000291190932A11A0932B11B0932C11E1EDC7
:10B43000F7E08491882341F09091C00095FFFCCF04
:10B440008093C6003196F5CFE9E9F7E0849188232F
:10B4500041F09091C00095FFFCCF8093C6003196DB
:10B46000F5CF8091C00085FFFCCF8AE08093C600B5
:10B470008091370C9DE4899F10011124D101A85CB3
:10B48000B34F1D01FD01E45BFF4F108220911D11A0
:10B4900030911E1140911F11509120112BA33CA3FC
:10B4A0004DA35EA36D964CAC5DAC6EAC7FAC6D975E
:10B4B000421A530A640A750A77FE08C070946094B1
:10B4C00050944094411C511C611C711CD1014D923F
:10B4D0005D926D927C9213972091211130912211EF
:10B4E00040912311509124112FA338A749A75AA79F
:10B4F000A1968CAC9DACAEACBFACA197821A930A5E
:10B50000A40AB50AB7FE08C0B094A09490948094A1
:10B51000811C911CA11CB11CD10114968D929D928D
:10B52000AD92BC9217972091251130912611409130
:10B530002711509128112BA73CA74DA75EA7A596D0
:10B54000CCACDDACEEACFFACA597C21AD30AE40AD2
:10B55000F50AF7FE08C0F094E094D094C094C11CA2
:10B56000D11CE11CF11CD1011896CD92DD92ED9217
:10B57000FC921B972091291130912A1140912B1197
:10B5800050912C112FA738AB49AB5AAB28962CAD54
:10B590003DAD4EAD5FAD28978FA598A9A9A9BAA9D1
:10B5A000281B390B4A0B5B0B57FF07C05095409582
:10B5B000309521953F4F4F4F5F4FA0912B02B09197
:10B5C0002C020E94D4BB24E630E040E050E00E9410
:10B5D000A8BBD1011C962D933D934D935C931F976F
:10B5E000C814D904EA04FB0414F475016401C216FA
:10B5F000D306E406F50614F469017A01D301C20109
:10B600004C145D046E047F0414F4D701C601F101EB
:10B61000808B918BA28BB38B0697A105B10508F4A3
:10B62000B8C7E85BFF4F8091A9089091AA08AA27A4
:10B6300097FDA095BA2F80839183A283B3836D96E3
:10B640002CAD3DAD4EAD5FAD6D978BA19CA1ADA175
:10B65000BEA1281739074A075B0724F0D10190964D
:10B660001C9203C081E0F10180A3A1962CAD3DADF9
:10B670004EAD5FADA1978FA198A5A9A5BAA5281732
:10B6800039074A075B073CF4D10190968C9190975B
:10B69000826090968C93A5962CAD3DAD4EAD5FAD7E
:10B6A000A5978BA59CA5ADA5BEA5281739074A0768
:10B6B0005B073CF4D10190968C91909784609096B2
:10B6C0008C9328962CAD3DAD4EAD5FAD28978FA5E0
:10B6D00098A9A9A9BAA9281739074A075B073CF412
:10B6E000D10190968C919097886090968C93E8AD5C
:10B6F000F9AD8081D10191968C9345284628472841
:10B7000009F05F98F10184819581A681B781892B29
:10B710008A2B8B2B09F08A98F10180859185A2856F
:10B72000B385892B8A2B8B2B41F09FB7F89480919E
:10B7300008018E7F809308019FBFF1018485958564
:10B74000A685B785892B8A2B8B2B11F012984798E9
:10B75000D1011C962D913D914D915C911F972CAF7D
:10B760003DAF4EAF5FAF232B242B252BF1F4B091CF
:10B770003D11BBA3E0913E11EFA3F0913F11FBA758
:10B78000209140112FA72B2F3E2F4F2F5FA56CA983
:10B790007BA9C8010E94B5B787FD18C03CA93BA38F
:10B7A0004BA94FA30BA71FA711C0509159115BA321
:10B7B00080915A118FA390915B119BA7A0915C116E
:10B7C000AFA7252F382F492F5A2FE1CF80911D1178
:10B7D00090911E11A0911F11B09120116D962CAD6A
:10B7E0003DAD4EAD5FAD6D97281B390B4A0B5B0B22
:10B7F000CA01B9010E9457B820916D1130916E11A4
:10B8000040916F11509170110E94BCB72B013C0107
:10B81000698B7A8B8B8B9C8B80912111909122115B
:10B82000A0912311B0912411A1962CAD3DAD4EAD48
:10B830005FADA197281B390B4A0B5B0BCA01B901FD
:10B840000E9457B82091711130917211409173117B
:10B85000509174110E94BCB74B015C016D8B7E8BC3
:10B860008F8B988F8091251190912611A09127118F
:10B87000B0912811A5962CAD3DAD4EAD5FADA5970D
:10B88000281B390B4A0B5B0BCA01B9010E9457B840
:10B890002091751130917611409177115091781166
:10B8A0000E94BCB76B017C01698F7A8F8B8F9C8F54
:10B8B0008091291190912A11A0912B11B0912C11F6
:10B8C00028962CAD3DAD4EAD5FAD2897281B390BAA
:10B8D0004A0B5B0BCA01B9010E9457B8209179113C
:10B8E00030917A1140917B1150917C110E94BCB72C
:10B8F0006CAB7DAB8EAB9FAB60912B0270912C0239
:10B90000882777FD8095982F0E9457B89B01AC013E
:10B910006CA97DA98EA99FA90E948ABA20E030E077
:10B9200048EC52E40E94BCB76D8F7E8F8F8F98A336
:10B93000D1012D913D914D915C91139728AF39AF75
:10B940004AAF5BAF2630310541055105FCF4149632
:10B950000D911D912D913C911797063011052105F0
:10B960003105A4F418960D911D912D913C911B97D2
:10B9700006301105210531054CF4DC01CB01BF7700
:10B98000F10186A797A7A0ABB1AB25C0C301B20157
:10B990000E9435BB2B013C01C501B4010E9435BB9F
:10B9A0009B01AC01C301B2010E94DCB64B015C01FA
:10B9B000C701B6010E9435BB9B01AC01C501B401B2
:10B9C0000E94DCB60E94F7BAD1019E966D937D93DA
:10B9D0008D939C93D197D1019E962D913D914D9140
:10B9E0005C91D19769962CAF3DAF4EAF5FAF699731
:10B9F00060E070E080E89FE30E94BCB79B01AC016F
:10BA00006BA17FA18BA59FA50E948ABA2B013C0147
:10BA10009091370C8091360CE92FF0E0E81BF1098A
:10BA2000EF70FF27FDABECABA301920160E074E285
:10BA300084E799E40E94BCB70E945ABA6B017C016A
:10BA40002CA93DA9223031050CF442C04901AA2499
:10BA500097FCA094BA2CC501B4010E9457B820E00D
:10BA600030E040E051E40E94B5B787FF31C08091DB
:10BA70008D1190918E11A0918F11B0919011C816D7
:10BA8000D906EA06FB0620F5BC01CD016C197D093B
:10BA90008E099F09660F771F881F991FA5019401C2
:10BAA0000E9486BBCA01B9010E9455B80E945ABAC9
:10BAB0006C0D7D1D8E1D9F1D0E9455B89B01AC0114
:10BAC00060E074E284E799E40E94BCB72B013C017A
:10BAD000A301920169966CAD7DAD8EAD9FAD699766
:10BAE0000E948ABA24966CAF7DAF8EAF9FAF249729
:10BAF000D10192966D937D938D939C9395975096DB
:10BB00006D917D918D919C9153970E9455B86BA337
:10BB10007CA38DA39EA3A30192010E948ABA0E94D6
:10BB2000A2B70E9429B86B017C01F10160AF71AF2F
:10BB300082AF93AF8E010F5E1F4F2DE731E1639609
:10BB40003FAF2EAF6397AE014F5D5F4F5AA349A33E
:10BB5000CE0101962F969FAF8EAF2F971FA21BA6E7
:10BB600090E89FA7AFE3ABABF80161917191819130
:10BB700091918F01A30192010E948ABA2F96AEADD6
:10BB8000BFAD2F976D937D938D939D932F96BFAFF0
:10BB9000AEAF2F979B01AC015F772D962CAF3DAFD9
:10BBA0004EAF5FAF2D976396AEADBFAD63978D90EF
:10BBB0009D90AD90BD906396BFAFAEAF6397A5016A
:10BBC00094012D966CAD7DAD8EAD9FAD2D970E94ED
:10BBD000B8B91816F4F42D962CAD3DAD4EAD5FAD51
:10BBE0002D97C501B4010E94BCB7B62EA72E982E82
:10BBF000892E262F372F482F592F6FA17BA58FA570
:10BC00009BA90E94B5B787FD04C0BFA2ABA69FA6A3
:10BC10008BAAE9A1FAA10E171F0709F0A5CF20E012
:10BC200030E040E85FE36FA17BA58FA59BA90E9450
:10BC3000B5B787FF3FC05E01F1E1AF0EB11C8E01C9
:10BC40000F5F1F4F2FA13BA54FA55BA9D8016D9199
:10BC50007D918D919C910E948ABAF80161937193B4
:10BC6000819391938F01EA15FB0561F72FA13BA505
:10BC70004FA55BA924966CAD7DAD8EAD9FAD24978D
:10BC80000E948ABAD10192966D937D938D939C9375
:10BC90009597C701B6010E9455B82FA13BA54FA5A6
:10BCA0005BA90E948ABA0E9429B8F10160AF71AF06
:10BCB00082AF93AF69962CAD3DAD4EAD5FAD699748
:10BCC0006BA17CA18DA19EA10E94BCB76B017C01E0
:10BCD00028AD39AD4AAD5BAD232B242B252B59F56F
:10BCE000F10184819581A681B781892B8A2B8B2BC9
:10BCF00011F580859185A285B385892B8A2B8B2BA5
:10BD0000D1F4209151113091521140915311509121
:10BD10005411C701B6010E948ABA0E94A2B78101DC
:10BD20000C5B1F4F0E9429B8D8016D937D938D93B2
:10BD30009C931397F4C02091551130915611409166
:10BD4000571150915811C701B6010E948ABA0E943A
:10BD5000A2B70E9429B881010C5B1F4FF8016083D4
:10BD600071838283938340902D1150902E116090A7
:10BD70002F11709030110E9455B84B015C0168ADD5
:10BD800079AD8AAD9BAD0E9457B89B01AC01C5014E
:10BD9000B4010E948ABA2BA13CA14DA15EA10E94D0
:10BDA000BCB74B015C01C301B2010E9455B89B01B5
:10BDB000AC01C501B4010E94B8B9181634F4D80119
:10BDC0004D925D926D927C921397409031115090FC
:10BDD00032116090331170903411F80160817181DB
:10BDE000828193810E9455B84B015C01D101149668
:10BDF0006D917D918D919C9117970E9457B89B01F1
:10BE0000AC01C501B4010E948ABA2BA13CA14DA18D
:10BE10005EA10E94BCB74B015C01C301B2010E944C
:10BE200055B89B01AC01C501B4010E94B8B9181600
:10BE30002CF4F80140825182628273824090391161
:10BE400050903A1160903B1170903C1181010C5B55
:10BE50001F4FD8016D917D918D919C910E9455B895
:10BE60004B015C016CAD7DAD8EAD9FAD0E9457B8AE
:10BE70009B01AC01C501B4010E948ABA2BA13CA16F
:10BE80004DA15EA10E94BCB74B015C01C301B20190
:10BE90000E9455B89B01AC01C501B4010E94B8B91C
:10BEA00018162CF4F801408251826282738240900D
:10BEB0003511509036116090371170903811D801BB
:10BEC0006D917D918D919C910E9455B84B015C01C3
:10BED000F10160857185828593850E9457B89B0129
:10BEE000AC01C501B4010E948ABA2BA13CA14DA1AD
:10BEF0005EA10E94BCB74B015C01C301B2010E946C
:10BF000055B89B01AC01C501B4010E94B8B918161F
:10BF100034F4D8014D925D926D927C921397F101A9
:10BF2000EC5BFF4F60817181828193810E9455B8E3
:10BF30004B015C01A70196010E94BCB7AC966CAFA7
:10BF40007DAF8EAF9FAFAC97F10162AB73AB84ABAB
:10BF500095AB2DEB37E346E051E4C501B4010E94F7
:10BF60008ABA0E9424B8D1015C966D937D938D931B
:10BF70009C935F9720914D1130914E1140914F113C
:10BF8000509150112D962CAF3DAF4EAF5FAF2D9716
:10BF900020E030E040E05FE32D966CAD7DAD8EADEE
:10BFA0009FAD2D970E948ABA6BA37FA38BA79FA7F3
:10BFB0008D809E80AF80B8848091491190914A1104
:10BFC000A0914B11B0914C1161968CAF9DAFAEAF6B
:10BFD000BFAF619720E030E040E05FE3BC01CD01FE
:10BFE0000E948ABAF62EE72ED82EC92EC501B401BA
:10BFF0009F772F2D3E2D4D2D5C2D0E94B8B9181620
:10C0000084F42F2D3E2D4D2D5C2D6BA17FA18BA592
:10C010009FA50E94B5B787FD04C0FBA2EFA2DBA6D7
:10C02000CFA629853A854B855C85E0962CAF3DAF40
:10C030004EAF5FAFE0978091451190914611A0916E
:10C040004711B091481165968CAF9DAFAEAFBFAFB1
:10C05000659720E030E040E05FE3BC01CD010E9445
:10C060008ABAF62EE72ED82EC92EE0966CAD7DAD9D
:10C070008EAD9FADE0979F772F2D3E2D4D2D5C2DE2
:10C080000E94B8B9181684F42F2D3E2D4D2D5C2D2D
:10C090006BA17FA18BA59FA50E94B5B787FD04C0AA
:10C0A000FBA2EFA2DBA6CFA62D853E854F85588942
:10C0B000E4962CAF3DAF4EAF5FAFE497C090411117
:10C0C000D0904211E0904311F090441120E030E014
:10C0D00040E05FE3C701B6010E948ABA762E672E60
:10C0E000582E492EE4966CAD7DAD8EAD9FADE49794
:10C0F0009F77272D362D452D542D0E94B8B918163F
:10C1000084F4272D362D452D542D6BA17FA18BA5B1
:10C110009FA50E94B5B787FD04C07BA26FA25BA656
:10C120004FA6D1019296BC91BBABF101F3A1F8AF40
:10C13000D1019496BC91BCAFF101F5A12196FFAF5E
:10C1400021972BA938AD4B2F5F2F6BA17FA18BA51A
:10C150009FA50E94B5B787FD0AC02BA92BA338ADB8
:10C160003FA34CAD4BA721965FAD21975FA78CA94C
:10C170009DA902970CF423C1909109119CABA09149
:10C180000A11A696AFAFA697B0910B11A796BFAFB5
:10C19000A797E0910C11A896EFAFA89727E137EB8E
:10C1A00041ED58E3692F7A2F8B2F9E2F0E94B8B94B
:10C1B00018160CF004C120910D1130910E11409110
:10C1C0000F115091101169817A818B819C810E949D
:10C1D000DBB62B013C0120911111309112114091DD
:10C1E000131150911411C501B4010E94DBB64B012B
:10C1F0005C01A3019201C301B2010E948ABA2B0122
:10C200003C01A5019401C501B4010E948ABA9B01B9
:10C21000AC01C301B2010E94DCB60E94F7BA4B0127
:10C220005C012D962CAD3DAD4EAD5FAD2D970E94BE
:10C23000B8B918166CF4A50194012D966CAD7DADBE
:10C240008EAD9FAD2D970E94BCB73B018C0104C001
:10C25000612C712C00E81FE361962CAD3DAD4EAD15
:10C260005FAD6197C501B4010E94B8B9181664F4B6
:10C27000A501940161966CAD7DAD8EAD9FAD6197CA
:10C280000E94BCB73B018C01209115113091161111
:10C290004091171150911811E0966CAD7DAD8EADA7
:10C2A0009FADE0970E94DBB64B015C01E894B7F8C4
:10C2B00065962CAD3DAD4EAD5FAD6597C501B40142
:10C2C0000E94B8B91816E4F4A501940165966CAD06
:10C2D0007DAD8EAD9FAD65970E94BCB7B62EA72EE3
:10C2E000982E892E262F372F482F592FB301C8019A
:10C2F0000E94B5B787FD04C06B2C7A2C092D182D30
:10C300002091191130911A1140911B1150911C115B
:10C31000E4966CAD7DAD8EAD9FADE4970E94DBB62B
:10C320004B015C01E894B7F8A7019601C501B4017F
:10C330000E94B8B91816C4F4A5019401C701B6014A
:10C340000E94BCB7F62EE72ED82EC92E262F372FE7
:10C35000482F592FB301C8010E94B5B787FD04C00B
:10C360006F2C7E2C0D2D1C2D9301A8016BA978AD8F
:10C370008CAD21969FAD21970E948ABAA62E072FD9
:10C38000182FB92E262F372F482F592F6CA9A69674
:10C390007FADA697A7968FADA797A8969FADA897B4
:10C3A0000E94B5B787FF0FC0ACA8A6960FADA697A1
:10C3B000A7961FADA797A896BFACA89704C0ABA03F
:10C3C0000FA11BA5BFA48A2D902FA12FBB2DF1017A
:10C3D00082A793A7A4A7B5A7AC966CAD7DAD8EAD93
:10C3E0009FADAC9790589B01AC010E94DCB669965A
:10C3F0002CAD3DAD4EAD5FAD69970E948ABA9B01F1
:10C40000AC016BE077ED83E29BE30E94DBB60E9418
:10C41000F7BA7B01D82EC92E9B01482F592F6A2DC0
:10C42000702F812F9B2D0E94B5B787FD04C0AE2CC5
:10C430000F2D1D2DBC2C8A2D902FA12FBB2DF1016E
:10C4400086A397A3A0A7B1A797014D2D5C2D6BA93B
:10C4500078AD8CAD21969FAD21970E94B5B7181687
:10C460002CF081E0D101D7968C9302C0F10117AA7C
:10C4700081E0D101D6968C9380E1FE013196ADE04A
:10C48000B1E101900D928A95E1F78BA998ADACAD21
:10C490002196BFAD21978093091190930A11A09323
:10C4A0000B11B0930C119C01AD016BA17FA18BA569
:10C4B0009FA50E94BCB76B017C012BA938AD4CAD88
:10C4C00021965FAD21976A2D702F812F9B2D0E94A1
:10C4D000BCB7AB01BC0197018601C1010E94AD53FD
:10C4E0002996BFAD2997B093370C6D962CAD3DAD15
:10C4F0004EAD5FAD6D9720931D1130931E1140938B
:10C500001F1150932011A1968CAD9DADAEADBFAD66
:10C51000A1978093211190932211A0932311B0939E
:10C520002411A5962CAD3DAD4EAD5FADA5972093E2
:10C5300025113093261140932711509328112896E6
:10C540008CAD9DADAEADBFAD289780932911909372
:10C550002A11A0932B11B0932C110E946457CD582F
:10C56000DF4F0FB6F894DEBF0FBECDBFDF91CF9186
:10C570001F910F91FF90EF90DF90CF90BF90AF9001
:10C580009F908F907F906F905F904F903F902F90F3
:10C59000D2C1CD58DF4F0FB6F894DEBF0FBECDBF6E
:10C5A000DF91CF911F910F91FF90EF90DF90CF908F
:10C5B000BF90AF909F908F907F906F905F904F90C3
:10C5C0003F902F900895EF92FF920F931F93CF9378
:10C5D000DF937B018A01E90120916D1130916E1189
:10C5E00040916F1150917011FC01608171818281C5
:10C5F00093810E948ABA0E945ABA60931D11709367
:10C600001E1180931F119093201120917111309170
:10C6100072114091731150917411F7016081718111
:10C62000828193810E948ABA0E945ABA6093211132
:10C6300070932211809323119093241120917511EE
:10C64000309176114091771150917811F801608105
:10C650007181828193810E948ABA0E945ABA609342
:10C660002511709326118093271190932811209102
:10C67000791130917A1140917B1150917C11688130
:10C6800079818A819B810E948ABA0E945ABA6093FA
:10C69000291170932A1180932B1190932C1129E268
:10C6A00031E145E251E161E271E18DE191E10E9408
:10C6B000D56B1092091110920A1110920B11109261
:10C6C0000C1110920D1110920E1110920F11109268
:10C6D0001011109211111092121110921311109248
:10C6E0001411109215111092161110921711109228
:10C6F00018111092191110921A1110921B11109208
:10C700001C11DF91CF911F910F91FF90EF90089531
:10C710002091791130917A1140917B1150917C11C7
:10C72000FC0160817181828193810E948ABA0E949A
:10C730005ABA6093291170932A1180932B11909308
:10C740002C1189E291E10C94116C60933F0270937B
:10C75000400280934102909342020895CF92DF926B
:10C76000EF92FF920F931F93CF93DF9300D01F920E
:10C77000CDB7DEB76DE5C62E61E1D62E7DE6E72E9C
:10C7800071E1F72E0DE211E1F60161917191819154
:10C7900091916F01F70121913191419151917F0167
:10C7A00029833A834B835C830E9455B829813A815F
:10C7B0004B815C810E948ABA0E9429B8F80161937A
:10C7C0007193819391938F01FDE6CF16F1E1DF061E
:10C7D000D9F60F900F900F900F90DF91CF911F918E
:10C7E0000F91FF90EF90DF90CF9008958091A61168
:10C7F000811109C08091A511811105C08091A411FA
:10C80000811101C00895E2E2F0E18491882341F0B2
:10C810009091C00095FFFCCF8093C6003196F5CF74
:10C82000E3E1F8E08491882341F09091C00095FF06
:10C83000FCCF8093C6003196F5CF8091A611882356
:10C84000F1F06091A7117091A8118091A9119091B8
:10C85000AA110E9457B820916D1130916E1140912C
:10C860006F11509170110E94BCB7AB01BC018FE0F9
:10C8700098E00E9422198FEF97E00E940D87809127
:10C88000A5118823F1F06091AB117091AC118091EA
:10C89000AD119091AE110E9457B820917111309155
:10C8A000721140917311509174110E94BCB7AB0189
:10C8B000BC018BEF97E00E9422198BEE97E00E945B
:10C8C0000D878091A4118823F1F06091AF117091D0
:10C8D000B0118091B1119091B2110E9457B820917E
:10C8E00075113091761140917711509178110E9415
:10C8F000BCB7AB01BC0187EE97E00E94221987ED1F
:10C9000097E00E940D878091C00085FFFCCF8AE0F0
:10C910008093C6001092A6111092A5111092A41136
:10C9200008951092A6111092A5111092A4110895C5
:10C93000809353020895EFE6F0E080818260808367
:10C9400008951F920F920FB60F9211240BB60F92FB
:10C950000F931F932F933F934F935F936F937F9307
:10C960008F939F93AF93BF93EF93FF938091D711D2
:10C970009091D811892B09F086C19091370C809144
:10C98000360C981771F0E091360C8DE4E89FF001B9
:10C990001124E85CF34FDF01A45BBF4F81E08C936F
:10C9A00002C0E0E0F0E0F093D811E093D7113097A7
:10C9B00009F463C1DF01A45BBF4F81E08C93109247
:10C9C000BA111092BB111092BC111092BD1160AD42
:10C9D00071AD61349CE9790728F461329EE47907EE
:10C9E00048F002C060E47CE9769567957695679596
:10C9F00084E007C0613197E2790730F0769567955A
:10CA000082E08093B71107C08093B711603271053F
:10CA100010F460E270E060527109611588E07807F7
:10CA2000D0F0872F9927880F991F880F991F8E5D47
:10CA3000934FFC01329645915491AA27659F90012E
:10CA4000649F210D3A1F06942A1F3A1F1124FC01EE
:10CA5000859194911DC0CB01969587958C7F8E5DB5
:10CA6000974FFC01459154910296FC018591949158
:10CA7000FB01E770FF278E9F90018F9F300D9E9FD7
:10CA8000300D1124E3E036952795EA95E1F7CA01C8
:10CA9000821B930B84369105A0F4EAEEF3E08191BA
:10CAA000882339F09091C00095FFFCCF8093C60099
:10CAB000F6CF4AE050E082E795E00E94FC1684E65B
:10CAC00090E09093B6118093B5118091B71199279A
:10CAD00087FD90959093B4118093B311E091D71195
:10CAE000F091D81164AD75AD7093B9116093B81120
:10CAF00061349CE9790728F461328EE4780748F0C4
:10CB000002C060E47CE9769567957695679584E048
:10CB100007C0613197E2790730F07695679582E03A
:10CB20008093B71108C081E08093B711603271051E
:10CB300010F460E270E060527109611588E07807D6
:10CB4000E0F0872F9927880F991F880F991F8E5D16
:10CB5000934FFC01329625913491AA27639FA0013F
:10CB6000629F410D5A1F06944A1F5A1F1124FC014F
:10CB700025913491241B350B1EC0CB0196958795CA
:10CB80008C7F8E5D974FFC01259134910296FC01BC
:10CB900045915491FB01E770FF274E9FC0014F9FC5
:10CBA000900D5E9F900D1124F3E096958795FA9570
:10CBB000E1F7281B390B24363105A0F4EAEEF3E047
:10CBC0008191882339F09091C00095FFFCCF80932C
:10CBD000C600F6CF4AE050E082E795E00E94FC16DE
:10CBE00024E630E0C901A0E0B0E08093BE1190934C
:10CBF000BF11A093C011B093C1113093890020934D
:10CC00008800E091D711F091D81180899189A2898B
:10CC1000B389B695A79597958795B095A09590956A
:10CC200081959F4FAF4FBF4F8093D2119093D311F7
:10CC3000A093D411B093D5118093CE119093CF11BE
:10CC4000A093D011B093D1118093CA119093CB11BE
:10CC5000A093CC11B093CD118093C6119093C711BE
:10CC6000A093C811B093C9111092C2111092C311B0
:10CC70001092C4111092C51106C080ED97E09093F8
:10CC8000890080938800E091D711F091D8113097F6
:10CC900009F4DCC480A18093D61180FF41C0899A39
:10CCA0008FEF80934F02809153028823E9F12CB1DA
:10CCB00031E025FB222720F9232779F18091A31168
:10CCC000882359F1E091D711F091D8118081918199
:10CCD000A281B381181619061A061B06F4F4809176
:10CCE000911190919211A0919311B0919411809310
:10CCF000A7119093A811A093A911B093AA113093F2
:10CD0000A61180899189A289B3898093C2119093D9
:10CD1000C311A093C411B093C5112093A31104C0F3
:10CD2000899881E080934F028091D61181FF41C0A4
:10CD30008F9A8FEF80935002809153028823E9F1FC
:10CD40002091030131E026952170232779F180910C
:10CD5000A211882359F1E091D711F091D811848163
:10CD60009581A681B781181619061A061B06F4F4D8
:10CD70008091951190919611A0919711B091981171
:10CD80008093AB119093AC11A093AD11B093AE1101
:10CD90003093A51180899189A289B3898093C211AA
:10CDA0009093C311A093C411B093C5112093A21105
:10CDB00004C08F9881E0809350028091D6119FB774
:10CDC00082FF48C0F89480910B018D7F80930B0106
:10CDD0009FBF8FEF8093510280915302882309F403
:10CDE00043C029B131E023FB222720F9232779F121
:10CDF0008091A111882359F1E091D711F091D811B8
:10CE000080859185A285B385181619061A061B061A
:10CE1000F4F48091991190919A11A0919B11B09185
:10CE20009C118093AF119093B011A093B111B09366
:10CE3000B2113093A41180899189A289B38980931A
:10CE4000C2119093C311A093C411B093C511209344
:10CE5000A1110AC0F89480910B01826080930B01AC
:10CE60009FBF81E0809351028091D611E091D7114C
:10CE7000F091D81183FF08C081A1813011F443984B
:10CE800001C0169A8FEF07C081A1813011F4439A37
:10CE900001C0169881E08093520220E08091B71182
:10CEA00028170CF0C7C18091C00087FF19C03091CE
:10CEB000C6004091F3055091F405CA0101968F77A1
:10CEC00099276091F5057091F6058617970741F04F
:10CED000FA01ED58FA4F30839093F4058093F305EF
:10CEE000E091D711F091D8118091D2119091D31186
:10CEF000A091D411B091D51140815181628173818B
:10CF0000840F951FA61FB71F8093D2119093D31142
:10CF1000A093D411B093D511181619061A061B0642
:10CF2000CCF5889AE091D711F091D8118091D21167
:10CF30009091D311A091D411B091D511408951890C
:10CF400062897389841B950BA60BB70B8093D21152
:10CF50009093D311A093D411B093D51140914F0267
:10CF60008091911190919211A0919311B09194118F
:10CF7000552747FD5095652F752F840F951FA61FC8
:10CF8000B71F8093911190939211A0939311B09336
:10CF900094118898E091D711F091D8118091CE1119
:10CFA0009091CF11A091D011B091D11144815581B0
:10CFB00066817781840F951FA61FB71F8093CE11BE
:10CFC0009093CF11A093D011B093D11118161906D8
:10CFD0001A061B06CCF58E9AE091D711F091D81164
:10CFE0008091CE119091CF11A091D011B091D1111B
:10CFF0004089518962897389841B950BA60BB70BF5
:10D000008093CE119093CF11A093D011B093D111F2
:10D01000409150028091951190919611A091971195
:10D02000B0919811552747FD5095652F752F840FA6
:10D03000951FA61FB71F8093951190939611A093EB
:10D040009711B09398118E98E091D711F091D81163
:10D050008091CA119091CB11A091CC11B091CD11BA
:10D060004085518562857385840F951FA61FB71F64
:10D070008093CA119093CB11A093CC11B093CD1192
:10D08000181619061A061B060CF047C09FB7F8942D
:10D0900080910B01886080930B019FBFE091D711B5
:10D0A000F091D8118091CA119091CB11A091CC111F
:10D0B000B091CD114089518962897389841B950B88
:10D0C000A60BB70B8093CA119093CB11A093CC11F0
:10D0D000B093CD11409151028091991190919A1184
:10D0E000A0919B11B0919C11552747FD5095652F3C
:10D0F000752F840F951FA61FB71F809399119093CA
:10D100009A11A0939B11B0939C119FB7F8948091B2
:10D110000B01877F80930B019FBFE091D711F091A6
:10D12000D8118091C6119091C711A091C811B091EA
:10D13000C9114485558566857785840F951FA61F7F
:10D14000B71F8093C6119093C711A093C811B093D5
:10D15000C911181619061A061B060CF043C081A146
:10D16000813011F4419A01C0149AE091D711F091E5
:10D17000D8118091C6119091C711A091C811B0919A
:10D18000C9114089518962897389841B950BA60B4B
:10D19000B70B8093C6119093C711A093C811B09399
:10D1A000C9114091520280919D1190919E11A091C0
:10D1B0009F11B091A011552747FD5095652F752FF0
:10D1C000840F951FA61FB71F80939D1190939E11EA
:10D1D000A0939F11B093A01181A1813011F44198C7
:10D1E00001C014988091C2119091C311A091C411F3
:10D1F000B091C5110196A11DB11D8093C2119093EC
:10D20000C311A093C411B093C5114091C2115091A4
:10D21000C3116091C4117091C511E091D711F091C3
:10D22000D81180899189A289B389481759076A075B
:10D230007B07B0F04091C2115091C3116091C411AD
:10D240007091C511E091D711F091D8118489958919
:10D25000A689B78984179507A607B70718F4DAC017
:10D260002F5F1CCE4091BE115091BF116091C01133
:10D270007091C111048D158D268D378DAA27419F80
:10D28000B12D529FC001629F900D619F800D911D35
:10D29000429FB00D811D9A1F519FB00D811D9A1F95
:10D2A000609FB00D811D9A1F509FB10D8A1F9A1F5C
:10D2B000B6958A1F9A1F112444AD55AD480F591FCA
:10D2C0005093B9114093B81180AD91ADA2ADB3ADFB
:10D2D00060E070E084179507A607B70720F49093E5
:10D2E000B9118093B8116091B8117091B91161347E
:10D2F0009CE9790728F461328EE4780748F002C08F
:10D3000060E47CE9769567957695679584E007C03B
:10D31000613197E2790730F07695679582E08093E6
:10D32000B71108C081E08093B7116032710510F425
:10D3300060E270E060527109611588E07807E0F002
:10D34000872F9927880F991F880F991F8E5D934FFC
:10D35000FC01329625913491AA27639FA001629F18
:10D36000410D5A1F06944A1F5A1F1124FC01259192
:10D370003491241B350B1EC0CB01969587958C7F6D
:10D380008E5D974FFC01259134910296FC014591E9
:10D390005491FB01E770FF274E9FC0014F9F900DF6
:10D3A0005E9F900D112413E0969587951A95E1F7ED
:10D3B000281B390B24363105A0F4EAEEF3E0819105
:10D3C000882339F09091C00095FFFCCF8093C60070
:10D3D000F6CF4AE050E082E795E00E94FC1624E692
:10D3E00030E030938900209388008091BE119091A5
:10D3F000BF11A091C011B091C111820F931FA11D47
:10D40000B11D8093BE119093BF11A093C011B09332
:10D41000C111F7C04091C2115091C3116091C41164
:10D420007091C511808D918DA28DB38D8417950754
:10D43000A607B70708F0D9C04091BA115091BB11A7
:10D440006091BC117091BD11048D158D268D378DA5
:10D45000AA27419FB12D529FC001629F900D619FED
:10D46000800D911D429FB00D811D9A1F519FB00DDF
:10D47000811D9A1F609FB00D811D9A1F509FB10D95
:10D480008A1F9A1FB6958A1F9A1F11242091B811DE
:10D490003091B911E05CFF4F2817390718F420814B
:10D4A000318102C0281B390B80819181A281B38117
:10D4B000A90160E070E0481759076A077B0708F484
:10D4C0009C0121349CE9390728F421328EE4380785
:10D4D00048F002C020E43CE936952795369527951B
:10D4E00084E007C0213197E2390730F0369527955F
:10D4F00082E08093B71108C081E08093B711203299
:10D50000310510F420E230E0B90160527109611573
:10D5100088E07807E0F0872F9927880F991F880FF8
:10D52000991F8E5D934FFC01329625913491AA2765
:10D53000639FA001629F410D5A1F06944A1F5A1F04
:10D540001124FC0125913491241B350B1EC0CB0105
:10D55000969587958C7F8E5D974FFC012591349130
:10D560000296FC0145915491FB01E770FF274E9F05
:10D57000C0014F9F900D5E9F900D112443E0969542
:10D5800087954A95E1F7281B390B24363105A0F41D
:10D59000EAEEF3E08191882339F09091C00095FF85
:10D5A000FCCF8093C600F6CF4AE050E082E795E0DA
:10D5B0000E94FC1624E630E0309389002093880016
:10D5C0008091BA119091BB11A091BC11B091BD1185
:10D5D000820F931FA11DB11D8093BA119093BB11AF
:10D5E000A093BC11B093BD110CC08091B511909166
:10D5F000B61190938900809388008091B311809335
:10D60000B7114091C2115091C3116091C411709132
:10D61000C511E091D711F091D81180899189A28923
:10D62000B389481759076A077B0780F01092D81111
:10D630001092D7119091370C8091360C981731F0D9
:10D640008091360C8F5F8F708093360CFF91EF9135
:10D65000BF91AF919F918F917F916F915F914F910A
:10D660003F912F911F910F910F900BBE0F900FBE06
:10D670000F901F901895819A879AEAE0F1E08081D7
:10D68000826080830E9A3B9A579A5F9A829A8A9A0E
:10D69000E7E0F1E08081816080839FB7F894E8E063
:10D6A000F1E08081816080839FBF0A9A129A3F9A3D
:10D6B000479A6C98749AE4E0F1E080818E7F8083D1
:10D6C0009FB7F894E5E0F1E08081816080839FBF9F
:10D6D0006D98759AE4E0F1E080818D7F80839FB73B
:10D6E000F894E5E0F1E08081826080839FBF5398E9
:10D6F0005B9A809A88985F9A869A8E988A9AEAE0CE
:10D70000F1E08081886080839FB7F894EBE0F1E0DE
:10D710008081877F80839FBF9FB7F894E8E0F1E026
:10D720008081816080839FBF0C9A1498129A399AE5
:10D730004198479AA1E8B0E08C918F7E8C938C91B0
:10D7400088608C93E0E8F0E080818D7F8083808129
:10D750008E7F808380818F73808380818F7C8083A4
:10D760008C91887F82608C9380E090E49093890014
:10D77000809388001092850010928400EFE6F0E01C
:10D7800080818260808381E0809353027894089541
:10D790009091370C8091360C981731F035D20E9459
:10D7A00085230E945088F4CF0895CF93DF93EFB77D
:10D7B000F894EC0188819981AA81BB8180939111B1
:10D7C00090939211A0939311B0939411EB018881DF
:10D7D0009981AA81BB818093951190939611A09312
:10D7E0009711B0939811EA0188819981AA81BB8130
:10D7F0008093991190939A11A0939B11B0939C11CF
:10D80000E90188819981AA81BB8180939D119093C0
:10D810009E11A0939F11B093A011EFBFDF91CF9104
:10D8200008952FB7F894FC0180819181A281B38182
:10D8300080939D1190939E11A0939F11B093A0117E
:10D840002FBF08952FB7F89494E0899FF001112419
:10D85000EF56FE4E60817181828193812FBF0895C2
:10D8600097DF5F9A8A9A9FB7F894E8E0F1E08081A9
:10D87000816080839FBF129A479A089580916F00BC
:10D880008D7F80936F009091370C8091360C9813A8
:10D890000CC01092D8111092D71180916F00826045
:10D8A00080936F001092FE0808959091370C80913C
:10D8B000360C981741F38091360C8F5F8F708093F0
:10D8C000360CE1CF2F923F924F925F926F927F92F0
:10D8D0008F929F92AF92BF92CF92DF92EF92FF9280
:10D8E0000F931F93CF93DF9300D000D0CDB7DEB757
:10D8F0008C01F62E21E0261760F5E2E3F1E1849138
:10D90000882341F09091C00095FFFCCF8093C60022
:10D910003196F5CF8F2D90E04AE050E0BC0182E7D0
:10D9200095E00E94BF16E8E2F0E18491882341F07F
:10D930009091C00095FFFCCF8093C6003196F5CF43
:10D940008091C00085FFFCCF8AE08093C6000E94D2
:10D950004C236F2D70E0FB01EE0FFF1FE45CFB4FCB
:10D96000408151815E834D83452B09F4A6C0FB01A4
:10D97000E65CFB4F50815A832D813E812C5F3F4FE7
:10D9800081E090E089836A81861708F07BC0DC0122
:10D99000F901459154910196B9016C5F7F4F0417CD
:10D9A00015070CF06DC00297AC01440F551F440FD2
:10D9B000551F4E5F5F4F6D817E81460F571FFA01E5
:10D9C00065917491880F991F880F991FED81FE81D1
:10D9D0008E0F9F1FFC01A590B490FD01EE0FFF1F5D
:10D9E000EE0FFF1F3296AD81BE81EA0FFB1FC5907F
:10D9F000D490FA01E590F490F90125903490FC015F
:10DA0000259134913C832B83882777FD8095982F2F
:10DA10000E9457B82B013C01B8016A197B0988277D
:10DA200077FD8095982F0E9457B84B015C01B60195
:10DA30006E197F09882777FD8095982F0E9457B827
:10DA40009B01AC01C501B4010E948ABA6B017C0143
:10DA5000B1014B815C81641B750B882777FD809534
:10DA6000982F0E9457B89B01AC01C701B6010E94D4
:10DA7000BCB79B01AC01C301B2010E94DCB606C079
:10DA80009B0180CF60E070E080E090E0A981BA81E6
:10DA9000AB132BC02D813E81E4E0AE9F200D311DE4
:10DAA000112422503109F90165917491882777FD7D
:10DAB0008095982F0E9457B818C0B801882777FD25
:10DAC0008095982F0E9457B820E030E04AEF5EE33F
:10DAD0000E948ABA20E030E040E85DE30E948ABA02
:10DAE00020E030E0A9010E94DCB626960FB6F8943B
:10DAF000DEBF0FBECDBFDF91CF911F910F91FF9081
:10DB0000EF90DF90CF90BF90AF909F908F907F90DD
:10DB10006F905F904F903F902F90089580914E129C
:10DB200090914F129093110980931009209103094D
:10DB300020FD09C01092461210924712109248120E
:10DB4000109249120AC060E0BDDE609346127093E5
:10DB500047128093481290934912809150129091ED
:10DB6000511290931309809312092091030921FF08
:10DB70000BC061E0A7DE60934A1270934B12809352
:10DB80004C1290934D1208C010924A1210924B12F0
:10DB900010924C1210924D1210924012109241129B
:10DBA00010924212109243128FB7F89410923F12C3
:10DBB0008FBF0895209165023091660240916702FF
:10DBC0005091680260E070E08FE793E40E94BCB778
:10DBD0006093FF11709300128093011290930212D0
:10DBE00060930312709304128093051290930612AF
:10DBF000089597FF03C08091F61104C0FC01E9501D
:10DC0000FE4E808190E008952F923F924F925F9256
:10DC10006F927F928F929F92AF92BF92CF92DF923C
:10DC2000EF92FF920F931F93CF93DF93CDB7DEB7A1
:10DC3000A2970FB6F894DEBF0FBECDBF80913F1202
:10DC4000882309F4D2C16ADF8091690290916A0247
:10DC5000A0916B02B0916C028D8B9E8BAF8BB88FB5
:10DC60008091650290916602A0916702B09168026E
:10DC7000898F9A8FAB8FBC8F8091610290916202E5
:10DC8000A0916302B09164028D8F9E8FAF8FB8A375
:10DC9000A6E4B2E1BA8BA98BE4E5F2E1F88BEF8759
:10DCA0008FE092E19A878987A7EFB1E1BA83A983D0
:10DCB000E5E5F2E0F887EF838EEE91E19C8B8B8BAC
:10DCC0000DEF11E147E3242E42E1342EAFE2B2E141
:10DCD000BC83AB83E7E1F2E1FE83ED831AA219A2D4
:10DCE000A989BA898D909D90AD90BD90BA8BA98B72
:10DCF000EF85F88961907190F88BEF87B3018827E1
:10DD000077FD8095982F0E9457B8A50194010E9435
:10DD1000DBB66B017C01A985BA856D937D938D93EC
:10DD20009D93BA87A98720E030E040E251E40E9449
:10DD3000B8B9181624F421E0F8012083D6C020E0F9
:10DD400030E040E251ECC701B6010E94B5B787FD53
:10DD500002C0672821F4E1E0D801EC93CDC0D801DE
:10DD60008C91882331F0F10110821182128213828A
:10DD70001C92A70196016D897E898F89988D0E94DA
:10DD80008ABA6B877C878D879E87E9A1FAA1E95DB6
:10DD9000FD4E6083718382839383D1012D913D91E8
:10DDA0004D915C91C701B6010E94DCB66B017C010C
:10DDB000E9A1FAA1E95FFD4E508061807280438045
:10DDC000252D362D472D542D0E94B5B787FD16C041
:10DDD000E9A1FAA1E150FE4E50806180728043803B
:10DDE000252D362D472D542DB601C7010E94B8B9F7
:10DDF000181624F05C2C6D2C7E2C4F2C852D962D26
:10DE0000A72DB42DF10180839183A283B383252DA7
:10DE1000362D472D542D698D7A8D8B8D9C8D0E94CA
:10DE20008ABA2B013C01E9A1FAA1E15EFD4E6083B3
:10DE3000718382839383AB81BC812D913D914D9100
:10DE40005C91C501B4010E94DBB69B01AC016D8DF4
:10DE50007E8D8F8D98A10E948ABA20ED3CEC4CE417
:10DE60005DE30E948ABA6B017C0123E333E343E75D
:10DE70005FE3ED81FE8160817181828193810E94E7
:10DE80008ABA9B01AC01C701B6010E94DCB66B01E6
:10DE90007C01AD81BE816D937D938D939C9313978F
:10DEA000EB81FC8180829182A282B382A3019201E4
:10DEB0006B857C858D859E850E94DCB6A7019601C9
:10DEC0000E94DBB66B017C0120E030E0A9010E94DA
:10DED000B5B787FD11C020E030E040E853E4C7014A
:10DEE000B6010E94B8B9181654F4C12CD12C30E8F0
:10DEF000E32E33E4F32E03C0C12CD12C7601AB8981
:10DF0000BC898D919D91BC8BAB8BBC01882777FD23
:10DF10008095982F0E9457B89B01AC01C501B401B0
:10DF20000E94B8B91816F4F4EF81F88580819181C8
:10DF3000BC01882777FD8095982F0E9457B89B01D8
:10DF4000AC01C501B4010E94B5B787FF0BC0C70182
:10DF5000B6010E9424B8CB0195958795A981BA8115
:10DF60008C9303C0E981FA81108289A19AA1049659
:10DF70009AA389A3A981BA811196BA83A983EF8153
:10DF8000F8853296F887EF830F5F1F4FF4E02F0E6E
:10DF9000311C8B819C8104969C838B83AD81BE81D7
:10DFA0001496BE83AD83E9A1FAA1389709F098CE03
:10DFB0000E94A5B00091F9111091FA112091FB1166
:10DFC0003091FC11601B710B820B930B683873410D
:10DFD0008105910550F00E94A5B06093F9117093EE
:10DFE000FA118093FB119093FC11A2960FB6F8944E
:10DFF000DEBF0FBECDBFDF91CF911F910F91FF907C
:10E00000EF90DF90CF90BF90AF909F908F907F90D8
:10E010006F905F904F903F902F900895CF93DF9334
:10E02000C0915502D0915602109207121092081218
:10E030001092091210920A12209165023091660224
:10E04000409167025091680260E070E08FE793E4CE
:10E050000E94BCB76093FF1170930012809301126D
:10E0600090930212D0935802C093570210920B1251
:10E0700010920C1210920D1210920E126093031255
:10E08000709304128093051290930612249A809143
:10E090000101806180930101809101018062809380
:10E0A00001018091010180648093010187ED8093DB
:10E0B0007A0010927E0010927D0080917E00886030
:10E0C00080937E0080917E00806180937E008091AD
:10E0D0007D00806480937D0080E888BD80916E0023
:10E0E000846080936E006AEF70E080E090E00E94B0
:10E0F000D4B085E090E09093EF118093EE1160E052
:10E100008091F2119091F311DDDB20E030E040EAE4
:10E1100050E40E94B5B787FF0AC08091F211909138
:10E12000F31140969093F3118093F211E8CF80E9B8
:10E1300091E0909356028093550260E080915902DD
:10E1400090915A02BFDB20E030E048EC53E40E949B
:10E15000B8B9181654F48091590290915A02409718
:10E1600090935A0280935902E8CF85E090E0909313
:10E17000F1118093F01161E08091F4119091F5110B
:10E18000A1DB20E030E040EA50E40E94B5B787FF11
:10E190000AC08091F4119091F51140969093F51179
:10E1A0008093F411E8CF80E991E090935802809336
:10E1B000570261E080915B0290915C0283DB20E07A
:10E1C00030E048EC53E40E94B8B9181654F480913A
:10E1D0005B0290915C02409790935C0280935B029B
:10E1E000E8CFDF91CF9108950895109255121092C3
:10E1F0005412E6E5F2E1118210821092531210924D
:10E2000052121092F7112C981092F8119FB7F894AF
:10E21000E2E0F1E080818F7E80839FBF10925312F5
:10E22000109252121092F6119FB7F89480818F7D50
:10E2300080839FBF08952F923F924F925F926F927B
:10E240007F928F929F92AF92BF92CF92DF92EF9286
:10E25000FF920F931F93CF93DF93CDB7DEB7AE97A7
:10E260000FB6F894DEBF0FBECDBF6C8F7D8F8E8F43
:10E270009F8F5EA74DA73CA72BA70E94A5B069A3BF
:10E280007AA38BA39CA32DA53EA5233031051CF4B6
:10E29000EDEFF3E017C0E0E1F4E08191882339F07D
:10E2A0009091C00095FFFCCF8093C600F6CF80917F
:10E2B000C00085FFFCCF15C29091C00095FFFCCF38
:10E2C0008093C60081918111F7CF8091C00085FFB6
:10E2D000FCCF8AE08093C60088DF4DA55EA580E86C
:10E2E00057FF43C08093F61189A19AA1ABA1BCA1AD
:10E2F000898B9A8BAB8BBC8B8D879E87AF87B88BB6
:10E300001D8290E4998FACE1AA8FB6E4BB8F1D8A81
:10E310001E8A1F8A188E20E830E040E050E02983F2
:10E320003A834B835C83F0E84F2E512C612C712C87
:10E330001DA21EA21FA218A631E038A31C861B86B0
:10E34000312C00E010E0212C4DA55EA549505E4E19
:10E350005AA749A78DA59EA5880F991F880F991FB9
:10E360008A5B9D4E9A87898708C0EDA5FEA5E95076
:10E37000FE4E8083B9CF0E94508880913F1288233F
:10E3800009F4DCC0CBDBADA5BEA5B7FF09C030905A
:10E39000401200914112109142122090431206C087
:10E3A000E985FA853080018112812380232D302F69
:10E3B000412F522D6D897E898F89988D0E94B8B921
:10E3C000181624F03D8A0E8B1F8B288E232D302F9C
:10E3D000412F522D6D81798D8A8D9B8D0E94B5B70D
:10E3E00087FD04C03D82098F1A8F2B8EF8A1FF2371
:10E3F00009F451C02C8D3D8D4E8D5F8D632D702F96
:10E40000812F922D0E94B8B918160CF097C00E9467
:10E41000A5B029893A894B895C89621B730B840BEF
:10E42000950B693873418105910508F487C0D301C4
:10E43000C20129813A814B815C81821B930BA40B21
:10E44000B50B4DA55EA5B595A7959795879557FFF3
:10E4500003C08093F61103C0E9A5FAA580830E944A
:10E46000A5B06D877E878F87988B9B01AC018989CA
:10E470009A89AB89BC89281B390B4A0B5B0B2DA3EE
:10E480003EA34FA358A79C8D9D8BAD8DAE8BBE8DAB
:10E49000BF8BEF8DE88F2C8D3D8D4E8D5F8D632D65
:10E4A000702F812F922D0E94B5B787FFF0C20E9476
:10E4B000A5B02D853E854F855889621B730B840B53
:10E4C000950B693873418105910508F4E0C20E94FB
:10E4D000A5B0698B7A8B8B8B9C8BDC01CB012D8556
:10E4E0003E854F855889821B930BA40BB50B4B853A
:10E4F0005C85452B09F011C189819A81AB81BC8172
:10E50000840D951DA61DB71D2DA53EA5B595A795F6
:10E510009795879537FFB7C28093F6112B853C8579
:10E520002F5F3F4F3C872B873C8D3D834D8D498F1F
:10E530005E8D5A8F8F8D8B8F91E098A320E030E015
:10E5400040EA51E46C8D7D8D8E8D9F8D0E94DCB6EE
:10E550009B01AC01632D702F812F922D0E94B8B9C1
:10E56000181694F4E3ECF0E18491882341F0909143
:10E57000C00095FFFCCF8093C6003196F5CF809107
:10E58000C00085FFFCCFADC00E94A5B029A13AA173
:10E590004BA15CA1621B730B840B950B613D774013
:10E5A0008105910508F450C04DA55EA557FF10C028
:10E5B000E090F611F12CEDEBF0E184918823C9F0A5
:10E5C0009091C00095FFFCCF8093C6003196F5CFA7
:10E5D000A9A5BAA5EC90F12CE7EBF0E18491882392
:10E5E00041F09091C00095FFFCCF8093C60031961A
:10E5F000F5CF22E030E0432D502F612F722D82E7BE
:10E6000095E00E949517E3EBF0E18491882341F0B7
:10E610009091C00095FFFCCF8093C6003196F5CF56
:10E620004AE050E0B70182E795E00E94BF16809172
:10E63000C00085FFFCCF8AE08093C6000E94A5B091
:10E6400069A37AA38BA39CA30E94A5B06B017C0154
:10E650000E94A5B089889A88AB88BC882D853E85A4
:10E660004F855889820E931EA41EB51EC818D9085E
:10E67000EA08FB08C60ED71EE81EF91E31E8C316CD
:10E680003FE4D30632E1E306F10490F0E6E9F0E17D
:10E690008491882341F09091C00095FFFCCF809336
:10E6A000C6003196F5CF8091C00085FFFCCF19C020
:10E6B0004B855C858BA59CA5841795070CF05BCEDC
:10E6C000E5E4F0E18491882341F09091C00095FF4A
:10E6D000FCCF8093C6003196F5CF8091C00085FFB6
:10E6E000FCCF8AE08093C600AE960FB6F894DEBFEA
:10E6F0000FBECDBFDF91CF911F910F91FF90EF9093
:10E70000DF90CF90BF90AF909F908F907F906F9051
:10E710005F904F903F902F9008958DA09EA0AFA046
:10E72000B8A4880E991EAA1EBB1E2DA13EA14FA102
:10E7300058A5281B390B4A0B5B0BCA01B90129816B
:10E740003A814B815C810E9450BBA50194010E94DB
:10E75000A8BB240D351D461D571D2431310541052B
:10E76000510504F129013A013DEE431651046104BB
:10E7700071042CF07CEE472E512C612C712C41E859
:10E780004416510461047104DCF08FEF90E0A0E0C6
:10E79000B0E084199509A609B70989839A83AB83E8
:10E7A000BC8312C064E1462E512C612C712C24E1F3
:10E7B00030E040E050E029833A834B835C8304C01F
:10E7C00049825A826B827C82EAE2F1E18491882359
:10E7D00041F09091C00095FFFCCF8093C600319628
:10E7E000F5CF2AE030E0B301A20182E795E00E9474
:10E7F0009C16E5E2F1E18491882341F09091C000FC
:10E8000095FFFCCF8093C6003196F5CF2AE030E02B
:10E8100049815A816B817C8182E795E00E949C1638
:10E82000EEE1F1E18491882341F09091C00095FFE1
:10E83000FCCF8093C6003196F5CF22E030E04D81C9
:10E84000598D6A8D7B8D82E795E00E949517E7E1EF
:10E85000F1E18491882341F09091C00095FFFCCFB5
:10E860008093C6003196F5CF22E030E04D895E8975
:10E870006F89788D82E795E00E9495178091C0009E
:10E8800085FFFCCF8AE08093C6002B853C85233032
:10E8900031050CF431CE69817A818B819C810E9493
:10E8A00057B820E030E040E850E40E948ABA6B019B
:10E8B0007C012D81398D4A8D5B8D6D897E898F8993
:10E8C000988D0E94DBB620ED3FE049E450E40E94C1
:10E8D0008ABA20E030E040E05FE30E948ABA9B0100
:10E8E000AC01C701B6010E94BCB76B017C01C50138
:10E8F000B4010E9457B820E030E04AE754E40E9497
:10E90000BCB74B015C01E1E1F1E18491882341F066
:10E910009091C00095FFFCCF8093C6003196F5CF53
:10E9200022E030E0B701A60182E795E00E9495174A
:10E93000EBE0F1E18491882341F09091C00095FFD4
:10E94000FCCF8093C6003196F5CF22E030E0B501D0
:10E95000A40182E795E00E9495178091C00085FF91
:10E96000FCCF8AE08093C6002AE939E949E15FE3F8
:10E97000C701B6010E948ABA6B017C019B01AC0100
:10E980000E94DCB6A50194010E94BCB76D837E8312
:10E990008F839887A5019401C701B6010E948ABAA6
:10E9A00020E030E040E05EE30E948ABA4B015C0167
:10E9B000EEEFF0E18491882341F09091C00095FF43
:10E9C000FCCF8093C6003196F5CF8091C00085FFC3
:10E9D000FCCF8AE08093C600E8EFF0E184918823C1
:10E9E00041F09091C00095FFFCCF8093C600319616
:10E9F000F5CF22E030E0B701A60182E795E00E9462
:10EA000095178091C00085FFFCCF8AE08093C600F7
:10EA1000E2EFF0E18491882341F09091C00095FFEE
:10EA2000FCCF8093C6003196F5CF22E030E04D81D7
:10EA30005E816F81788582E795E00E9495178091CD
:10EA4000C00085FFFCCF8AE08093C600ECEEF0E1C9
:10EA50008491882341F09091C00095FFFCCF809372
:10EA6000C6003196F5CF22E030E0B501A40182E77F
:10EA700095E00E9495178091C00085FFFCCF8AE049
:10EA80008093C60039CDE9A5FAA5808347CD18A2A9
:10EA900055CD1F920F920FB60F9211240BB60F9205
:10EAA0002F933F934F935F936F937F938F939F9396
:10EAB000AF93BF93EF93FF9380915402811127C0CE
:10EAC0008091F7118093ED11882329F0809102093C
:10EAD000813109F42C9A8091F8118093EC118823EC
:10EAE00041F09FB7F8948091020180618093020108
:10EAF0009FBF8091F6118093EB11882341F09FB75F
:10EB0000F894809102018062809302019FBF9091EE
:10EB1000ED1180915402891728F08091020981310A
:10EB200009F42C989091EC1180915402891740F0CF
:10EB30009FB7F894809102018F7E809302019FBF5E
:10EB40009091EB1180915402891740F09FB7F8948F
:10EB5000809102018F7D809302019FBF80915402BA
:10EB60008F5F8F77809354028091EA1190E0883014
:10EB7000910508F08BC0FC01EE58FF4F0C94C4BB0C
:10EB800010927B0083E480937C0080917A00806403
:10EB900080937A000E94D18781E019C0209178008B
:10EBA000309179008091E6119091E711A091E811E0
:10EBB000B091E911820F931FA11DB11D8093E61141
:10EBC0009093E711A093E811B093E91182E080934C
:10EBD000EA115CC088E080937B0086E480937C002F
:10EBE00080917A00806480937A000E94D18783E0CC
:10EBF000EECF20917800309179008091E2119091D0
:10EC0000E311A091E411B091E511820F931FA11DB2
:10EC1000B11D8093E2119093E311A093E411B0939E
:10EC2000E51184E0D4CF10927B0084E480937C00D3
:10EC300080917A00806480937A000E94D18785E079
:10EC4000C6CF20917800309179008091DE119091AB
:10EC5000DF11A091E011B091E111820F931FA11D6E
:10EC6000B11D8093DE119093DF11A093E011B0935A
:10EC7000E11186E0ACCF0E94D18787E0A8CF109247
:10EC8000EA118091DD118F5F8093DD118091DD119C
:10EC9000803108F460C080913F12811118C08091CA
:10ECA000E6119091E71190934F1280934E1280914C
:10ECB000DE119091DF119093511280935012809148
:10ECC000E2119091E311909345128093441281E0F8
:10ECD00080933F121092DD111092E6111092E7110D
:10ECE0001092E8111092E9111092DE111092DF11CA
:10ECF0001092E0111092E1111092D9111092DA11D4
:10ED00001092DB111092DC111092E2111092E311BB
:10ED10001092E4111092E51180911009909111095F
:10ED20002091030981389E4314F0227001C02160B4
:10ED300020930309809112099091130920910309EE
:10ED400081389E4314F0217001C022602093030992
:10ED500081E080930709FF91EF91BF91AF919F915F
:10ED60008F917F916F915F914F913F912F910F9074
:10ED70000BBE0F900FBE0F901F9018952DEB37E331
:10ED800046E05EE30C948ABA2DEB37E346E05EE39F
:10ED90000C94BCB72DEB37E346E05EE30C94BCB7B4
:10EDA0002DEB37E346E05EE30C948ABA1092A6128C
:10EDB0001092A7121092A8121092A9128AE292EA57
:10EDC00090936F0280936E020895109255121092E4
:10EDD000541210925712109256121092531210920F
:10EDE0005212E4CF1092A6121092A7121092A812FB
:10EDF0001092A9128AEE90E890936F0280936E02AF
:10EE000082E080936D020895FB0160916E02709123
:10EE10006F0270939F1260939E126091A612709180
:10EE2000A71270939D1260939C1262E060936D0232
:10EE300061E07FE970936F0260936E0290939B1282
:10EE400080939A12F0939912E0939812662757FDD7
:10EE50006095762F4093941250939512609396127A
:10EE600070939712C901AA2797FDA095BA2F809396
:10EE7000901290939112A0939212B093931280816A
:10EE80009181AA2797FDA095BA2F8093A6129093FF
:10EE9000A712A093A812B093A9120895CF93DF935D
:10EEA000262FFC01EB5BFF4F40815181EC01CD5BD4
:10EEB000DF4F6881798104960E94F8AB28813981FF
:10EEC000280F311D87FD3A953983288381E090E032
:10EED000DF91CF91089581E090E09093F6128093B6
:10EEE000F51284E190E09093F8128093F7128091EC
:10EEF000FE08853019F460E474E004C0873031F412
:10EF00006BE474E082EB92E10E9431B381E090E027
:10EF10009093F6128093F5128BE290E09093F812A2
:10EF20008093F71266E574E082EB92E10C9431B3C2
:10EF3000CF93DF93FC016491EC012196662331F0BD
:10EF400082EB92E10E9432B3CE01F4CFDF91CF91F8
:10EF50000895EF92FF920F931F93CF93DF93EB01EE
:10EF6000790190E001962CE0289F8001299F100DE7
:10EF700011241092F6121092F5121093F8120093C9
:10EF8000F712642F82EB92E10E9432B3FE0164918A
:10EF9000662331F082EB92E10E9432B32196F6CFE4
:10EFA0006AE382EB92E10E9432B38DE590E09093A8
:10EFB000F6128093F5121093F8120093F712B7012E
:10EFC00082EB92E1DF91CF911F910F91FF90EF9033
:10EFD0000C9431B380911D0991E0892780931D091C
:10EFE000882319F084E395E102C080E395E10C9455
:10EFF000C319CF92DF92EF92FF9285E08093FE08D3
:10F000001092FF0810920009109268121092691273
:10F0100010926A1210926B1210926C1210926D1272
:10F0200010926E1210926F12C12CD12C88E4E82E2F
:10F0300082E4F82EC0927012D0927112E092721295
:10F04000F0927312C0927412D0927512E0927612FE
:10F05000F092771260910A0970910B09625371095D
:10F06000882777FD8095982F0E9457B86093781273
:10F070007093791280937A1290937B12C0927C12D3
:10F08000D0927D12E0927E12F0927F1260938012F5
:10F0900070938112809382129093831260910C0975
:10F0A00070910D0962537109882777FD8095982F1B
:10F0B0000E9457B8609384127093851280938612D1
:10F0C00090938712C0928812D0928912E0928A128D
:10F0D000F0928B1260938C1270938D1280938E122B
:10F0E00090938F1263DE88E894E1FF90EF90DF90B9
:10F0F000CF900C94C319AF92BF92CF92DF92EF9250
:10F10000FF920F931F93CF93DF931F92CDB7DEB77C
:10F110009EEFA92E98E0B92E87E0F501808380E06C
:10F1200090E0A0E0B0E48093F0089093F108A09301
:10F13000F208B093F308198220E030E040EA50E48E
:10F1400060913702709138028091390290913A02B1
:10F150000E94BCB79E012F5F3F4F69017B018C016C
:10F1600024EF38E040EF58E06CEE78E088EE98E06D
:10F170000E94CD58F501108285E99DE890936F02B9
:10F1800080936E0282E080936D021092A61210921C
:10F19000A7121092A8121092A9128EE692E10E9474
:10F1A000C3190F90DF91CF911F910F91FF90EF90B6
:10F1B000DF90CF90BF90AF9008950E94361A0C94C4
:10F1C000D711DF92EF92FF920F931F93CF93DF93AC
:10F1D000D82FF62ED72EC42FE22E61E086EB92E1D7
:10F1E0004E3311F04632A9F40E94DEAD8CE0D89F78
:10F1F000A00111244D5F5F4F0CE010E020E830E0EB
:10F2000060E070E086EB92E10E9435B060E086EB52
:10F2100092E10E94DEAD1092F6121092F5128D2F3F
:10F2200090E001962CE0289FF001299FF00D112419
:10F23000F093F812E093F712CE3311F06C2F01C067
:10F2400060E282EB92E10E9432B3CF2DDD2D11E11D
:10F250001F0D912F9C1BFE016491662331F082EB00
:10F2600092E10E9432B32196F4CFC92FCC2339F01A
:10F2700060E282EB92E10E9432B3C150F7CF6E2D73
:10F2800082EB92E10E9432B360E282EB92E10E9453
:10F2900032B361E086EB92E1DF91CF911F910F9144
:10F2A000FF90EF90DF900C94DEADCF92DF92EF9263
:10F2B000FF920F931F93CF93DF931F92CDB7DEB7CB
:10F2C000E091FF0828E0E29FF0011124E859FD4E8B
:10F2D00080819181A281B3818093E8089093E908AD
:10F2E000A093EA08B093EB0884819581A681B78149
:10F2F0008093EC089093ED08A093EE08B093EF088C
:10F30000198220E030E040E752E460912F027091D2
:10F31000300280913102909132020E94BCB79E016E
:10F320002F5F3F4F69017B018C0124EF38E040EFF4
:10F3300058E06CEE78E088EE98E00E94CD580E948C
:10F34000C86B1092F0081092F1081092F208109217
:10F35000F308198220E030E040E251E46091370286
:10F36000709138028091390290913A020E94BCB7A4
:10F370007B018C0124EF38E040EF58E06CEE78E040
:10F3800088EE98E00E94CD580E94C86B0F90DF91E4
:10F39000CF911F910F91FF90EF90DF90CF90089544
:10F3A000CF92DF92EF92FF920F931F93CF93DF9351
:10F3B0001F92CDB7DEB787E08093FE0880E090E033
:10F3C000A0E0B0E48093F0089093F108A093F208D5
:10F3D000B093F308198220E030E040EA50E46091F5
:10F3E0003702709138028091390290913A020E945E
:10F3F000BCB79E012F5F3F4F69017B018C0124EF59
:10F4000038E040EF58E06CEE78E088EE98E00E943B
:10F41000CD58CCDC8091FF0881508093FF0881306B
:10F4200039F480910009823040F41092000905C03F
:10F43000811103C084E08093FF0837DF0F90DF91D4
:10F44000CF911F910F91FF90EF90DF90CF90089593
:10F45000CF92DF92EF92FF920F931F93CF93DF93A0
:10F460001F92CDB7DEB787E08093FE0880E090E082
:10F47000A0E0B0E48093F0089093F108A093F20824
:10F48000B093F308198220E030E040EA50E4609144
:10F490003702709138028091390290913A020E94AD
:10F4A000BCB79E012F5F3F4F69017B018C0124EFA8
:10F4B00038E040EF58E06CEE78E088EE98E00E948B
:10F4C000CD5874DC8091FF088F5F8093FF088530F2
:10F4D00031F484E08093000981E08093FF08E5DE49
:10F4E0000F90DF91CF911F910F91FF90EF90DF90E0
:10F4F000CF900895CF9382E080936D020E94A5B0D3
:10F500006C507E4F8F4F9F4F6093AC127093AD1233
:10F510008093AE129093AF12389ACAE0409A63E09B
:10F5200070E080E090E00E94D4B0409863E070E02A
:10F5300080E090E00E94D4B0C15081F7CF9108954F
:10F540001092A6121092A7121092A8121092A9124D
:10F5500089E790E890936F0280936E02CBCFCF92B1
:10F56000DF92EF92FF920F931F93CF93DF938091DF
:10F57000A6129091A712A091A812B091A912813061
:10F580009048A105B10540F01092A6121092A71262
:10F590001092A8121092A9126091A6127091A7124F
:10F5A0008091A8129091A91225E030E040E050E04F
:10F5B0000E9486BB8091B01290E0A0E0B0E02817D6
:10F5C00039074A075B0710F42093B012D091B012AC
:10F5D000C0E025E0C22ED12CE12CF12C11E060918D
:10F5E000A6127091A7128091A8129091A912D11120
:10F5F00037C020916D02222369F026E26530710543
:10F600008105910510F446E201C040E264E275E133
:10F610008C2FD7DD8091B11282FD12C020E030E046
:10F6200040E251E46091641270916512809166121B
:10F63000909167120E94B5B787FD77C003E036C18D
:10F640008091A6129091A712A091A812B091A91230
:10F650000597A105B10510F74DDF8CED9CE770C152
:10F66000D13081F520916D02222391F0A7019601FE
:10F670000E9486BB213031054105510519F42AEF5E
:10F680004EE302C02AEF40E26DE175E18C2F99DD77
:10F690008091B11282FFC2CF6091A6127091A71221
:10F6A0008091A8129091A912A70196010E9486BB91
:10F6B000213031054105510509F0B0CF1BDF8CE346
:10F6C0009CE83EC1D23009F0A9CF20916D022223DF
:10F6D00091F0A70196010E9486BB223031054105B9
:10F6E000510519F42AEF4EE302C02AEF40E266E129
:10F6F00075E18C2F66DD8091B11282FF8FCF609112
:10F70000A6127091A7128091A8129091A912A70138
:10F7100096010E9486BB223031054105510509F052
:10F720007DCFE8DE8FE89BE80BC1D33031F08091CC
:10F73000030980FD39C004E072C080916D02882306
:10F74000D1F06091A6127091A7128091A8129091A9
:10F75000A912A70196010E9486BB233031054105FD
:10F76000510519F42AEF4EE302C02AEF40E26FE0A0
:10F7700075E18C2F26DD8091B11282FFD8CF609188
:10F78000A6127091A7128091A8129091A912A701B8
:10F7900096010E9486BB233031054105510539F69B
:10F7A000A9DE80EC99E8CCC0D43011F005E037C078
:10F7B00080916D028823D1F06091A6127091A712FA
:10F7C0008091A8129091A912A70196010E9486BB70
:10F7D000243031054105510519F42AEF4EE302C0EA
:10F7E0002AEF40E264E075E18C2FEBDC8091B112EE
:10F7F00082FFDCCF6091A6127091A7128091A812AF
:10F800009091A912A70196010E9486BB2430310570
:10F810004105510559F66EDE8CE09BE891C0809160
:10F82000030981FF43C00D1711F00F5F3FC08091A6
:10F830006D028823F1F06091A6127091A712809159
:10F84000A8129091A912A70196010E9486BB802F51
:10F8500090E0A0E0B0E0281739074A075B0719F4E9
:10F860002AEF4EE302C02AEF40E269EF74E18C2FE9
:10F87000A8DC8091B11282FFD8CF6091A61270915E
:10F88000A7128091A8129091A912A70196010E9437
:10F8900086BB802F90E0A0E0B0E0281739074A0728
:10F8A0005B0719F627DE86E89AE84AC06091A6123F
:10F8B0007091A7128091A8129091A912A7019601A8
:10F8C0000E9486BB802F90E0A0E0B0E028173907A7
:10F8D0004A075B0788F025E0029FC00111240197C9
:10F8E000AA2797FDA095BA2F8093A6129093A712EE
:10F8F000A093A812B093A9126091A6127091A712BA
:10F900008091A8129091A912A70196010E9486BB2E
:10F910008091B01290E00496422F50E08417950732
:10F920004CF48CEF820F8093B01210936D02DBEFDA
:10F93000D20FCFEFCF5FDF5FC53008F450CE0CC0E1
:10F9400090936F0280936E021092A6121092A712EB
:10F950001092A8121092A912DF91CF911F910F91CE
:10F96000FF90EF90DF90CF9008958DEC9CECACEC85
:10F97000BDE38093641290936512A0936612B093D6
:10F980006712EDCD80E090E0A0E8BFE380936412C1
:10F9900090936512A0936612B0936712E0CD80E059
:10F9A00090E0A0E2B1E48093641290936512A0937A
:10F9B0006612B0936712D3CD8F929F92AF92BF928F
:10F9C000CF92DF92EF92FF921F93CF93DF938091BC
:10F9D000A6129091A712A091A812B091A9128130FD
:10F9E0009048A105B10540F01092A6121092A712FE
:10F9F0001092A8121092A9126091A6127091A712EB
:10FA00008091A8129091A91225E030E040E050E0EA
:10FA10000E9486BB8091B01290E0A0E0B0E0281771
:10FA200039074A075B0710F42093B012D091B01247
:10FA3000C0E035E0C32ED12CE12CF12C43E1842E23
:10FA4000912CA12CB12C11E06091A6127091A712FB
:10FA50008091A8129091A912D11122C020916D021B
:10FA6000222369F026E2653071058105910510F4C5
:10FA700046E201C040E26BED74E18C2FA2DB809185
:10FA8000B11282FF2AC08091A6129091A712A09174
:10FA9000A812B091A9120597A105B105F0F4D1C043
:10FAA000D13009F045C020916D02222391F0A701C9
:10FAB00096010E9486BB213031054105510519F49C
:10FAC0002AEF4EE302C02AEF40E261ED74E18C2F91
:10FAD00078DB8091B11282FD16C08091A6129091C0
:10FAE000A712A091A812B091A9124497A105B1053F
:10FAF00008F483C08092A6129092A712A092A81236
:10FB0000B092A9127AC06091A6127091A71280914A
:10FB1000A8129091A912A70196010E9486BB2130DC
:10FB2000310541055105C9F6E5DC8FEC9CE78CC039
:10FB3000D23081F520916D02222391F0A701960128
:10FB40000E9486BB223031054105510519F42AEF88
:10FB50004EE302C02AEF40E268EC74E18C2F31DB07
:10FB60008091B11282FFB9CF6091A6127091A71255
:10FB70008091A8129091A912A70196010E9486BBBC
:10FB8000223031054105510509F0A7CFB3DC82ECE5
:10FB90009CE75AC0D33009F0A0CF20916D022223F8
:10FBA00091F0A70196010E9486BB233031054105E3
:10FBB000510519F42AEF4EE302C02AEF40E26DEB43
:10FBC00074E18C2FFEDA8091B11282FF86CF6091B2
:10FBD000A6127091A7128091A8129091A912A70164
:10FBE00096010E9486BB233031054105510509F07D
:10FBF00074CF80DC85EB9CE727C06091A6127091E2
:10FC0000A7128091A8129091A912A70196010E94B3
:10FC100086BB8091B01290E00496422F50E084178A
:10FC200095074CF48CEF820F8093B01210936D0205
:10FC3000DBEFD20FCFEFCF5FDF5FC53008F404CF2B
:10FC40000FC058DC8CE395E990936F0280936E02AD
:10FC50001092A6121092A7121092A8121092A91236
:10FC6000DF91CF911F91FF90EF90DF90CF90BF90E9
:10FC7000AF909F908F9008952091030920FF08C0B6
:10FC8000809105139091061390935512809354120E
:10FC900021FF08C08091051390910613909357128D
:10FCA0008093561280910709811108C08091031337
:10FCB00090910413909353128093521280910113E8
:10FCC000909102139093AA088093A9086FD80C947E
:10FCD000F4702091030920FF08C08091FF129091D9
:10FCE0000013909355128093541221FF08C0809105
:10FCF000FF129091001390935712809356128091A7
:10FD00000709811108C08091FD129091FE12909315
:10FD10005312809352128091FB129091FC12909397
:10FD2000AA088093A90842D80C94F4709F92AF92CD
:10FD3000BF92CF92DF92EF92FF920F931F93CF93D8
:10FD4000DF932091C1062F5F2093C1068AE0289F90
:10FD5000E001112430E08091C6069091C706281773
:10FD6000390720F48E01065F1F4F06C00091C806B8
:10FD70001091C9060C0F1D1F54E3E52E59E0F52E16
:10FD80006AE2C62E62E1D62E74E1972EEAE0AE2E2C
:10FD9000B12CC017D10778F56091C2067091C306E7
:10FDA000615071096C1B7D0B7093C5066093C4068E
:10FDB00083E299E00E94B14FFF92EF92DF92CF92DF
:10FDC0001F929F92CE01B5010E945FBB989E900149
:10FDD000999E300D112427503A4F3F932F930E9444
:10FDE0006ABF21968DB79EB708960FB6F8949EBF4E
:10FDF0000FBE8DBFCECF89E093E890936F028093C2
:10FE00006E021092A6121092A7121092A8121092CF
:10FE1000A912DF91CF911F910F91FF90EF90DF908A
:10FE2000CF90BF90AF909F9008959F92AF92BF9256
:10FE3000CF92DF92EF92FF920F931F93CF93DF93B6
:10FE40002091C10621502093C1068AE0289FE0013D
:10FE5000112430E08091C6069091C7062817390713
:10FE600020F48E01065F1F4F06C00091C806109156
:10FE7000C9060C0F1D1FF4E3EF2EF9E0FF2EA7E2D9
:10FE8000CA2EA2E1DA2EB4E19B2E8AE0A82EB12C74
:10FE9000C017D10778F56091C2067091C306615012
:10FEA00071096C1B7D0B7093C5066093C40683E2D9
:10FEB00099E00E94B14FFF92EF92DF92CF921F9292
:10FEC0009F92CE01B5010E945FBB989E9001999EC2
:10FED000300D112427503A4F3F932F930E946ABF51
:10FEE00021968DB79EB708960FB6F8949EBF0FBEA9
:10FEF0008DBFCECF89E093E890936F0280936E021E
:10FF00001092A6121092A7121092A8121092A91283
:10FF1000DF91CF911F910F91FF90EF90DF90CF90E5
:10FF2000BF90AF909F9008957F928F929F92AF92D3
:10FF3000BF92CF92DF92EF92FF920F931F93CF93D6
:10FF4000DF9380912609882309F4C5C080916D0252
:10FF5000811104C08091B11282FFBDC083E299E09B
:10FF60000E9407509093C3068093C2069093C506E3
:10FF70008093C4062AE030E0B9010E945FBB709311
:10FF8000C7066093C606009719F46115710529F438
:10FF90009093C9068093C8060AC03093C90620937F
:10FFA000C806615071097093C7066093C6068091B8
:10FFB000C6069091C706892B29F4E090C806F090F8
:10FFC000C90603C05AE0E52EF12C1092C10667E283
:10FFD00079E087E799E00E943A3B809127098F32C8
:10FFE000A1F41092CA06C0E0D0E094E3C92E99E0D3
:10FFF000D92E06E614E024E1722E3AE0A32EB12CAD
:020000021000EC
:1000000047E2842E49E0942E36C081E08093CA06F0
:10001000EACF6091C2067091C306615071096C1BF2
:100020007D0B7093C5066093C40683E299E00E943D
:10003000B14F80913409811122C09F928F921F93FA
:100040000F931F927F92CE01B5010E945FBB789EF5
:100050009001799E300D112427503A4F3F932F93F2
:100060000E942EBF8DB79EB708960FB6F8949EBF1C
:100070000FBE8DBF2196CE15DF0559F61EC0DF924B
:10008000CF921F930F931F927F92CE01B5010E94D2
:100090005FBB789E9001799E300D112427503A4F16
:1000A0003F932F930E942EBF8DB79EB708960FB631
:1000B000F8949EBF0FBE8DBFDDCF89E093E890938B
:1000C0006F0280936E021092A6121092A7121092E5
:1000D000A8121092A912DF91CF911F910F91FF905A
:1000E000EF90DF90CF90BF90AF909F908F907F90D8
:1000F0000895CF93DF93C1E0D0E0D093F612C09380
:10010000F51289E090E09093F8128093F71269E677
:1001100074E082EB92E10E9431B3D093F612C09367
:10012000F51286E190E09093F8128093F7126AE757
:1001300074E082EB92E10E9431B365E874E082EBF7
:1001400092E10E9431B3D093F612C093F51283E28C
:1001500090E09093F8128093F7126BE874E082EBD2
:1001600092E10E9431B3D093F612C093F51280E36E
:1001700090E09093F8128093F7126DE974E082EBAF
:1001800092E10E9431B3D093F612C093F5128DE341
:1001900090E09093F8128093F71262EB74E082EB98
:1001A00092E10E9431B38091B11282FF10C0809120
:1001B0000209823119F48CEC92E902C08CE395E9D2
:1001C00090936F0280936E02DF91CF9193C9DF917C
:1001D000CF910895EF92FF920F931F93CF93DF93E8
:1001E000C1E0D0E0D093F612C093F51289E090E020
:1001F0009093F8128093F7126EEB74E082EB92E129
:100200000E9431B3D093F612C093F51283E190E0CF
:100210009093F8128093F7126AEC74E082EB92E10B
:100220000E9431B3D093F612C093F5128DE190E0A5
:100230009093F8128093F7126FED74E082EB92E1E5
:100240000E9431B36EEBE62E60E2F62E00E210E083
:1002500024E030E04EE150E060E370E086EB92E1B4
:100260000E9487A88091B11282FF17C082E180931B
:10027000020910921D098BE08093FE0885E99DE834
:1002800090936F0280936E0235D91092A61210924D
:10029000A7121092A8121092A912DF91CF911F916C
:1002A0000F91FF90EF900895EF92FF920F931F939D
:1002B000CF93DF937A01282F30E02F5F3F4F8CE000
:1002C000829F8001839F100D11241092F6121092CC
:1002D000F5121093F8120093F71282EB92E10E944C
:1002E00032B3C2EBD6E1FE016491662331F082EBBA
:1002F00092E10E9432B32196F6CF6AE382EB92E15B
:100300000E9432B38DE590E09093F6128093F5123F
:100310001093F8120093F712C701DF91CF911F914C
:100320000F91FF90EF900C949877CF92DF92EF921D
:10033000FF920F931F93CF93DF9388E090E0909309
:10034000F6128093F5128DE090E09093F81280936E
:10035000F71262EF74E082EB92E10E9431B3809178
:10036000FF08823038F080910009823018F481E073
:10037000809300098091A6129091A712A091A812D3
:10038000B091A91281309048A105B10540F01092BA
:10039000A6121092A7121092A8121092A9126091A0
:1003A000A6127091A7128091A8129091A91225E02F
:1003B00030E040E050E00E9486BB8091B01290E0B7
:1003C000A0E0B0E0281739074A075B0710F4209334
:1003D000B012D091B012C2E075E0C72ED12CE12C42
:1003E000F12C11E0DD2371F0209100096091A6123B
:1003F0007091A7128091A8129091A912211136C074
:1004000001E064C080916D028823A9F08091A6125A
:100410009091A712A091A812B091A91220E205977D
:10042000A105B10510F44EE301C040E26EE772E1B0
:100430008C2F0E94E1788091B11282FFD5CF8091FC
:10044000A6129091A712A091A812B091A912059797
:10045000A105B10548F64ED8DF91CF911F910F91BC
:10046000FF90EF90DF90CF900C94287AD13069F50F
:1004700020916D02222399F0A70196010E9486BB6C
:10048000213031054105510519F420E24EE302C047
:1004900020E240E269E772E18C2F0E94E1788091CE
:1004A000B11282FF4AC06091A6127091A71280918A
:1004B000A8129091A912A70196010E9486BB213033
:1004C000310541055105C9F58CC002E00D1336C058
:1004D00020916D022223B9F0A70196010E9486BBEC
:1004E000802F90E0A0E0B0E0281739074A075B07AB
:1004F00019F420E24EE302C020E240E262E772E13A
:100500008C2F0E94E1788091B11282FF17C0609118
:10051000A6127091A7128091A8129091A912A7011A
:1005200096010E9486BB802F90E0A0E0B0E02817E3
:1005300039074A075B0711F460C002E00F5F609162
:10054000A6127091A7128091A8129091A912A701EA
:1005500096010E9486BB802F90E0A0E0B0E02817B3
:1005600039074A075B0788F025E0029FC001112484
:100570000197AA2797FDA095BA2F8093A612909372
:10058000A712A093A812B093A9126091A61270911D
:10059000A7128091A8129091A912A70196010E941A
:1005A00086BB8091B01290E00496422F50E08417F1
:1005B00095074CF48CEF820F8093B01210936D026C
:1005C000DBEFD20FCFEFCF5FDF5FC53008F40ACF8C
:1005D000DF91CF911F910F91FF90EF90DF90CF901F
:1005E00008950E947A7ADF91CF911F910F91FF9029
:1005F000EF90DF90CF900C94D0790E947A7ADF91BF
:10060000CF911F910F91FF90EF90DF90CF900C94BE
:100610007B782F923F924F925F926F927F928F9250
:100620009F92AF92BF92CF92DF92EF92FF920F9381
:100630001F93CF93DF93CDB7DEB7A9970FB6F8948A
:10064000DEBF0FBECDBF80916D02811104C08091CD
:10065000B11282FF0FC32091C1063AE0239FF0013F
:100660001124FAA3E9A330E08091C6069091C70651
:100670002817390738F429A13AA1265F3F4F38A33C
:100680002F8F0AC08091C8069091C906E9A1FAA1EE
:10069000E80FF91FF8A3EF8F8091A6129091A7128F
:1006A000A091A812B091A91281309048A105B1057E
:1006B00040F01092A6121092A7121092A812109257
:1006C000A9126091A6127091A7128091A812909120
:1006D000A91225E030E040E050E00E9486BB809106
:1006E000B01290E0A0E0B0E0281739074A075B0796
:1006F00010F42093B0122090B012312CF5E0CF2EE0
:10070000D12CE12CF12C8091C106811150C0222006
:1007100019F12CE0329EC0011124FC013396FCA398
:10072000EBA39C01245F3F4F3EA32DA3832D90E0BC
:1007300001962CE0289FF001299FF00D1124F8A7C5
:10074000EFA389A09AA011E031E0320D39A7422C25
:10075000512C612C712C6CC080916D028823A9F002
:100760008091A6129091A712A091A812B091A912FF
:1007700026E20597A105B10510F446E201C040E26A
:100780006AE472E1832D0E94E1788091B11282FFC8
:10079000C0CF8091A6129091A712A091A812B091FB
:1007A000A9120597A105B10508F0B3CF53C22110D6
:1007B000B0CF80916D028823A9F08091A61290910C
:1007C000A712A091A812B091A91220E20597A10545
:1007D000B10510F44EE301C040E261E472E1832D03
:1007E0000E94E1788091B11282FF93CF8091A6128E
:1007F0009091A712A091A812B091A9120597A105F6
:10080000B10508F086CF0E947A7A0FDB33C280915F
:10081000C2069091C3060197881999099093C5065D
:100820008093C406121551F01F5FFFEF8F1A9F0AC5
:100830002F8D38A18216930650F3B9C080916D02B6
:10084000882309F49DC06091A6127091A71280912F
:10085000A8129091A912A70196010E9486BBC4011B
:100860006AE070E0241535054605570509F054C0C7
:100870000E945FBB44E1489F5001499FB00C112486
:10088000C50187509A4F5C01FC0180818111138A58
:1008900061E086EB92E10E94DEAD0CE010E020E822
:1008A00030E04BA15CA160E070E086EB92E10E9439
:1008B00035B060E086EB92E10E94DEAD1092F61258
:1008C0001092F5122DA13EA13093F8122093F71249
:1008D00060E282EB92E10E9432B3850133E1A30E24
:1008E0008A2D801BF80161918F01662329F082EB2C
:1008F00092E10E9432B3F4CF182F112339F060E255
:1009000082EB92E10E9432B31150F7CF61E086EBA7
:1009100092E10E94DEAD34C00E945FBBF4E1F89F1B
:100920008001F99F100D112407501A4FF8018081A2
:100930008111138A1092F6121092F5122FA138A588
:100940003093F8122093F71260E282EB92E10E945A
:1009500032B358010D5E102F1A19F50161915F0134
:10096000662329F082EB92E10E9432B3F4CF112387
:1009700039F060E282EB92E10E9432B31150F7CF7E
:100980008091B11282FF0DC16091A6127091A712E1
:100990008091A8129091A912A70196010E9486BB8E
:1009A000241535054605570509F0FBC0FCC04091EC
:1009B000C6065091C7066091A6127091A712809149
:1009C000A8129091A9124115510509F463C0209114
:1009D000C8063091C906232B09F45CC02091C106DA
:1009E00030E024173507B8F5121156C020916D027A
:1009F0002223B9F0A70196010E9486BB812F90E0C7
:100A0000A0E0B0E0281739074A075B0719F420E295
:100A10004EE302C020E240E267E372E1832D0E94D0
:100A2000E1788091B11282FF37C06091A612709177
:100A3000A7128091A8129091A912A70196010E9475
:100A400086BB812F90E0A0E0B0E0281739074A0765
:100A50005B0711F5FBC02417350709F054C01211CC
:100A60001BC020916D022223A1F1A70196010E94D3
:100A700086BB812F90E0A0E0B0E0281739074A0735
:100A80005B0719F426E246E202C026E240E262E396
:100A900072E11CC0121511F01F5F35C020916D026C
:100AA0002223B9F0A70196010E9486BB812F90E016
:100AB000A0E0B0E0281739074A075B0719F426E2DF
:100AC00046E202C026E240E26DE272E1832D0E941E
:100AD000E1788091B11282FFDFCF6091A612709110
:100AE000A7128091A8129091A912A70196010E94C5
:100AF00086BB812F90E0A0E0B0E0281739074A07B5
:100B00005B0751F6A7C06091A6127091A712809161
:100B1000A8129091A912A70196010E9486BB812F6D
:100B200090E0A0E0B0E0281739074A075B0788F09B
:100B300035E0139FC00111240197AA2797FDA095C6
:100B4000BA2F8093A6129093A712A093A812B093E5
:100B5000A9126091A6127091A7128091A81290918B
:100B6000A912A70196010E9486BB8091B01290E065
:100B70000496422F50E08417950764F48CEF820F9F
:100B80008093B01241E040936D02EBEF2E2E220EC7
:100B900033243A943394239484E0831508F0B3CD3E
:100BA00069C019A542CE0E947A7A809102098231E9
:100BB00021F483E292E10E94C3196091C40683E2AA
:100BC00099E00E94B14F87E299E09F938F938CE167
:100BD00092E19F938F938E010F5F1F4F1F930F938F
:100BE0000E94A6BFE4E3F9E00F900F900F900F90E2
:100BF0000F900F908191882339F09091C00095FF5C
:100C0000FCCF8093C600F6CF8091C00085FFFCCF5B
:100C10008AE08093C6007E01F5E0EF0EF11CF7013B
:100C20008081882349F0992787FD90950E948EBE88
:100C3000F70181937F01F3CFC8010E94501988E129
:100C400092E10E94C3190E94D67614C00E947A7A5B
:100C50006DD810C00E947A7A85E99DE890936F0262
:100C600080936E021092A6121092A7121092A812F0
:100C70001092A912A9960FB6F894DEBF0FBECDBF91
:100C8000DF91CF911F910F91FF90EF90DF90CF9068
:100C9000BF90AF909F908F907F906F905F904F909C
:100CA0003F902F900895CF93DF93FC01E95BFF4FB6
:100CB0002081EC012496211105C081E08083CE01C2
:100CC0000E947EADCE01DF91CF910C94B1ADEF9239
:100CD000FF920F931F9361E081E40E9485B261E06F
:100CE00081E40E94BEB282EB92E1DDDF63E178E154
:100CF00086EB92E10E946BAC61E086EB92E10E9490
:100D0000DEAD0091B8121091B9122091B612309157
:100D1000B71240E050E060E070E086EB92E10E94A4
:100D200035B061E086EB92E10E94DEAD86EB92E1A8
:100D30000E94B5AD8111DACF82EB92E1B4DFAEE76C
:100D4000EA2EACE1FA2E00E410E020E130E040E0D1
:100D500050E060E070E086EB92E10E9487A886EBAD
:100D600092E10E94B5AD8111EACF1F910F91FF90E2
:100D7000EF900895AF92BF92CF92DF92EF92FF92E1
:100D80000F931F93CF93DF935C016B01C2EBEC2EAB
:100D9000C2E1FC2EF701268137812552310905EF8A
:100DA00012E1F80111821082C7EFD2E13983288362
:100DB00063E178E186EB92E10E946BACC5010E9491
:100DC00098776AE3C7010E9432B3F7018681978161
:100DD00085972DE530E0F80131832083998388835E
:100DE000B601C701DF91CF911F910F91FF90EF9056
:100DF000DF90CF90BF90AF900C9431B32091FA1256
:100E000021110AC044E150E0BC0180E792E00E9459
:100E10001FBF82E080936D0208952091FA12211184
:100E20000AC044E150E0BC0180E792E00E94B5BEF8
:100E300082E080936D020895CF93DF93109225098D
:100E400083E299E00E949C4F0E943E6C81EB94E10A
:100E50000E94C319809108118823F9F0109208119B
:100E6000C091AB08D0E0CC0FDD1FCC5ADD4E6881BD
:100E70007981882777FD8095982F0E9457B8209117
:100E80004702309148024091490250914A020E9423
:100E9000B8B9181614F4198218828DEA94E10E94E8
:100EA000C3190E94D67683EA94E1B7DF0E94A5B009
:100EB0006093CC067093CD068093CE069093CF06B8
:100EC00081E08093FE08DF91CF910895CF92DF9269
:100ED000EF92FF928091050980FD44C092E09093CB
:100EE000FE0890910409992339F087FF28C01092D9
:100EF00005098EE994E121C0C0901609D090170928
:100F0000E0901809F090190920E030E0A901C7012C
:100F1000B6010E94B5B7882391F0A70196016091B0
:100F2000F0087091F1088091F2089091F3080E9406
:100F3000B5B7882321F089E994E10E94C319109282
:100F4000160910921709109218091092190983E2D4
:100F500099E00E94B64A8CE894E1FF90EF90DF9010
:100F6000CF905BCFFF90EF90DF90CF90089583E21A
:100F700099E00E94BD4A83E08093FE0880910509B4
:100F800080FF03C087E592E102C08FE492E145CF84
:100F900044DF81E08093FA120C94D6761092FA1214
:100FA0000895CF92DF92EF92FF92CF93C6B1C6FB26
:100FB000CC27C0F981E0C827349BC260C090AC1236
:100FC000D090AD12E090AE12F090AF120E94A5B09A
:100FD000C616D706E806F90610F4329B39C0C0934E
:100FE000B1128091B11281709091B11291FD826025
:100FF0009091AB12891721F18130F1F028F0823005
:1010000089F08330A1F01CC0913021F49091AA1294
:101010009F5F05C09230A1F49091AA1291509093D5
:10102000AA120EC0992391F3933051F4F5CF923068
:1010300069F3913029F4F0CF933041F3992361F3B0
:101040008093AB12CF91FF90EF90DF90CF900895F7
:10105000C460C5CF3CDE60E08FE10E9485B260E0F5
:1010600081E20E9485B260E081E30E9485B2469AE7
:10107000449A60E083E20E9485B2429A9FB7F89456
:10108000EBE0F1E08081816080839FBF8091090166
:10109000809581708093A51284DF1092AA12089522
:1010A000CF92DF92EF92FF92CF93DF937ADF80911E
:1010B0000901817091E089272091A5128217E1F042
:1010C00082E080936D02809109018170892780936D
:1010D000A512FDDD8091A512882339F083E299E005
:1010E0000E94EF498AE092E106C083E299E00E9403
:1010F000B24A8DEF91E191DEC090A112D090A21280
:10110000E090A312F090A4120E94A5B0C616D706D4
:10111000E806F90608F0C3C04091AA12442361F121
:1011200081E080936D02552747FD5095652F752FFF
:101130008091A6129091A712A091A812B091A91225
:10114000840F951FA61FB71F8093A6129093A71216
:10115000A093A812B093A9121092AA120E94A5B04F
:101160006856754C8F4F9F4F609358127093591269
:1011700080935A1290935B128091B11282FF0EC03D
:101180000E94A5B06856754C8F4F9F4F60935812C0
:101190007093591280935A1290935B1280910713A7
:1011A0008F5F8093071382EB92E17DDDCDE7D0E086
:1011B00063E178E186EB92E10E946BACD093F6128A
:1011C000C093F5121092F8121092F7128091071343
:1011D00080FF02C061E001C060E086EB92E10E9406
:1011E000DEAD4FE350E06FE770E086EB92E10E94E6
:1011F000C3AD61E086EB92E10E94DEADE0916E024C
:10120000F0916F02199580916D02811107C0809154
:10121000FE089BEF980F943068F007C086EB92E1D0
:101220000E94B5AD8111C4CFF2CFC1E08C3018F46B
:10123000C0E001C0C1E0C0905812D0905912E090B7
:101240005A12F0905B120E94A5B0C616D706E806A7
:10125000F90648F480916E0290916F028A52924A88
:1012600011F0CC23B1F080916D02882319F08150E8
:1012700080936D020E94A5B06C597F4F8F4F9F4F96
:101280006093A1127093A2128093A3129093A41260
:1012900006C00E94D67682E080936D02E4CFDF9193
:1012A000CF91FF90EF90DF90CF9008958091B11291
:1012B00082FB882780F90895FC01808190E02AE074
:1012C00030E0B9010E9473BB482FCB01B9010E94E5
:1012D00073BB805D80935C12405D40935D12109201
:1012E0005E128CE592E1089520E030E040E251E4A6
:1012F000FC0160817181828193810E948ABA0E947F
:1013000024B877FD02C02BE201C02DE220935C12CD
:101310009B0177FF04C022273327261B370BC90107
:1013200068EE73E00E9473BBCB01EAE0F0E0BF011E
:101330000E9473BB805D80935D12C90164E670E01A
:101340000E9473BBCB01BF010E9473BB805D809381
:101350005E12C901BF010E9473BB282FCB01BF01E0
:101360000E9473BB805D80935F128EE28093601257
:10137000205D20936112109262128CE592E1089533
:10138000CF92DF92EF92FF920F931F938091A6125C
:101390009091A712A091A812B091A9120097A1054F
:1013A000B10509F486C020910209BC01882777FDA8
:1013B0008095982F223139F40E9457B82DEC3CECDF
:1013C0004CEC5DE30AC00E9457B820916412309142
:1013D000651240916612509167120E948ABA9B0171
:1013E000AC016091F0087091F1088091F208909141
:1013F000F3080E94DCB66093F0087093F1088093C4
:10140000F2089093F30820E030E0A9016091F00821
:101410007091F1088091F2089091F3080E94B5B79D
:1014200087FF08C01092F0081092F1081092F2089D
:101430001092F30860910E0970910F09882777FDCB
:101440008095982F0E9457B86B017C019B01AC01DD
:101450006091F0087091F1088091F2089091F30882
:101460000E94B8B9181644F4C092F008D092F1085E
:10147000E092F208F092F3081092A6121092A712CE
:101480001092A8121092A9129BEAC92E98E0D92EA8
:10149000E12CF12C00E810E424EF38E040EF58E0B4
:1014A0006CEE78E088EE98E00E94CD5881E0809361
:1014B0006D0280916D02882339F080EF98E014DF8F
:1014C000BC018EE295E156DC8091B11282FF17C01B
:1014D0000E947A7A80910209823119F48CEC92E9A7
:1014E00002C08FEA9AE790936F0280936E02109287
:1014F000A6121092A7121092A8121092A9121F9170
:101500000F91FF90EF90DF90CF900895BF92CF9210
:10151000DF92EF92FF920F931F93CF93DF931F926F
:10152000CDB7DEB78091A6129091A712A091A81214
:10153000B091A9120097A105B10509F443C0BC01FF
:10154000882777FD8095982F0E9457B820916412C4
:101550003091651240916612509167120E948ABACA
:101560009B01AC016091F4087091F5088091F60838
:101570009091F7080E94DCB66093F4087093F50828
:101580008093F6089093F7081092A6121092A71273
:101590001092A8121092A912BB24B394B982CE0162
:1015A00001966C01E12CF12C00EA11E424EF38E003
:1015B00040EF58E06CEE78E088EE98E00E94CD585D
:1015C000B0926D0280916D02882339F084EF98E02B
:1015D0008BDEBC0180EF94E1CDDB8091B11282FF04
:1015E00010C00E947A7A8FEA9AE790936F028093F4
:1015F0006E021092A6121092A7121092A8121092C8
:10160000A9120F90DF91CF911F910F91FF90EF9052
:10161000DF90CF90BF900895CF92DF92EF92FF922C
:101620000F931F93CF93DF931F92CDB7DEB78091B7
:10163000A6129091A712A091A812B091A91200979A
:10164000A105B10509F442C0BC01882777FD80954A
:10165000982F0E9457B820916412309165124091E2
:101660006612509167120E948ABA9B01AC01609188
:10167000F4087091F5088091F6089091F7080E949F
:10168000DCB66093F4087093F5088093F6089093A5
:10169000F7081092A6121092A7121092A812109298
:1016A000A9121982CE0101966C01E12CF12C00EAFD
:1016B00011E424EF38E040EF58E06CEE78E088EE7B
:1016C00098E00E94CD5881E080936D0280916D0278
:1016D000882339F084EF98E007DEBC0187EE94E1BF
:1016E00049DB8091B11282FF10C00E947A7A8FEAA2
:1016F0009AE790936F0280936E021092A612109256
:10170000A7121092A8121092A9120F90DF91CF91F8
:101710001F910F91FF90EF90DF90CF900895CF929F
:10172000DF92EF92FF920F931F938091A6129091F8
:10173000A712A091A812B091A9120097A105B10516
:1017400009F474C0BC01882777FD8095982F0E940A
:1017500057B82091641230916512409166125091F1
:1017600067120E948ABA2091EC083091ED084091EE
:10177000EE085091EF080E94DCB66B017C0120E07E
:1017800030E0A9010E94B5B787FD09C0C092EC08FE
:10179000D092ED08E092EE08F092EF0808C01092A7
:1017A000EC081092ED081092EE081092EF0860918C
:1017B0000C0970910D09882777FD8095982F0E945C
:1017C00057B86B017C019B01AC016091EC087091F2
:1017D000ED088091EE089091EF080E94B8B91816B4
:1017E00044F4C092EC08D092ED08E092EE08F0923A
:1017F000EF081092A6121092A7121092A81210923F
:10180000A9125BEAC52E58E0D52EE12CF12C00EF91
:1018100011E424EF38E040EF58E06CEE78E088EE19
:1018200098E00E94CD5881E080936D0280916D0216
:10183000882339F08CEE98E057DDBC0185EE94E109
:1018400099DA8091B11282FF10C00E947A7A8FEAF1
:101850009AE790936F0280936E021092A6121092F4
:10186000A7121092A8121092A9121F910F91FF9027
:10187000EF90DF90CF900895CF92DF92EF92FF929A
:101880000F931F938091A6129091A712A091A81276
:10189000B091A9120097A105B10509F474C0BC016B
:1018A000882777FD8095982F0E9457B82091641261
:1018B0003091651240916612509167120E948ABA67
:1018C0002091E8083091E9084091EA085091EB082E
:1018D0000E94DCB66B017C0120E030E0A9010E948F
:1018E000B5B787FD09C0C092E808D092E908E09238
:1018F000EA08F092EB0808C01092E8081092E90894
:101900001092EA081092EB0860910A0970910B0995
:10191000882777FD8095982F0E9457B86B017C012E
:101920009B01AC016091E8087091E9088091EA0898
:101930009091EB080E94B8B9181644F4C092E808D8
:10194000D092E908E092EA08F092EB081092A61211
:101950001092A7121092A8121092A9127BEAC72E19
:1019600078E0D72EE12CF12C00EF11E424EF38E0E1
:1019700040EF58E06CEE78E088EE98E00E94CD5899
:1019800081E080936D0280916D02882339F088EEAA
:1019900098E0AADCBC0183EE94E1ECD98091B1120D
:1019A00082FF10C00E947A7A8FEA9AE790936F02C2
:1019B00080936E021092A6121092A7121092A81293
:1019C0001092A9121F910F91FF90EF90DF90CF908E
:1019D000089520E030E040E251E4FC016081718133
:1019E000828193810E948ABA0E9424B8FB0177FD0C
:1019F0002FC0CB0168EE73E00E9473BBCB012AE0DD
:101A000030E0B9010E9473BB805D80935C12CF010E
:101A100064E670E00E9473BBCB01B9010E9473BB06
:101A2000805D80935D12CF01B9010E9473BB482F86
:101A3000CB01B9010E9473BB805D80935E128EE280
:101A400080935F12405D409360121092611235C026
:101A50002DE220935C12EE27FF27E61BF70BCF0148
:101A600068EE73E00E9473BBCB012AE030E0B9015D
:101A70000E9473BB805D80935D12CF0164E670E0CD
:101A80000E9473BBCB01B9010E9473BB805D809340
:101A90005E12CF01B9010E9473BB482FCB01B9017F
:101AA0000E9473BB805D80935F128EE28093601210
:101AB000405D40936112109262128CE592E10895AC
:101AC000FC0180819181843691055CF064E670E0D0
:101AD0000E9473BBCB016AE070E00E9473BB805D23
:101AE00001C080E280935C12808191818A309105EF
:101AF0005CF02AE030E0B9010E9473BBCB01B90170
:101B00000E9473BB805D01C080E280935D12808182
:101B100091816AE070E00E9473BB805D80935E12E9
:101B200010925F128CE592E10895CF92DF92EF92CE
:101B3000FF920F931F93CF93DF938091FE08813024
:101B400011F41092FE088091A6129091A712A09114
:101B5000A812B091A91281309048A105B10540F0BA
:101B60001092A6121092A7121092A8121092A91207
:101B70006091A6127091A7128091A8129091A9125B
:101B800025E030E040E050E00E9486BB8091B0123A
:101B900090E0A0E0B0E0281739074A075B0710F48F
:101BA0002093B012D091B012C0E011E0A5E0CA2E8F
:101BB000D12CE12CF12CDD2371F0209102096091F0
:101BC000A6127091A7128091A8129091A9122131AA
:101BD00009F035C22EC080916D028823A9F0809152
:101BE000A6129091A712A091A812B091A91226E274
:101BF0000597A105B10510F446E201C040E261EC91
:101C000076E18C2F0E94E1788091B11282FFD5CFCE
